:020000040000FA
:06000000020A3F0201B0FC
:03002B000209EDDA
:0300330002068240
:030043000208AE02
:03004B0002074C5D
:03005300020103A4
:03005B0002075B3E
:030063000207672A
:03006B0002066822
:1000830002014C0101FF01010503010F10FEFF03F3
:100093000003000300030003000300030003000345
:1000A3000005000A00140028004F009E00000062B3
:1000B3001362136213621324121E126213011F00D0
:1000C300000000631F000000000C0000000C000192
:1000D300D904FF0400010200F51100000068126456
:1000E300000202000800000502071E02051E020AA4
:1000F30003B80B02803E0103320002F4FF02020642
:10010300C0E074F21203C2E5A7F8E5A1F958541050
:100113006008121A6A53A1EF802AE8A2E0C0D0E96E
:10012300A2E092F012098E158182F0501790619827
:10013300E0F890157DE0C398A2D265D0335002E871
:10014300F053A1FE7F01020479C0E074F21203C2EE
:100153009061A4E0F8759B00E59158540860087518
:1001630091F7121AAC802AE59158541060087591E2
:10017300EF121AB2801BE8A2E0C0D0E591A2E09290
:10018300F012098E158182F05007E0C2E0F0121BD5
:10019300D29061A3E0F8E5E9585404600E121BA85D
:1001A30075E9FB906193E0A2E640F28097C0E074AA
:1001B300F21203C29061A5E0F8E5BF58540460064B
:1001C30053BFFB121BEA020147C3E498F8E499F911
:1001D30012020D8026C3E49AFAE49BFBE920E7E9C7
:1001E30012020DE498F8E499F922C3E498F8E4992B
:1001F300F912020DE498F8E499F9C3E49AFAE49B3E
:10020300FB22EB20E7CFE920E7E0B90010BB0008B1
:10021300E88AF084F8AAF022E4FBC8FA22EB702201
:100223007B10C833C8C933C9335007C39AC3DBF241
:1002330080069A50012ADBEAC833F4C8C933F4C9EB
:10024300FA2275F008E4C833C8C933C933C99AC957
:100253009B5004C92AC93BD5F0ECFBC833F4C8E46E
:10026300C9FA22080808EAC0E0EBC0E086F0E7A478
:10027300FA180986F0E7A42AFA180986F0E7A42AEF
:10028300FA180986F0E7A42AFA1986F0E7A4FBE531
:10029300F02AFA190886F0E7A42BFBE5F03AFA19DD
:1002A3000886F0E7A42BFBE5F03AFA18180986F064
:1002B300E7A4C5F02BFBE43AFA1908E7C5F0C6A496
:1002C30026F6E5F03BFBE43AFA1886F0E7A4F6E5F8
:1002D300F00826F6E43B08F6E43A08F6D0E0FBD053
:1002E300E0FA22E4CFC0E0E4CEC0E0E4CDC0E0E435
:1002F300CCC0E075F020C3E633F608E633F608E633
:1003030033F608E633F6181818EC33FCED33FDEE3C
:1003130033FEEF33FFC3EC9709ED9709EE9709EF2F
:1003230097191919400FFFEC97FC09ED97FD09EE9A
:1003330097FE191906D5F0BEECF709EDF709EEF7AC
:1003430009EFF7191919D0E0FCD0E0FDD0E0FED099
:10035300E0FF222510C582C0E0E51134FFC583C04C
:10036300E0E510C3958224F810AF088583118582D8
:10037300108008858311858210D2AFCEF0A3E520CB
:10038300F0A37808E608F0A3DEFAEFF0A3E58124F2
:10039300FAF8E608F0A3E608F0A3E608F0A30808D5
:1003A300E608F0A3E608F0A315811581D0E0FED09E
:1003B300E0F8158115811581E8C0E0EEC0E022C0A8
:1003C300D02510C582C0E0E51134FFC583C0E0E548
:1003D30010C3958224F310AF0885831185821080A2
:1003E30008858311858210D2AFC8F0A3E9F0A3EA90
:1003F300F0A3EBF0A37908E709F0A3D8FAECF0A394
:10040300EDF0A3EEF0A3EFF0A3D0E0F0A3D0E0F083
:10041300A3D0E0F0A3E520F0A3E5F0F0A322120AB5
:10042300A1B90003020463E49002FF782E791880D7
:1004330002F0A3D8FCD9FA901A2CAA82AB839000BD
:1004430086787E79018015E493A3AC82AD838A829A
:100453008B83F0A3AA82AB838C828D83D8E9D9E7FF
:1004630075828C7583C5740312051D75827275833D
:100473001E740012051D851183851082E0C0E0A360
:10048300E0F9A3E0FAA3E0FBA37808E0F608A3DF12
:10049300FAE0FCA3E0FDA3E0FEA3E0FFA3E0C0E0DD
:1004A300A3E0C0E0A3E0F5D0A3E0F520A3E0A3F52B
:1004B300F010AF088583118582108008858311852C
:1004C3008210D2AFD082D083D0E0F8D0E032D08394
:1004D300D082ECC0E0EDC0E0E493A3FCE493A3FD81
:1004E300ED4C600D1205F3EC24FFFCED34FFFD80B1
:1004F300EFE493A3FCE493A3FDED4C600D1206F728
:10050300EC24FFFCED34FFFD80EFD0E0FDD0E0FCF8
:10051300E493A3C0E0E493C0E022C0F0F5F0E59FCC
:100523005407C0E0E59F54F845F0D0F0F59FE4731D
:10053300859FF053F0F8D0E045F0F59F22D083D0AB
:1005430082E59F5407C0E0E493C0E0740193C0E0E8
:100553007402935407C0F0F5F0E59F54F845F0D0CA
:10056300F0F59F22D083D082E9C0E0E493A3C38651
:10057300F0C5F095F0F908E493A386F0C5F095F083
:10058300700BE493A3C3994005E9048002A3E475C7
:10059300F002A42582F582E5F03583F583D0E0F9F6
:1005A300E493A3C0E0E493C0E02285118385108225
:1005B300E0A3FEE0A3F5207808E0A3F608DFFAE065
:1005C300A3FFE0A3C0E0E0A3C0E0E0A3C0E0E0A39A
:1005D300C0E0E0A3C0E010AF0885821085831180DE
:1005E30008858210858311D2AFD083D08202053370
:1005F300C0E0C3E49396087401939618400FE49304
:1006030066700808740193661870007019A3A3C379
:10061300E49396087401939618A3A3400DD0E0D0F9
:10062300E0D0E002050DA3A3A3A3A3A3D0E022D0AF
:1006330083D082C5F0E493A3C5F0C395F0F5F0E44D
:1006430093A3C395F04005E5F0048001E475F0023F
:10065300A42582F582E5F03583F583E493A3C0E016
:10066300E493C0E022C0E074F21203C2E589A2E180
:10067300500312192C758900C2C57F01020479C089
:10068300E074F21203C2E58BA2E0500312192C7539
:100693008B00C2E880E47404800474028000CCC040
:1006A300E0EDC0E0E510C39CCCAD1150011D10AFCF
:1006B300068C108D1180068C108D11D2AF12079508
:1006C300D0E0FDD0E0FC2274028000CCC0E0EDC09D
:1006D300E0E510C39CCCAD1150011D10AF068C108A
:1006E3008D1180068C108D11D2AF120773D0E0FDEF
:1006F300D0E0FC22C0E0C0F088F0E4936670080804
:1007030074019366187000A8F0A3A3700BD0F0D007
:10071300E0D0E0D0E002050DA3A3D0F0D0E022D0DA
:1007230083D082CCC0E0E493A360061207D5147093
:10073300FAE493A360061208C51470FAD0E0FCE44F
:1007430093A3C0E0E493C0E022C0E074F21203C2BA
:100753001219B07F01020479C0E074F21203C212CD
:1007630019B680EFC0E074F21203C21219BC80E321
:10077300CAC0E0E493A3C582CCC582C583CDC5833B
:10078300F0A3C582CCC582C583CDC583DAE5D0E0AD
:10079300CA22CAC0E0E0A3C582CCC582C583CDC549
:1007A30083F0A3C582CCC582C583CDC583DAE6D0E9
:1007B300E0CA22C008C3E096F50808A3E096420801
:1007C30008A3E096420808A3E09645087001D3D039
:1007D3000822C0E0E493A3D39C5010E493A3C39CEA
:1007E300400AD0E0D0E0D0E002073FA3A3A3D0E0CB
:1007F300227009080808226016181818C6C333C6E1
:1008030008C633C608C633C608C633C6D5E0EA22CF
:100813007404800A74038006740280027401C0E0C9
:10082300F40412082ED0E0120A7C222510F582105F
:10083300AF08F510400215118008F510400215119C
:10084300D2AF85118322C0D0251010AF08F5105008
:100853000205118008F51050020511D2AFD0D02245
:10086300BB0102E722C082C08389828A83BB000363
:10087300E08002E493D083D082226016080808C681
:10088300C313C618C613C618C613C618C613C6D5CF
:10089300E0EA22C3E0C696F608A3E0C696F608A3EC
:1008A300E0C696F608A3E0C696F622C0E074F212FC
:1008B30003C2C2C0E5D1A2E450031219E67F0102CC
:1008C3000479C0E0E493A36C7009D0E0D0E0D0E0F9
:1008D30002073FA3A3D0E022251010AF08F5104074
:1008E3000215118008F51040021511D2AF22E066FF
:1008F300701008A3E066700A08A3E066700408A3FA
:10090300E06622C3E09608A3E09608A3E09608A356
:10091300E096A2D265D03322C3E096F008A3E09616
:10092300F008A3E096F008A3E096F022E026F00892
:10093300A3E036F008A3E036F008A3E036F022E0A7
:1009430026F608A3E036F608A3E036F608A3E03659
:10095300F622E627F60809E637F60809E637F60829
:1009630009E637F622E657F60809E657F60809E6D8
:1009730057F60809E657F622E056F608A3E056F6BE
:1009830008A3E056F608A3E056F622C0E0E8C0E06C
:10099300E58124FCF8E6A2E7D0E0F8D0E022E046C7
:1009A300F008A3E046F008A3E046F008A3E046F011
:1009B30022E056F008A3E056F008A3E056F008A39F
:1009C300E056F022E647F60809E647F60809E64747
:1009D300F60809E647F622700422600D18C6C333F1
:1009E300C608C633C6D5E0F41822C0E074F2120379
:1009F300C2C2C7121AEE7F01020479E4C396F60855
:100A0300E496F608E496F608E496F622C3E7960819
:100A130009E7960809E7960809E79622C3E09608CE
:100A2300A3E09608A3E09608A3E09622C6F4C608BE
:100A3300C6F4C608C6F4C608C6F4C62275D0007547
:100A430081407510FF75110200020421600C08C675
:100A5300C313C618C613C6D5E0F422E6F008A3E60E
:100A6300F008A3E6F008A3E6F022E0F608A3E0F618
:100A730008A3E0F608A3E0F622CAC0E0E6F0A30864
:100A8300DAFAD0E0FA22E0FAA3E0FBA3E0FCA3E069
:100A9300FD22EAF0A3EBF0A3ECF0A3EDF022E5C70F
:100AA30054F84401F5C77901222510F582E4351184
:100AB300F5832212054023DF021205400BE00212E8
:100AC3000540D9E00212054018E30212054055E43F
:100AD30002120540F0E402120540EBE50212054064
:100AE30009E602120540918701120540C4870112ED
:100AF3000540E38701120540058801120540178868
:100B030001120540458801120540A78801120540DE
:100B13002C8901120540CA8901120540168A011267
:100B23000540558A01120540728A01120540A18AC7
:100B330001120540F78A01120540128B011205408C
:100B4300398B01120540748B01120540B48B0112DD
:100B53000540D58B01120540258C01120540DF8C21
:100B630001120540648D01120540EE8D011205400E
:100B7300CF8E01120540FC8E011205404B8F0112EE
:100B83000540738F011205409C900112054014919A
:100B9300011205403A91011205406091011205408E
:100BA300849101120540969101120540A091011212
:100BB30005404A9201120540B692011205407D9309
:100BC300011205408593011205401094011205405E
:100BD30044940112054054940112054019950112E1
:100BE3000540C7950112054026960112054033972B
:100BF30001120540AC97011205400098011205400F
:100C0300759801120540139A01120540279A0112A3
:100C13000540899A011205400E9B011205405B9B1A
:100C230001120540799C011205406B9D011205409C
:100C3300D89D01120540549E01120540CA9E01121F
:100C43000540029F01120540DF9F0112054002A1EA
:100C5300011205405FA101120540A8A10112054040
:100C6300D0A10112054059A201120540EFA20112C1
:100C7300054055A3011205407AA301120540F3A3D1
:100C83000112054087A4011205401AA5011205406F
:100C93003EA50112054062A60112054075A6011288
:100CA3000540E6A601120540FBA6011205405CA71C
:100CB30001120540A6A701120540E1A70112054054
:100CC30002A901120540C9AA01120540D3AA0112C3
:100CD3000540DDAA01120540E7AA01120540F1AA69
:100CE300011205400BAB0112054015AB0112054083
:100CF3001FAB0112054029AB011205404AAB01129B
:100D0300054098AB01120540A2AB01120540C6ABEA
:100D130001120540EAAB0112054043AC0112054044
:100D230088AC01120540A6AC011205401DAD0112AD
:100D3300054067AD011205409DAD011205401CAE93
:100D430001120540A5AE0112054082B00112054013
:100D53004AB10112054070B10112054058B20112A7
:100D6300054030B501120540BDB60112054085B8F6
:100D730001120540CBB801120540F5B90112054037
:100D830046BA01120540B1BA01120540BBBA0112BD
:100D9300054081BC0112054035BD0112054087BDE8
:100DA3000112054043BE0112054008BF0112054070
:100DB30093C001120540B6C0011205400AC10112D9
:100DC3000540F8C1011205402AC2011205407EC246
:100DD3000112054083C301120540CAC30112054035
:100DE30010C4011205406FC401120540BCC50112B5
:100DF300054008C60112054012C701120540B9C9D2
:100E030001120540DDC901120540A8CB01120540BE
:100E1300FFCB01120540FBCC0112054084CD01122A
:100E23000540DECD011205403ECE01120540CDCE78
:100E33000112054043CF01120540AECF0112054018
:100E4300B02200120540022300120540F2240012D2
:100E53000540A12500120540D52500120540FF26B7
:100E630000120540B62900120540C42A00120540AD
:100E73009D330012054057360012054043370012D8
:100E830005400938001205405B3900120540603AFD
:100E930000120540733D00120540853F00120540D6
:100EA300E53F00120540BD4000120540E840001236
:100EB3000540864100120540644200120540454347
:100EC300001205401544001205404244001205403B
:100ED300644400120540A646001205406047001214
:100EE3000540B747001205401A4800120540D04894
:100EF30000120540054900120540594900120540FA
:100F0300894900120540C74900120540154A0012DD
:100F130005401A4A00120540714A00120540994AD9
:100F230000120540944B001205401C4C0012054072
:100F33009D4E001205405A4F00120540EF5000121B
:100F430005406453001205400C54001205408454BC
:100F530000120540AD5600120540525700120540DD
:100F6300995700120540655900120540795900123E
:100F73000540865900120540B05900120540BC597E
:100F830000120540DA5900120540BC5B001205400F
:100F93001B5C001205406F5C001205407A5D001275
:100FA3000540D65D001205408D5E00120540D55EFA
:100FB300001205406F5F00120540536000120540A8
:100FC3000961001205403A620012054020630012D5
:100FD3000540C863001205405C6400120540736459
:100FE30000120540AC6400120540B66400120540CF
:100FF300C26400120540E06400120540246500123B
:101003000540926500120540B96500120540D3659D
:101013000012054028670012054072670012054060
:101023007B6800120540A068001205400A6900129F
:1010330005406C6900120540DD6900120540EF6A46
:10104300001205409A6B00120540826C00120540A5
:10105300E06C001205406A6D001205405B6E0012E1
:1010630005408A6E00120540F16E00120540CB6FF9
:1010730000120540F16F001205405A70001205403E
:101083007F7000120540A57000120540DB7000124E
:101093000540F77200120540E77300120540AD7476
:1010A3000012054047760012054090760012054075
:1010B300BC7600120540437700120540AB7700125F
:1010C3000540FD77001205402378001205406A7839
:1010D30000120540967800120540CB7800120540B7
:1010E3001B79001205407979001205402C7A001211
:1010F3000540EE7B00120540607C00120540897CB0
:1011030000120540FD7C00120540727D001205406F
:10111300B47D00120540F07D00120540157E0012DB
:1011230005405B7E00120540787E00120540157F66
:101133000012054076E703120540C1E7031205409C
:10114300918002120540BF80021205407D81021288
:1011530005406382021205406A8302120540F5844A
:10116300021205406A8502120540198602120540E3
:10117300168702120540818702120540D4870212A6
:1011830005402888021205403288021205407888FB
:1011930002120540DB8802120540738902120540E2
:1011A300E88902120540D48A021205404F8B0212CD
:1011B3000540698B02120540988B02120540C58BCE
:1011C300021205405C8C021205406C8C0212054031
:1011D300BF8C02120540CB8C02120540D78C021241
:1011E3000540E08C021205402B8D02120540868DCE
:1011F30002120540D78D02120540F28D02120540FE
:10120300288E02120540498E02120540538E0212A7
:101213000540688F02120540868F02120540F88F41
:10122300021205400B90021205401990021205406C
:10123300BA90021205408E9102120540AF9202123B
:1012430005402B9302120540359302120540A893E3
:1012530002120540BF930212054001940212054099
:101263003F94021205406E9402120540A5940212A7
:101273000540C39402120540E794021205402895E5
:10128300021205401796021205405D9602120540B0
:10129300889602120540FB9602120540229702121D
:1012A3000540679702120540759702120540CE97D5
:1012B300021205400B980212054052980212054093
:1012C300839802120540A69802120540B1980212B3
:1012D3000540CF98021205408B990212054095995B
:1012E30002120540DA99021205401E9A02120540C5
:1012F300329A021205401D9B02120540309B0212D6
:101303000540459B02120540ED9B02120540399CA6
:1013130002120540EF9C02120540FA9C021205409E
:10132300489E02120540749E02120540B59E0212A9
:101333000540CF9E02120540409F02120540CC9FFC
:101343000212054003A00212054066A202120540E4
:10135300EEA2021205406EA302120540B1A50212CD
:101363000540C1A502120540C4A502120540D0A53F
:1013730002120540E4A50212054003A6021205402D
:1013830036A602120540FBA60212054062A702120E
:101393000540C6A70212054050A80212054001A944
:1013A300021205402FA902120540C5A902120540E9
:1013B300F4A90212054016AA021205403DAA021220
:1013C3000540A2AA0212054055AC0212054058ACD2
:1013D30002120540C2AC02120540B5AD021205402F
:1013E3009CAE0212054063D9021205406AB0021294
:1013F30005402DB10212054066B10212054097B1B6
:1014030002120540A0B10212054084B20212054047
:1014130014B302120540B2B30212054072B40212B1
:101423000540EBB4021205401AB50212054057B548
:1014330002120540AC8A03120540BA8A0312054022
:10144300E4DE02120540688B03120540B08B0312E1
:101453000540B78D03120540998F0312054058923A
:1014630003120540849203120540A492031205401F
:10147300079303120540459303120540719303122A
:101483000540AB930312054020DE0312054050DEF6
:1014930003120540A5DE03120540F693031205402F
:1014A300009403120540449403120540EB94031285
:1014B30005400E9503120540AE950312054076983C
:1014C30003120540849803120540D7980312054080
:1014D300FD9803120540559903120540C59903125F
:1014E3000540189A03120540819A03120540AF9AEA
:1014F300031205402D9B031205408D9B03120540EB
:10150300CC9B03120540DE9B03120540F09B0312A4
:1015130005400F9C03120540B19C03120540EB9C50
:10152300031205406AE403120540B4DA03120540CE
:1015330013DB031205403CDB0312054032DC0312CC
:1015430005403EE6021205401DE70212054059E739
:101553000212054002E90212054044E90212054065
:10156300EFEA0212054033EB02120540FBEB0212D5
:10157300054088EC0212054019ED021205406FED9B
:1015830002120540AFED0212054055EF021205406D
:10159300FAF00212054048F30212054056F3021214
:1015A3000540BEF302120540FAF60212054013E9A4
:1015B3000312054029E90312054018E80312054008
:1015C300BBCB03120540CECB031205405BCC031209
:1015D300054096CC03120540B1CC03120540D6CC8E
:1015E300031205400ACD031205403BCD031205400B
:1015F3005ACE03120540F4D80312054061D90312F1
:1016030005407DD903120540BFD903120540E8D92F
:101613000312054080DA0312054099DA03120540EC
:10162300B1DA03120540D3A5031205406FA60312D6
:101633000540A1A703120540B5A8031205400BAA54
:1016430003120540EFAA031205402CAC0312054018
:1016530044AC031205405EAD031205400080031243
:1016630005404B8003120540378103120540EA8190
:1016730003120540FF81031205404982031205400E
:10168300988203120540AB8203120540F7820312CE
:1016930005400B830312054045830312054057841D
:1016A30003120540BA8403120540C984031205409E
:1016B3000A85031205403E85031205409E850312E9
:1016C3000540BC8503120540368603120540C287D8
:1016D30003120540E48703120540198803120540ED
:1016E300448803120540548803120540608803129E
:1016F3000540638803120540AF88031205404E89F5
:1017030003120540738903120540968903120540AD
:10171300A689031205401A8A03120540358A03126B
:101723000540578A03120540928A03120540A18A95
:1017330003120540CBE703120540E3E7031205401C
:10174300009E031205404F9E03120540F19F0312B2
:1017530005409DA103120540E5A1031205401CA30A
:1017630003120540A9A403120540CBA403120540AC
:101773001DA5031205409FA50312054000D00112C9
:10178300054021D001120540A7D001120540FBD02E
:10179300011205407CD101120540D8D10112054048
:1017A30024D20112054097D2011205401BD3011226
:1017B300054091D301120540D3D301120540FDD753
:1017C30001120540C6D901120540C1DA01120540D4
:1017D30009DB0112054099DC011205400FDF0112FC
:1017E30005409EDF01120540D9E00112054017E4D0
:1017F3000112054027E40112054077E50112054077
:10180300A3E501120540C2E60112054012E80112E8
:101813000540C4E80112054056E9011205400EEAED
:101823000112054097EA0112054048EB01120540F9
:1018330028EC011205409DEC0112054058EF0112FE
:10184300054009F00112054059F00112054029F243
:1018530001120540E3F2011205404AF3011205406B
:10186300ADF40112054054F601120540BDF7011213
:1018730005405AF80112054022F9011205406DE6B0
:1018830003120540A6E603120540ABE6031205402A
:10189300D6E60312054045D303120540AFD3031226
:1018A300054068D403120540CED40312054043C655
:1018B300031205409CC6031205402BC803120540C2
:1018C300EDE60312054037E7031205406BDC031214
:1018D300054079DC0312054051E903120540119DCF
:1018E30003120540219D031205403F9D031205404D
:1018F300A09D031205403AE20312054061E2031280
:101903000540E6E2031205403FE303120540DD9D77
:101913000312054058E3031205407AE3031205401E
:10192300E4E303120540EFE30312054033E403123B
:101933000540B4B203120540C2B20312054003B31B
:10194300031205401DB3031205406EB30312054095
:101953006FB40312054094B403120540B1B40312EB
:101963000540CEB403120540F3B4031205402CB571
:10197300031205406AB503120540E1B503120540A1
:101983007DB60312054032B70312054040B7031278
:101993000540BAB70312054076B80312054001BBF0
:1019A30003120540AFDF03120540E8DF03120540D1
:1019B30005E00312054063E003120540C8E003128B
:1019C30005408DAD03120540FAAD03120540B4AED8
:1019D3000312054021AF0312054047B0031205402F
:1019E300BAB1031205401EB2031205406AB20312D4
:1019F300054073B20312054082B20312054095B24B
:101A030003120540ABB20312054072FA01120540FE
:101A1300C5FA0112054039FD011205406BFD0112A3
:101A230005408DFD01120540A6FD01120540BFFDD5
:101A330001120540F1FE0112054087FF0112054026
:101A430025D70312054057D70312054063D7031266
:101A5300054096D703120540BFD703120540EDD7C3
:101A6300031205406AD80312054099D803120540B2
:101A730071CE0312054097CE03120540D4CE031254
:101A83000540E6CE0312054002CF0312054070CF96
:101A93000312054079CF03120540D8CF0312054046
:101AA300FCCF03120540BBD003120540C8D003127C
:101AB3000540D9D0031205408EFF02120540DBFF1B
:101AC30002120540E6BE031205400EC00312054094
:101AD3001BC0031205403AC00312054050C0031255
:101AE300054064C003120540DEC0031205405CC11B
:101AF30003120540D5C1031205401DC20312054060
:101B03002DC203120540567F001205407A7F001252
:101B13000540A27F00120540CA7F0012054007D18D
:101B23000312054020D1031205402CD103120540B6
:101B330040D1031205405ED10312054068D1031260
:101B4300054072D10312054085D103120540B9D176
:101B530003120540F2D10312054023D203120540BC
:101B630071D203120540BED203120540D9D203122B
:101B73000540E3D203120540F4D2031205403AD3E1
:101B83000312054063E8031205403BF702120540C8
:101B930067F70212054083F70212054096F7021217
:101BA3000540ACF7021205401CF8021205404FF83D
:101BB30002120540A9FB02120540DFFC0212054098
:101BC30012FD0212054077FD0212054066FE021265
:101BD30005408EFE02120540A3FE02120540B3FE2D
:101BE30002120540F7FE021205404CFF02120540A7
:101BF30062FF0212054007E10312054022E10312CE
:101C030005404BE10312054065E1031205408AE1FB
:101C130003120540A9E103120540C1E10312054087
:101C2300EFE10312054009E203120540ABE803129A
:101C3300054066BB031205406DBB0312054079BC2A
:101C430003120540A9BC03120540CFBC0312054093
:101C530002BD0312054014BD031205404EBD03121D
:101C63000540B4BD03120540EDBD0312054039BE66
:101C73000312054066BE0312054086BE03120540EB
:101C83003FD50312054057D5031205403AD6031238
:101C9300054068E503120540BFE503120540FCE576
:101CA300031205403DE6031205403CC20312054002
:101CB3005BC203120540A6C203120540C2C203124F
:101CC3000540FAC20312054007C30312054024C3AB
:101CD3000312054007C4031205403EC40312054026
:101CE300F5C40312054000C50312054012C50312D3
:101CF30005401BC50312054025C503120540CCC88A
:101D030003120540ADCB03120540AA9D0312054003
:101D1300C6FF01120540EBE80312054033E9031245
:101D23000540FBD6021205409BD502120540F4D4B0
:101D3300021205401FD30212054066D1021205406C
:101D4300EDD00212054091D00212054034D00212A8
:101D530005400AD002120540FECD02120540CACD4D
:101D63000212054083CD0212054058CD02120540F0
:101D7300AECC0212054061CC02120540CFCA02125A
:101D83000540CCCA02120540DEC902120540AAC9A9
:101D930002120540E5C80212054018C702120540A9
:101DA300CBC602120540B3DE0212054095DE0212D5
:101DB300054027DE02120540E1DD021205404CDD3D
:101DC300021205409CC60212054099C60212054044
:101DD3008CC6021205409BDC0212054052C6021259
:101DE300054044C602120540FAC40212054076C4F7
:101DF30002120540308B031205408EDC02120540AF
:101E03003CC402120540E0C302120540B3C30212F0
:101E13000540C0C0021205407EC00212054072C0D8
:101E230002120540D2BF0212054009BF021205404B
:101E330059BC0212054085B90212054046B9021287
:101E43000540E5B70212054091B702120540D5B629
:101E530002120540A8B602120540FFB50212054062
:101E630098B502120540D2B50212054027AF020011
:101E7300000080FBE473000136360101000102011A
:101E83000001030100010401060605020000070129
:101E930000340801000F090401010D0100FF0E08C1
:101EA300000017020000190100FF1A0100011B01C5
:101EB30000051C0100081D0200001F010001200194
:101EC3000001210200002301000F2402000026016B
:101ED300000127010308280200FF2A0100072B0144
:101EE30002402C0100002D0100012E0100012F01F1
:101EF30000FF30010B1C310800003A010008030009
:101F030071003001600011007000310220035004A1
:101F13008000100061000000140063007300720071
:101F230062004300000013000600000000000400EC
:101F3300120000000000000000000400040037004D
:101F430037003C0244000000000000000000650070
:101F53000000350081000000050000008300000040
:101F630001037103010301030103010301032203BD
:101F73000203010310030003000300030003000333
:101F830000030003420300032403060300030003CA
:101F93000403120325032303250323030403040378
:101FA30000030003000344030003000323030003AF
:101FB30065032100350381030003050300030003C8
:101FC3000003030471040204600411047004020496
:101FD30002040104020410046104000414046304F1
:101FE300730472046204430400041304060400042B
:101FF3000004040412040004000400040004510457
:102003006400000400040004440400040004000409
:10201300000465040004350481046400050400041D
:102023008304000401017101010101011101010196
:102033003101010101018001100161013B00140024
:10204300630173017201620143010001130106017F
:102053003D013500040112010001000100010001EE
:1020630004010401330133013C0144013201360010
:102073000001000165010001350081010001050136
:102083008201830100010302710230016002110227
:1020930070020102020202028002100261023A008F
:1020A30041006302730272026202430200021302DE
:1020B30038000002000204021202000200020002C1
:1020C300000204020402370037003C02440200020B
:1020D300390000020002650200023502810200029B
:1020E300050282028302000236000100060000009E
:1020F3000F0000000000000000000000000003FFCC
:10210300FF00000403FFFF0000FFFF0FF4010005C1
:10211300C4040320000100000B00000000000000C5
:10212300000301000036181300D01701003618020F
:10213300009A170300A0170400A6170500AC1706A2
:1021430000B817FFFF000001700E06A00E089A0EDC
:102153000BAC0E10040E02760E058E0E077C0E0CD1
:102163005E0E0D6A0EFF000003000300040008006A
:1021730010001F003E007B00F600EC01D703AF0701
:102183005D0FB91E713D00007E12AE1284128A12D9
:10219300A8129C129612B412BA12C012CC12901248
:1021A30078127212D5C5C5B5A5A5958585757565D2
:1021B30065555545453535252515059C36063A7033
:1021C3003DD9404344AD47174B814EEA5100160FAA
:1021D30000000B150B020002220F32000006567797
:1021E3007777777777777777777777777777000169
:1021F30002030405060708090A0B0C0D0E0F6213F0
:1022030074137A134812801342124E1282117C11F6
:10221300B811BE11B2116A11D413F213F813DA1301
:102223006C1EE0130C0E020B040B0A0708000F00D0
:10223300383C3E363B3B352B432C00011916181610
:10224300161523030000034948424D1817250502BC
:10225300303017181921301B1D1F30303016181954
:1022630020231A1C1E30A212C612EC13D212D8124B
:10227300C81386138C13981392138E11941188111B
:10228300C4110005150D091008040000000000002A
:102293009A11AC1100BE040A150004000E000309D4
:1022A300280F010809000C040810050C08C082C09F
:1022B30083E99003CDF0E4900382F0121C80900335
:1022C300E0E4F0A3F09003CEF0A3F01210AA120BF7
:1022D30070120D3E121C86900344E4F0A3F09003A9
:1022E300F2E07002A3E060099003F2125C6B121E2D
:1022F300779022A4E493FA7902121CE002579274B5
:10230300F2120356EAFEEBFF74805FF9E47001E911
:10231300706DEE54207003022454750A007C027D14
:10232300007A201224E77C0079047A007B00120EE5
:10233300F48A088B09807F0CEC75F003A4A9F024C0
:102343004AF582E93421F583E49364FF602AE49338
:10235300FA8508828B83E06A70DDAA08EC75F003C6
:10236300A4244BF582E93421F583E493C0E074019E
:1023730093F583D082121E77AA08AB091214CA9070
:1023830003CDE0F91214D68A088B09EA7001EB60D9
:10239300047C0080A3EEFA74806FFB0224D07401E6
:1023A300850882850983A3A3A3A3A3A3A3A3A3F05F
:1023B300850C08850D09E5087002E509606E7C004F
:1023C3007904AA08AB09120EF48A0C8B0D750A0165
:1023D300E508240412760C24FFF0A3E034FF124630
:1023E300A17002A3E070C9850882850983A3A3A312
:1023F300A3A3A3A3A3A3A3E0640170A2850882857A
:102403000983A3A3A3A3A3A3E05404709174068533
:102413000882850983A3A3A3A3A3A3A3A3A3F07AF9
:10242300B78508828509831225968084120EC47CA1
:102433000079017A007B00120EF4EA7001EB700957
:10244300E50A70057A201224DC74206EFAEF022369
:102453009DEE54106007120D74741080EEEE54401C
:102463006007120DEC744080E2EE54806007120C9A
:1024730096748080D674015FF9E47001E9601A9064
:1024830003F4E07002A3E060099003F4125C6B12A2
:102493001E77EEFA740102239C74025FF9E4700163
:1024A300E9600A121074EEFA740202239C74045F4A
:1024B300F9E47001E960121260DC12591879011213
:1024C3003739EEFA740402239C7A007B008005748A
:1024D300031208497F060205AD7B009003CDE0F9A6
:1024E3001215DE227B009003CDE0F91215D8227479
:1024F300F4120356EAFEEBFF7508018E828F83A365
:10250300A3A3A3A3A3E0544060051229AA802E909D
:10251300036DE0A2E150238E828F83A3A3A3A3A321
:10252300A3A3E05410F9E47001E960047940800248
:1025330079001229AA120D4A8003120F7274FE6ADF
:10254300700374FF6B602C125C67125BB6120FF69C
:10255300E98E828F8360061250B9E480051250B968
:10256300740112433EFAA3E0FB121CDAE9F5097089
:102573000580127509CDAA098E828F83122596E9EB
:102583006003750800A908EEFAEFFB120ED0A90943
:1025930002474AE0240C126D49F9120E522274F6D6
:1025A300120356E9FEEAFF7A0F7B001214C4EA70A5
:1025B30001EB6019740C8A828B83F0EEA3A3F0EF16
:1025C3008A828B83A3F0125F6679008002791002FE
:1025D3005C1674F2120356EAFEEBFF8C088D098930
:1025E3000A740E120AACE0F50CA3E0F50D850C821B
:1025F300F583E4F0A31263B0E0F9120FD8E9602089
:102603001226EC701B8E828F83A3A3A3A3A3A3A381
:10261300A3A3126709850C82850D831259188003C1
:10262300750A00EE241D1226DE1206320109D92690
:102633004726612673267C266A269D26D926B02640
:10264300C926D226780C12081BAC08AD09EEFAEFA6
:10265300FB120D5C7402120849E9F50A8078EEFA60
:10266300EFFB120D62806FEEFAEFFB120DA4806692
:10267300EEFAEFFB12103280E0EE24171229926477
:10268300027053E50A700A126FB57003A3E0697014
:1026930045EEFAEFFB120FC6803CEE241712299287
:1026A30064027032EEFAEFFB120FAE80299003F64C
:1026B300E07002A3E0601FEEFAEFFB9003F6125CFA
:1026C3006B121E778010EEFAEFFB12103E8007EEBE
:1026D300FAEFFB12104AA90A0224D7124C1512264C
:1026E300E522E0F81263C1E0228E828F83A3A3A3C5
:1026F300A3A3A3A3A3A312631664022274F4120375
:102703005674DE1208DB8A088B098A828B83A3A3A3
:10271300E0F912474F7001EF700302280685088223
:10272300850983A3E064F16033850882850983A367
:10273300E064CD6027850882850983A3E0641A607D
:102743001B850882850983A3E064E9600F850882FD
:10275300850983A3E064E1600302289F8E828F834F
:10276300A3A3A3A3A3A3A3E05408F9E47001E9700E
:102773000302280E74058E828F83A3A3A3A3A3A3AE
:10278300A3A3A3F09003FAE07002A3E0600990030F
:10279300FA125C6B121E779003FCE07002A3E060F8
:1027A3003390036DE0A2E1502B8E828F8312762744
:1027B300A3A3A3A3A3A3A3A3124C0E88828983126A
:1027C300644B1210DAEA7001EB60099003FC125CAF
:1027D3006B121E778E828F83A3A3A3A3A3A3A3A3AA
:1027E300A3E06402701074068E828F83A3A3A3A355
:1027F300A3A3A3A3A3F0850882850983A3A3E0F978
:10280300120ED6120EC474220247477900120ED05C
:10281300E9700302289F90036DE0A2E1506B126DF3
:102823003E7002A3E060628E828F8312644B740356
:10283300120AAC126D50850882850983A3E064E90E
:10284300701B12299912081F850882850983A3E04A
:10285300F50A780A12081F1243E8120849740C1289
:102863000AAC123D4012334F1259187408120AACC5
:10287300E06004794080027900740E120AAC124CB5
:102883000E740C120AAC12333C8E828F83A3A3A363
:10289300A3A3A3E04420F0A3E00227868508828552
:1028A3000983A3E0C0E07402120AACD0E01256A57B
:1028B300126EEBEE240B122992851082851183AAE6
:1028C30082AB837005120CBA8003120FD285088283
:1028D300850983A3E064F16053850882850983A396
:1028E300E064CD6047850882850983A3E0641A60AC
:1028F3003B850882850983A3E064E1602F85088214
:10290300850983A3E064F060237402120AACE064D7
:10291300B7601912299912081F7403120AACE0F563
:102923000A780A12081F1243E812084990036DE05F
:10293300A2E140030227D78E828F83A3A3A3A3A37D
:10294300A3A3A3A3E06402702A8E828F83A3A3A30D
:10295300A3A3A3E05404601B1229AA120FF6E97083
:102963000D125C6774FFF0A3F074050227EB740388
:102973000227EB850882850983A3E064E9600302EB
:1029830027D7EEFAEFFB1210500227D7EE240FF5EC
:1029930082EF125665228E828F8312670DE8FAE961
:1029A300FB750A01780A228E828F831226E5FAA329
:1029B300E0FB2274F4120356EAFEEBFF7508007580
:1029C30009008E828F83A3A3A3A3A3E0603E7508AF
:1029D300088E828F8312644279FF121DB8EA700158
:1029E300EB601075082C8E828F83A3A3A3A3A3E0AF
:1029F300D2E0F08E828F83A3A3A3A3A3E054036446
:102A0300016003022A9A430811022A9AEE2418123B
:102A13002992603DEE241A122992701C126FB57030
:102A230003A3E0697005750822806C900382E0645B
:102A3300047064750901805FEE241B127636241A34
:102A4300122AAFEE2419122AB7120DB6E970488084
:102A5300E21226EC7003750801126FB57003A3E050
:102A6300697006E508D2E1F508E5088E828F83A335
:102A7300A36011E07006E508D2E58019E508D2E607
:102A8300F5088003E06010EE241D124E8664016099
:102A930006E508C2E0F508E508A2E1400AE5097089
:102AA30006E508D2E7F508A90802474AF582EF12BE
:102AB3005665FA22F582EF122ABE221272E9E0F974
:102AC3002274F012035674D21208DB7401120AAC9A
:102AD300126720120AAC12604B7408120AACE4F0BD
:102AE300A3F0740C120AACAC82AD837401120AAC6D
:102AF3001233827401120AAC1263BD126449120FBD
:102B03004E7401120AAC12644FF8A3E0F97419125F
:102B13000AAC125918740C120AACAA82AB83120EB7
:102B230064E9851082851183F07412120AACE060A7
:102B3300277423120AACE0FD740D120AACE0FC7496
:102B430001120AAC123387FAA3E0FB7901120ADA05
:102B5300E96003023330801490036AE0600E85104D
:102B630082851183E0A2E140030233308510828520
:102B73001183E0A2E6502D7429120AAC1226E164F7
:102B830003700D7429120AAC125F51E0640D6014D6
:102B9300740C120AACAA82AB83121026E96401708A
:102BA300030233307401120AACE0242C12469DF860
:102BB300A3E0F9900380E0687003A3E069703575C2
:102BC3000800780812081F780812081F7403120AF5
:102BD300AC123396F97403120AACE0242A12335868
:102BE3007403120AACE02412FAA3E03400FB12448B
:102BF30003120849740F120AACE0FA900370E06AFA
:102C030060030233307412120AACE07003022CEA40
:102C13007401120AACE0242A12469DFCA3E0FD7461
:102C230001120AAC123375FAA3E0FB1210DA740A2C
:102C3300120AAC125BB6740A120AACE07002A3E08B
:102C43007003023330740D120AACE0F87401120AF7
:102C5300AC123347F8A3E03400F9740D28F582E48D
:102C630039F583E0FA740A120AAC123343E06A605E
:102C73001E740A120AACA31237EDEAF090877F782C
:102C830008120A6D740A120AAC12337C120A5E79B6
:102C930004740D120AACE0FA7401120AAC12338701
:102CA3002AFCA3E034008C82F583A3AA82AB8312AF
:102CB30014B28A088B098C0A8D0B740A120AAC129F
:102CC3003343A3780C120A6D780C7908120A0F505B
:102CD300030233309087737808120942740A120A88
:102CE300AC12337C120A5E90036DE0A2E150030242
:102CF3002DCA900382E064046008E0640960030263
:102D03003330851082851183E0A2E550647401128B
:102D13000AAC123396C0E07405120AACD0E0F0742A
:102D230001120AAC12469AC0E07406120AACD0E053
:102D3300F07401120AACE0243012469DC0E074071F
:102D4300120AACD0E0F07401120AACE02424125051
:102D5300BC1206997409120AACAC82AD83741012CA
:102D63000AACAA82AB83120CC07404120849023362
:102D730030A2E640030233307429120AAC126456BF
:102D8300701C7423120AACE06402600302333074D3
:102D93000C120AACAA82AB83120FC6023330742919
:102DA300120AAC12333560030233307423120AACB7
:102DB300E064046003023330740C120AACAA82ABE1
:102DC30083120FBA023330741D120AACE0602D7403
:102DD30001120AACE0240212469DFAA3E0F5838AAD
:102DE30082A3A3A3A3A3A3E0141260F4A3A3A3E069
:102DF300C0E0741D120AACD0E0F0700A8510828521
:102E03001183E0C2E7F0851082851183E0A2E350CD
:102E13007A7408120AACE4F0A3741012569CA2E26E
:102E230050187411120AACE054E3F07411120AAC96
:102E3300E0131313541FFAE08038A2E450367411E0
:102E4300120AACE0541C1313543FFA600974076A66
:102E5300600E1AEA700A851082851183E0C2E7F0DA
:102E6300EA333354FCC0E07411120AACE054E3FAC1
:102E7300D0E04AF07411120AACE0C0E07401120A07
:102E8300AC125F4BA31250DAD0E0F0900382E064FF
:102E9300046005E0640970507415120AAC126FC225
:102EA3007003A3E06960197415120AAC1226F96065
:102EB3000F7411120AACE05403640160030233304F
:102EC300740E120AACE07003022D107429120AACBE
:102ED3001264567003022D857429120AAC1233351D
:102EE3006003023330022DAE7E008510828511838C
:102EF300E054617003023033E0A2E04003022F8DFF
:102F03007401120AAC123375FCA3E0FD740C120AAF
:102F1300ACAA82AB83120DF2E97065120F7EE9FE53
:102F2300851082851183E0A2E7505F7401120AAC19
:102F3300E02412123358740C120AACAA82AB831227
:102F43000DF8E9851082851183602DE0A2E3500B13
:102F53007403120AAC74FFF0A3800F7415120AAC49
:102F6300126966120AACE8F0A3E9F07408120AAC1D
:102F7300E04404F0A3E08011E0C2E5F07E00800AA3
:102F8300851082851183E0549FF08510828511831B
:102F9300E0A2E550617401120AAC123396C0E074EA
:102FA30005120AACD0E0F07401120AAC12469AC0C2
:102FB300E07406120AACD0E0F07401120AACE0240B
:102FC3003012469DC0E07407120AACD0E0F07401E1
:102FD300120AACE024241250BC1206997409120A96
:102FE300ACAC82AD837410120AACAA82AB83120C10
:102FF300C07404120849851082851183E0A2E6405B
:103003000302324D7403120AAC8582088583097862
:103013000812081BEEF97403120AAC12338D120A5C
:10302300ACAA82AB83120E58740212084902324BC7
:10303300740E120AACE0640170387429120AAC12DF
:1030430026E16405702C7403120AAC85820885831B
:1030530009780812081B79007403120AAC12338D25
:10306300120AACAA82AB83120E58740212084902E8
:103073003330741D120AACE0701879007415120A0B
:10308300AC124C0E7417120AAC12644B120D6E0282
:103093003330120ECAE960030233307424120AACCF
:1030A300E070030231707427120AAC124C0E7426BE
:1030B300120AACE0FA7425120AACE0F9120DB6E973
:1030C30070030231627426120AACE0701174151297
:1030D3000AAC126966120AACE8F0A3E9807074279F
:1030E300120AAC12644B7426120AACE0F9120DB04A
:1030F3007403120AAC125BB67414120AACE06004D7
:10310300780880027800E82408FA7413120AACE005
:103113006004780880027800E82AFA7411120AAC75
:10312300E06004780180027800E82AFA0AEAF87479
:1031330001120AAC123347FAA3E034008A82F58302
:10314300E014F07408120AACE04440F0A3E0F0127B
:103153000F7EE9FE7427120AAC1272DB02324D7441
:1031630027120AAC12644B12153C02333074151249
:103173000AAC126966120AACE8F0A3E912569CA2E3
:10318300E350047A4080027A00EAF50878081208CE
:103193001F7425120AACAC82AD837416120AAC12EA
:1031A300644B7411120AACE0F9120E227401120876
:1031B30049E960177408120AAC1261EE7401120A2D
:1031C300AC1233871263BCE0543FF07424120AAC90
:1031D300E060277415120AAC124C0E7425120AAC67
:1031E300AA82AB83120F487403120AAC125BB67443
:1031F30008120AACE044401261F1740E120AACE00A
:103203006401601579007417120AAC124C0E741520
:10321300120AAC12644B120DBC851082851183E037
:10322300A2E350047940800279007417120AAC12A9
:103233004C0E7415120AAC12333CE9600874081280
:103243000AAC1261EE120F7EE9FE7403120AACE0BF
:1032530064FE7004A3E064FF70027E008510828523
:103263001183E0A2E74003023330EE7003023330F0
:103273007401120AAC12336CFA7B001215368A0CF5
:103283008B0DEA7001EB70030233307401120AAC48
:10329300125F4B126C461208177404120AAC1233F5
:1032A3006CFC7D0012532612084990036AE07008F3
:1032B3007412120AACE060217423120AACE0FD74AC
:1032C3000D120AACE0FCAA0CAB0D7900120ADAE984
:1032D3006007AA0CAB0D02316A740E120AACE0C08F
:1032E300E0742B120AACD0E0F0742C120AACE4F0B8
:1032F300A3F0742B120AAC8582088583097808121F
:10330300081B740A120AAC12069DEEF5087808121F
:10331300081F7406120AAC1233827408120AAC1224
:103323005BA7120F367405120849E970A5742E02C3
:1033330050B11263BDE06407221258CE120D56221B
:103343001260FF2212334FA3A3E02822E0FAA3E086
:10335300F5838A822212335C22FAA3E03400FB8ACB
:10336300828B83E0FCA3E0FD22123370221250E42F
:10337300E022E02412126D49221250E07808221252
:103383003370F922125F4FA3E022E0241212335C60
:10339300740E22E0242E126D492274F01203567427
:1033A300EA1208DB8A0E8B0F124097750901850E0E
:1033B30082850F83A3E0F50CE50E2402FCE50F12D2
:1033C30040AC7408120AAC12604B740A120AAC7453
:1033D30002F07413120AACE4F0901A2FE07010EEAE
:1033E3007001EF700AE50C70067509C302358A9007
:1033F3000382E0640860067509C2023586850E8281
:10340300850F83A3A3A3A3A3A3A3A3A3A3E0A2E1E1
:10341300500EA2E350057508048011750803800C53
:10342300A2E350057508028003750801EE7001EFF1
:10343300607E8E828F83A3A3A3A3E06404600D8EBA
:10344300828F83A3A3A3A3E06403700C74046508B1
:10345300602C7403650860268E828F83A3A3A3A3C5
:10346300E06402600D8E828F83A3A3A3A3E06401B3
:10347300702474026508600674016508700B127489
:1034830097120AAC12591880278E828F83A3A3A3A5
:10349300A3E06402600D8E828F83A3A3A3A3E064E1
:1034A300017006126584121E771236497E007F0072
:1034B3007408120AACE064FE7004A3E064FF703C7D
:1034C300E50C60179003BFE06402700F901A361288
:1034D300749B120AACE8F0A3E98020850E82850F65
:1034E30083A3A3A3A3A3A3A3A3A3A3E05402F912B7
:1034F3000D7A7408120AACEAF0A3EBF07408120A0E
:10350300ACE064FE7004A3E064FF70057509C78036
:1035130072E50CF50A780A12081F850E82850F835F
:10352300A3A3A3A3A3A3A3A3A3A3E0F912363E7467
:1035330009120AAC12644B120CDE7401120849E939
:103543007041A90812363E7408120AAC1237328A47
:103553000A8B0BAE0AAF0BEE7001EF601E740265AF
:103563000C700D8E828F83A3A3A3A3A3E0D2E3F0F9
:10357300740A120AACE4F0F50980087408120AAC64
:1035830012604BE50C700F851082851183AA82AB04
:1035930083121CC28010FCA908851082851183AA9E
:1035A30082AB83120FB4E9FAEE7001EF6053E50CBE
:1035B30060208E828F83A3A3A3A3A3E0D2E6F0743B
:1035C30002650C700D8E828F83A3A3A3A3A3E0D205
:1035D300E5F0850E82850F83A3A3A3A3A3A3A3A3CF
:1035E300A3A3E0A2E6500D8E828F83A3A3A3A3A37C
:1035F300E0D2E7F08E828F83A3A3A3A3A3A3E00467
:10360300F0E5097003EA602EFC7D007A017B10125D
:103613001C8CEE7001EF60031236497408120AAC79
:10362300E064FE7004A3E064FF600B7408120AAC4C
:10363300126588121E7774160250B1E50E2402FC3F
:10364300E50F3400FD22E50E2402FAE50F3400FBFA
:10365300120BB22274F712035674F71208DBEAFE58
:10366300EBFF900382E06403600DE064016008E017
:103673006409600302372D8E828F83A3E060030207
:1036830037097C007D007A027B00121C8CEE240239
:10369300FAEF1260291267099003731259187953CC
:1036A300121CBC7900123739900382E06409600967
:1036B30090038012644B1210D47401125D71740470
:1036C300900382F07401120AACAA82AB83794A1286
:1036D3001CB67401120AACAC82AD837A787B0312F8
:1036E3001CA479007401120AACAC82AD83900376FA
:1036F30012373290036DE0A2E35004D2F08002C28D
:10370300F0125D5780218E828F83A3AE82AF83FC3C
:103713007D007A037B10121C8C8E828F83E0F9125A
:103723003739E4900382F0120EA6740902689812E6
:1037330058CE120B82229003801258CE120CD8223C
:10374300C082C083900344E07002A3E07041900301
:1037530082E01207220003016537057437068337B9
:10376300923790034CE07002A3E0607B90034C809F
:1037730070900348E07002A3E0606C90034880619E
:1037830090034AE07002A3E0605D90034A80529088
:103793000344E07002A3E06005123D4E70237900FC
:1037A3009003CE800909EA126AE0EB127608124907
:1037B300547001EB70EF9003CE12644B120CC68071
:1037C300269003451237EDA3A3A3E064027005120C
:1037D300106880139003F8E07002A3E0600990037F
:1037E300F8125C6B121E77025792126102227A0F53
:1037F3007B001214C48A0A8B0BAE0AAF0BEE2212A3
:10380300670D9003802274F412035674EB1208DBE5
:103813008A828B83A3A3A3A37808120A6D78081264
:103823000A2F90038378081209B47D7F7E7F7C0082
:10383300750801750900750A00750B00EC7808120C
:1038430007F4900383780812097B90877F78081226
:1038530008F1602A7F009003CE801288828983A3B7
:10386300A3E06C70010F126ADFE91276081249C2F5
:103873007001E970E6EFC39D5004EFFDECFE0CEC24
:10388300C3941B40AB8A828B83A3A3A3A3C082C030
:103893008390877F7808120A6DD083D082780812CC
:1038A30008F1605BEA124C02FAE9FB8A828B8378A7
:1038B30008120A6D9003837808120A5E8A828B834A
:1038C3007808120A6D8510828511837808120A5EC2
:1038D3007404120AAC7401F0900389E0C0E074052B
:1038E300120AACD0E0F07407120AAC123A588065A1
:1038F30090038012644B120D02900380125BB6900A
:1039030003CE1249C27001E960268882898312645A
:103913004B900380E06A7003A3E06B700A8882898E
:1039230083A3A3E06E60C9126ADFE912760880D22E
:10393300EE900375F0120E94E9601AE4900382F09E
:1039430090034EE07002A3E0600B79C490034E1223
:103953005C6B121E7702474574F412035674EB1224
:1039630008DB8A828B83A3A3A3A3A3A3A3A3A3128A
:1039730049C2FAE9FB7C00750801750900750A0064
:10398300750B00EC78081207F4900383780812098A
:103993007B90877F78081208F16037901A35E0C072
:1039A300E08C08EA2508F582EB122995FDD0E0C3E7
:1039B3009D501F750801750900750A00750B00EC11
:1039C30078081207F47808120A2F900383780812F4
:1039D30009B40CECC3941B409E90877F7808120AAD
:1039E3006D75830375828378081208F16041900333
:1039F300837808120A6D8510828511837808120A6C
:103A03005E7404120AAC7401F07407120AAC7401F8
:103A1300F0900389E0C0E07405120AACD0E0F074C2
:103A230007120AAC123A587406900382F08023E41A
:103A3300900382F0FCFD7A047B10121C8C90034EE1
:103A4300E07002A3E0600B79C490034E125C6B122A
:103A53001E77024745E412686D121CCE2274F212DF
:103A6300035674ED1208DBEAFEEBFF8E828F83A30D
:103A7300124B78851082851183AC82AD838E828F41
:103A830083A3A3A3A3A3A3A3124690126444120E79
:103A9300B8851082851183E0706A8E828F83A3A319
:103AA300A3A3A3A3A3A3E0C3940B405885088285D3
:103AB3000983A3A3A3A3A3A3A3A3E06402704590D4
:103AC3000382E064026042E06406603D900344E0E8
:103AD3007002A3E06005123D4E605E900382E064D5
:103AE300086005E06404701C7402120AACE0F97407
:103AF30007120AACAC82AD83850882850983126400
:103B030042120EBE74130224D4900344E07002A345
:103B1300E07026750A00780A12081F780A12081F37
:103B2300123D26127608123D57FCA3E0FD8508825C
:103B33008509831244071208499003CE1250D4908A
:103B430003CEE0F50AA3E0F50B80378E828F83E086
:103B5300F8A3123D57687003A3E06970198E828F32
:103B630083A3A3E0FAE508240DF582E5091229955C
:103B73006A7003023BFA8E0A8F0BEE126AE0EF12B1
:103B830050D1EE7001EF70C37A187B001215368A9C
:103B93000C8B0DAE0CAF0DEE7001EF7003023B0703
:103BA3009003CEE07002A3E070059003CE800AE597
:103BB3000A126AE0E50B127608126EEB8E828F838F
:103BC300126042EE240C12760574FFF0E48E828FAD
:103BD30083A3A3A3A3A3124325A3A3A3A3123D6A71
:103BE300E4F0A3F0E508240B12760C123D1C1246F8
:103BF300A1C4123D1CA3F07401120AAC125F56F06B
:103C03007402120AAC1258E4A3A3F0E508240DF5DC
:103C130082E509123D38A31261F6A3A3123D4012B7
:103C230059187402120AACE0640160117407120A95
:103C3300ACAC82AD83EE240D123D2F80117C087D48
:103C43000079FFEE240DFAEF3400FB1214AC74126A
:103C5300120AACE0C0E0EE2415127605D0E0F09035
:103C63001AA8E0C0E0123D26122AB2D0E0C39A405F
:103C730003023B071275FBE509127608A3E05480A3
:103C8300F9E47001E970099011ECE07003023B075D
:103C93007404120AAC1258E4700EE0704D740612EC
:103CA3000AACE07006023B07E060147405120AAC2C
:103CB300E0C0E0EE240C122AAFD0E0C39A502B856B
:103CC3000882850983127641125916123D2612295C
:103CD30095C0E0127602D0E0F07405120AACE0C0A1
:103CE300E0EE240C127605D0E0F07406120AACE084
:103CF300600D74018E828F83A3A3A3A3A3A3F07487
:103D030004120AACE07003023B0774018E828F83B6
:103D1300A3A3A3A3A3F0023B07540F8E828F83A315
:103D2300A3A322E5082410F582E50922FAEF340063
:103D3300FB121CA422124C18124251A322123D441E
:103D430022E0F8A3E0F98E828F832290034412438A
:103D5300E1640122E0F9850882850983A3A3A3A373
:103D6300A3A3A3A3A3E022A3F0EE2416124C1522CF
:103D730074F412035674C91208DB900382E06408DA
:103D83007003023E319003BFE06402703490229BC3
:103D9300E493900364F090229BE493900362F09089
:103DA30087737808120A6D90038B7808120A5E9065
:103DB30087737808120A6D90038F7808120A5E8061
:103DC3006D900393E0F824A3F582E43415F583E0C2
:103DD300F508900364F0E824A4F582E43415F58330
:103DE300E0F509900362F0750AFF750BFFE50878AB
:103DF3000A1209DAE50AF4F8E50BF4F93395E0FA67
:103E030090038BE8FCE9FDEAFE123F62750AFF7539
:103E13000BFFE509C39508780A1209DAE50AF4FCF1
:103E2300E50BF4FD3395E0FE90038F123F62E4123D
:103E33005D657904121CBC900393E07009741E1233
:103E43000AAC74018006741E120AACE4F0740F8588
:103E53001082851183F0901A341268697946121C16
:103E6300BC7401120AACE4F0901A91E0C0E0740251
:103E7300120AACD0E0F0900370E0C0E07403120AC1
:103E8300ACD0E0F07404120AACE4F07405120AAC8E
:103E9300E4F07407120AACE4F0900393E0C3940FC8
:103EA300500CE0C0E07406120AACD0E08007740640
:103EB300120AAC740FF07C947D037408120AACAA46
:103EC30082AB83121CA47C037D0079FF7410120A59
:103ED300ACAA82AB831214AC9003CCE0C0E07413A1
:103EE300120AACD0E0125E87120AAC125E76120F91
:103EF300A2900387E0C0E0741C120AACD0E0F090FB
:103F03000388E0C0E0741D120AACD0E0F0900375A2
:103F1300E0C0E0741A120AACD0E0F090038012679C
:103F2300097418120AAC1259187420120AACE4F07E
:103F330090038AE0C0E0741F120AACD0E0F074343E
:103F4300120AACE4F07429120AACE4123F6D741443
:103F5300120AACAA82AB83121CD47437024747EC13
:103F6300F0A3EDF0A3EEF0A3F022F07A737B0379D4
:103F730053123F7822121CBC7A767B03794B121CB6
:103F8300BC22C082C0838A828B83A3E06007E49053
:103F93000382F0804A7408900382F0900393E070E8
:103FA3001F90034EE07002A3E0600B790090034E74
:103FB300125C6B121E77900380124C0E7A05801AE6
:103FC3007900120CD2900373124C0E7A067B001206
:103FD3001C8C900376124C0E7A047B00121C8C020C
:103FE300579274F412035674EA1208DB8A088B0999
:103FF300124097EE7001EF70030240928E828F831E
:10400300A3A3A3A3E0640160278E828F83A3A3A34A
:10401300A3E06402601A8E828F83A3A3A3A3E06448
:1040230003600D8E828F83A3A3A3A3E06404705F58
:10403300E5082402FCE5091240AC127497120AAC9D
:10404300125918740A120AAC7401F07413120AACF0
:10405300126868121CC88908AC087D007A077B00C7
:10406300121C8C8E828F83A3A3A3A3A3E0C2E0F0D0
:1040730074018E828F83A3A3A3A3A3A3A3A3A3F0FB
:1040830074028E828F83A3A3A3A3A3A3A3A3F07419
:1040930016024747EA24020A0AEB3400FB120BA676
:1040A3008A0A8B0BAE0AAF0B223400FD8510828582
:1040B3001183AA82AB83121CA42274F712035690B5
:1040C30003CEE0FAA3E0800CEA24161250CE1215B8
:1040D3003CEEFAEFFBEA7001EB70ED9003CEE4F0F7
:1040E300A3F002689B74F41203568A088B09EA242E
:1040F30013F582EB1229956403700DEA240BFAEB96
:104103003400FB120BA6800BE0640270731269602B
:104113001276208A0A8B0BAE0AAF0BEE7001EF60AA
:104123005F850882850983A3E0700DE48E828F8307
:10413300A3A3A3A3A3A3804764F1600C850882858E
:104143000983A3E064E1701F8E828F83A3A3A3A3DB
:10415300A3A3E064017010126584121E77E508249E
:104163000BFAE5091236508E828F83A3A3A3A3A370
:10417300A3E0600C8E828F83A3A3A3A3A3A314F055
:1041830002474A74F21203568A0C8B0DECFEEDFFC4
:10419300890B8A828B83126AE58A828B8312424B54
:1041A300EEF8EFF9A30EAF838A828B83A3A3E0C457
:1041B30054F0FA88828983E04A12425A1242511219
:1041C3004255E0333354FCFA8E828F83E04A124225
:1041D30055A3E033333354F8FA8E828F83E04AF0E9
:1041E30008EFF9A30EAF83850C828B83A3A3A3A34C
:1041F300A3A3E0A2E0E492E013135480FA88828937
:1042030083E04AF0E50C2407F508EB125622120866
:10421300177C08125320120849126C5DE50C240F19
:10422300F508E50D3400F50978081208177C031228
:104233005320120849E50BC3940F400912431C1283
:104243003D38A3A3F00224D7A3124251F022E00287
:104253003D4912425AA322F0850C828B83A3A3A368
:104263002274F2120356EAFEEBFF890B8C0C8D0DC0
:104273008E828F83E08C828D83124325AE82AF833F
:10428300E012574212433DC4125742124330E054E6
:10429300038C828D8312433BA2E2E492E08C828DF5
:1042A3008312433A131313541F125742124339A272
:1042B300E7E492E08C828D83A3A3A3A31243308E01
:1042C300088F09750A0078081208177C087D00E535
:1042D3000C2407126C3D120849126C5D8E088F097D
:1042E30078081208177C037D00E50C240F126C3D3F
:1042F300120849E50BC3940F40148E828F83A3A346
:10430300A3E0C0E012431C127608D0E080071243FA
:104313001C127608E4F00224D7E50C2412F582E59A
:104323000D2212432922F08E828F83A322A3A3128C
:1043330043290EAF8322A3A3A3A3A3F08E828F836B
:10434300E02274F412035674F91208DBEAFEEBFF61
:10435300900344E07002A3E060101243DA64027039
:1043630009EEFAEFFB1210628068900380E06E7032
:1043730003A3E06F705C74016960097A947B031294
:104383006863704E7A007B029003CDE0F91215E466
:10439300EA7001EB703C9003837808120A6D851074
:1043A300828511837808120A5E900389E0C0E07465
:1043B30004120AACD0E0F07405120AAC7401F07474
:1043C30006120AAC7402126869120C84E960921234
:1043D3000C8A74070247479003441243E1221250A8
:1043E300E4A3A3E022E508240CF582E509122ABE22
:1043F3008A828B83A3A3A3A3A3A3A3A3A31233663A
:104403008A828B831258CE120F84740222E0F9023F
:10441300579274F61203569003DFE0701F7C007905
:10442300017A007B00120EF4EA7001EB600E8A82BF
:104433008B83E07002A3E06003120E4C025C16C093
:1044430082C0831248B2401079FF120EEEE9FA904F
:1044530022A9E493C39A5004790180027900025798
:104463009274F11203568A0A8B0B890E7509008A1E
:10447300828B83A3A3A3A3A3A3A3A3E0F9120EFA9E
:104483008A0C8B0DAE0CAF0D750801EE7001EF6059
:104493000302453A850A82850B83A3A3A3A3A3A39F
:1044A300124C0E850A82850B83A3A3A3A3A3A3A304
:1044B300A3E0F9850A82850B8312644B120EE28A0C
:1044C3000C8B0DAE0CAF0DEE7001EF70030246774F
:1044D3008E828F83A3A3A3A3E4F0A3F0E50A240BA6
:1044E300FAE50B126029E0C0E0127602D0E0F01288
:1044F3001002EE240C125BAF750901EE2406F8EFEF
:1045030012760F547FF0A3E054FC1246A1540460CA
:10451300030245BE901A8AE0F50A750B007407780A
:104523000A1209DA8E828F83A3A3A3A3A3A3E04570
:104533000AF0A3E0450BF08E828F83A3A3A3A3A36A
:10454300A3E05480F50AA3E05403F50B7407780A3B
:10455300120A4FE50E607774028E828F83A3A3A3A2
:10456300A3124339240D12469DA2E2500990036E13
:1045730012468E125916E50A7003024645EE2406CA
:10458300F8EF3400F9E8FAE9FB8A828B83E0547F81
:10459300FCA3E054FCFD74FF250AF50A74FF340004
:1045A300F50B7407780A1209DAE50A4CF8E50B4DA6
:1045B300F98A828B831259180246458E828F83A310
:1045C300A3A3A3A3A3E04480F0A3E0024539E50A33
:1045D3007005750800806B8E828F83A3A3A3A3A3AA
:1045E300A3E0542060171214BE8A0A747F550AF898
:1045F300745F288E828F83A3A3A3A380278E828FC9
:1046030083A3A3A3A3A3A3E05410600E1214BE8A32
:104613000A740F550AF8740180D88E828F83A3A37E
:10462300A3A37401F0A3E4F074048E828F83A3A385
:10463300A3A3A3A3A3A3A31248C17001EB70031206
:10464300468174016509702F8E828F83A3A3A3A370
:104653001268FCF9EEFAEFFB120EE8E96019EE249A
:104663000C1229927002A3E060031272D8EEFAEFE3
:10467300FB12153C750800A9087F070205AD7A20D7
:104683007B009003CDE0F91214FA22E0F8A3E0F9DD
:104693008E828F83A3A322E0242F126D49221260FE
:1046A300FBE02274F412035675080012474F7001A1
:1046B300EF70030247428E828F83A3A3A3A3A3A316
:1046C300A3A3A3E064067077120F188E828F83A3CF
:1046D300A3A3A3A3A3A3E05408F9E47001E9605CD6
:1046E3008E828F83124B6E7A007B00120EDCEA708F
:1046F30001EB7048124755121CEC7C007D007A00D8
:104703007B0080228E828F83124B687004A3E06447
:10471300FF6029124755121A10E9641A601E7C00C3
:104723007D00EEFAEFFB120EDC8A088B09AE08AFB0
:1047330009EE7001EF70CD7900121CF275080102C9
:104743002AAA74151208497F040205AD120EFA0253
:1047530037F8126C668E828F831258CE2274F7124A
:1047630003568A828B83E5827002E5837009900386
:10477300E080068A828B83A3A31249547001EB6005
:104783002C8A828B83A3A3A3A3A3A3A3E05408F936
:10479300E47001E960DDEC7001ED60158A828B83C2
:1047A3001226E16C7003A3E06D70C880047A007B6D
:1047B3000002689B74F21203568A088B09890AEC7B
:1047C300FEEDFF7A0E7B00121536EA7001EB603EB8
:1047D300E48A828B83A3A3A3A3A3A3A3A312481452
:1047E300E50A12566DA3A3126EE78A828B83A3A3F5
:1047F300A3A3E4F012481412566B127C58EA240C5B
:10480300F582EB124E8012566CA3A3F0A3F00224A0
:10481300D71273E002573674F5120356EAFEEBFF24
:10482300890A8C088D09EE7001EF605A7401650ADC
:1048330070147901120EEEE9FA9022AFE493C39A51
:10484300500F791180647404650A70341248B240C1
:10485300F18E828F83A3A3A3A3A3A3A3A3A3E50A98
:10486300124325A3127C568E828F83A3A3E4F0A365
:10487300F09003E0E07002A3E09003E0601B800A85
:104883007402650A60CB79C180201269D77002A3D4
:10489300E088828983A3A370F1EEF0A3EF1248C1ED
:1048A3007001EB700312468179007F030205AD7935
:1048B30004120EEEE9FA9022ADE493C39A22F07A41
:1048C300207B009003CDE0F91215E4EA22C082C0F8
:1048D30083E9FC79009003E0801D8A828B83A3A384
:1048E300A3A3A3A3A3A3A3E06C600574FF6C70014F
:1048F300098A828B83A3A31249547001EB70DB02F4
:10490300579274F71203568A828B83E5827002E50D
:104913008370099003E080068A828B83A3A31249E4
:10492300547001EB60248A828B83A3A3A3A3A3A364
:10493300A3A3A3E06970E1EC60148A828B83E02473
:104943000D126B91A2E240D080047A007B000268D2
:104953009B1258CEEA22C082C0839003E080068A6D
:10496300828B83A3A31249547001EB60128A828B5A
:1049730083A3A3A3A3A3A3A3A3E06970E280047A00
:10498300007B00025792C082C0839003E0800688B8
:10499300828983A3A31249C27001E9601B888289BB
:1049A30083E0FCA3E0F5838C82E06A7003A3E06BF1
:1049B30070DDE8FAE9FB80047A007B00025792126B
:1049C300670DE82274F11203568A0A8B0B8C0C8D47
:1049D3000D750800750900EA7001EB602E9003E085
:1049E30080068E828F83A3A31250D4EE7001EF60F2
:1049F3001AAC0CAD0DEEFAEFFB850A82850B831220
:104A03001E77E9640170DB8E088F09AA08AB0902DF
:104A1300467C790002053374F71203569003E012C3
:104A230067097C007D00800DE8FCE9FD88828983AD
:104A3300A3A3126709E87001E96030EA687002EB2A
:104A43006970E59003E012644BE86A7002E96B88D1
:104A5300828983A3A370081267099003E080091277
:104A630067098C828D83A3A312591802689B74F77C
:104A7300120356EAFEEBFFEE7001EF6016120F12FF
:104A8300124B827002A3E060031272D8EEFAEFFBBE
:104A930012153C02689B74F71203568A828B8312A9
:104AA3004B6E9003E01267097508007E008033881F
:104AB300828983A3A3A3A3A3A3A3A3A3E0640570F1
:104AC300180E88828983E0FFA3E0F5838F82E06C70
:104AD3007003A3E06D7002050888828983A3A31283
:104AE3006709E87001E970C79022A1E493FCE50827
:104AF300C39C500B9022A2E493FCEEC39C400F8A0C
:104B0300828B83A3A3A3A37401F0A3E48012900375
:104B13006E1267098A828B83A3A3A3A3E8F0A3E998
:104B2300F074058A828B83A3A3A3A3A3A3A3127305
:104B3300DBA3A3A3E0F0A3E0440812566D124B6875
:104B43007004A3E064FF6015900380124C0E8A8208
:104B53008B8312644B121CE6E9641A700579011207
:104B63001CF202689B1226E564FF221226E502333B
:104B7300678E828F83A3A3E0F508A3E0F5092212D1
:104B83006D421272EF8E828F831272EE1272DFE029
:104B93002274F712035674E11208DBEA2413F58238
:104BA300EB122995C0E07411120AACD0E0124F4FFA
:104BB3007409120AAC124F48124C02FCE9FD8C82B4
:104BC3008D83126709740B120AAC124F482414F533
:104BD30082EB122995C0E07412120AACD0E0F0EA1D
:104BE300240EF582EB122ABA8C828D83124C0E8529
:104BF3001082851183AA82AB83120DF80268962472
:104C030004F8EB3400F9E822124C1512336622EE55
:104C1300240FF582EF1272E92274F212035674FC28
:104C23001208DBEAFEEBFF750B00750A007508FE40
:104C33007509FF120ECAE960057911024E75EE245B
:104C4300151229926049901AA3E0C43354E0C0E0DE
:104C5300E0333354FCFAD0E04AC0E0EE2415127678
:104C630005D0E012671AFAA3E0FB79FF121DB8EA38
:104C73007001EB6017750B017508FF12298F44044F
:104C83001261F1EE2415122992D2E0F0750A408EDA
:104C9300828F831263106003124E7AEE241312295B
:104CA300927003741EF0EE2411122992640170199C
:104CB3009012BAE0600D90036AE0700D8E828F83CC
:104CC300E07006EE2411124E7DEE24141229927028
:104CD3001590035FE0C0E0EE2414127605D0E0F0F7
:104CE30090035FE004F090036DE0A2E15044E50B14
:104CF30070188E828F8312631060378E828F83E0E9
:104D03006008EE240B124E86602812298F544060EF
:104D130014EE24131229926401700A12298F54FB92
:104D23001261F1800DEEFAEFFB120F24E97003021A
:104D33004C3C8E828F83E064017012EE240B1226AA
:104D4300DE6402700812298F44401261F112298F28
:104D530054406003024DE7E50B6003024DE7900307
:104D63006DE0A2E1507EE50AF50B780B12081FEE09
:104D73002406FCEF3400FD8E828F83126449EE24F7
:104D830012122AB7120E227401120849E9600612A0
:104D93004E7A1261EB8E828F83A3A3A3A3A3A3E016
:104DA300601F8E828F83A3A312763C2407FAEF340D
:104DB30000FB120F488A088B0912298F44401261A5
:104DC300F18E828F83E064016008A90A124E921269
:104DD3000DBCA90A8E828F83124E92120D56E96082
:104DE300031261EB851082851183AC82AD83EEFAE9
:104DF300EFFB120F3C8A0A8B0B74FE650870047478
:104E0300FF65097003124B74EA7001EB60608E82D8
:104E13008F83E0C0E07401120AACD0E0F074021298
:104E23000AAC126EEB7401120AAC85820C85830DF9
:104E3300780C12081BEE240F12760512069DEE2441
:104E43000E122992F50C780C12081F7405120AAC85
:104E5300E0F9AC08AD09120F367405120849E9FEF2
:104E630074106E700BAA0AAB0B12153C80027E10F5
:104E7300EEF974040224D4EE2412F582EF124C18D6
:104E8300E4F022124C151226E5F9120FD8E922A3F9
:104E9300A3A3A31269021258CE22C082C08374DE78
:104EA3001208DB8A828B83A3A3A3A3126709740E60
:104EB300120AACE8F0A3E9124F4F740C120AAC12B9
:104EC3004F48240DF582EB122995C0E0741A120A9B
:104ED300ACD0E0F01269601267067420120AAC12BB
:104EE3004F482415F582EB122995C0E07408120A85
:104EF300ACD0E0F0EA241CF582EB126706741212C0
:104F03000AAC12591874FF851082851183F074015D
:104F1300120AAC74FFF07402120AAC74FFF09087AB
:104F23007F1206997404120AACAC82AD8374071223
:104F33000AACAA82AB83120CC0740412084979002C
:104F4300742202578FE8F0A3E9F0EA22F08A828BF9
:104F530083A3A312670D2274F012035674EE120892
:104F6300DB7410120AAC125BB68C0E8D0F890D74B4
:104F730022120AACE0F50C7423120AAC1250D47559
:104F830008107A1E7B001215367402120AAC125BEB
:104F9300B67402120AACE07002A3E070030250A9D7
:104FA300750900AA0EAB0F125B9A7001E9602388A2
:104FB300828983A3A3A3A3E06401600D888289830C
:104FC300A3A3A3A3E064037009EE54407004740424
:104FD3004FFF74045FF9E47001E96003750901850B
:104FE3001082851183AA82AB8379501259A1120AC8
:104FF300AC1250DAA3125BB67402120AACE0240BB3
:105003001250BC7402F0120AAC1250DA7402F0129D
:105013000AAC125C6BE50EF0A3E50FF07402120A02
:10502300ACE0241B1250BCE50DF07402120AACE094
:10503300240C1250BCE50CF07410120AAC1259AADD
:10504300120AACE0241C1250BC125BB67408120A9C
:10505300AC126EEB740A120AACE50CF07425120A5A
:10506300AC125C6BC082C083740D120AACAC82AD0F
:1050730083D083D0827403120795A9097402120A9C
:10508300ACAA82AB83120ED0E964017011E509600A
:1050930008A90C120EFA120F1E750800800874027C
:1050A300120AAC1272DBA90874128002740212088D
:1050B300497F080205ADE0240DF8A3E01250C32296
:1050C3003400F98882898322EA240BF582EB124C9F
:1050D30018E0FEA3E0FF221250E00257371250E41B
:1050E30022E0F8A3E0F583888202573774F01203B5
:1050F30056EAFEEBFF8C088D0974088E828F8312AB
:105103003D6AE0600874108E828F83A3F0EE24174B
:1051130012299260098E828F83A3E02408F0EE2483
:105123001512299260088E828F83A3E004F08E8289
:105133008F83A3A3A3A3A3A3E060198E828F83A36A
:10514300A3A3A3A3A3A3E0C3332402FA8E828F8372
:10515300A3E02AF0EE24111229926005750B0E804C
:1051630003750B008E828F83A3E0C0E0EE240D1243
:105173007605D0E0FAE02A250B8C828D83F0EE24AD
:105183001112299260051259452AF0850882850972
:1051930083E0C394754003025313E0FA7B001215B6
:1051A300368A0E8B0FEA7001EB7003025319EEFA85
:1051B300EFFB120F42EA850E82850F83125BB7EE77
:1051C3002402F812532C12534BF0EE240408081255
:1051D300532CA3A312534BA3A3F0EE241312533760
:1051E300F0EE2414125337A3F0750C08EE241612B4
:1051F30029926013EE2418124C0BE50E2408FAE5ED
:105203000F123D31750C10EE24171229926019EE1E
:10521300241A124C0B850C08E50E2508FAE50F122B
:105223003D317408250CF50C8E828F83A3A3A3A3B1
:10523300A3A3E060718E828F83A3A3A3A3A3A3A3DD
:10524300E0C0E0850C08E50E2508F582E50F12762F
:1052530008D0E0125341E0C0E0850C08E50E2508B4
:10526300F582E50F127608D0E0125341126C461214
:1052730008178E828F83A3A3A3A3A3A3A3E0C3339F
:10528300FCE433FD850C08E50E2508FAE50F126CE6
:10529300401208498E828F83A3A3A3A3A3A3A3E0F1
:1052A300C333250CF50CEE24151229926010C0E0CF
:1052B300E50E250CF582E50F127608D0E0F01276A4
:1052C30002126C47120817EE240D122992FC7D007E
:1052D300850B088E828F83A3125641E50828FAE4D2
:1052E30039125325120849EE24111229926027EE30
:1052F300240D122992FD8E828F83A3E0FCAA0EABAC
:105303000F7900120ADAE9600DAA0EAB0F12153CF1
:10531300750E00750F00AA0EAB0F0250B47D00EEA0
:10532300FAEFFB1214A0740322EF127613850E8298
:10533300850F8322124C15125352A3A3A322F00507
:105343000C8E828F8302573312535D12535222E025
:10535300850E82850F83A3A3A322A3A31260FBA3BD
:105363002274F6120356EA2415F582EB122995608E
:10537300047C0180027C008A828B83E0FE900370B0
:10538300125405740278081209DAE5084EFEAF09D3
:10539300EA24121253FF740678081209DAE5084E5C
:1053A300F8E5094FF9ECFDE8FCED49FDEA2411129B
:1053B30053FF740978081209DAE5094DFDEA24164A
:1053C3001253FF740B78081209DAE5094DFDEA243C
:1053D300171253FF740C78081209DAE5094DFD8A98
:1053E300828B83A3A3A3A3A3A3125405740A7808EF
:1053F3001209DAECFAE5094DFB025C16F582EB12B1
:105403004C18E0F5087509002274F612035674FD72
:105413001208DBEAFEEBFFECFAEDFB7401120AACB7
:10542300858208858309780812081B7402120AAC66
:10543300AC82AD83120D98740212084985108285DF
:10544300118312424C7401120AAC12468EE8F0A387
:10545300E912569C148E828F83A312569CC333F891
:10546300E433F97401120AACE028F8A3E039F974C3
:10547300FE28F58274FF39F58312644B7403025CD2
:105483001374F012035674FE1208DB8A0E8B0FECB2
:10549300FEEDFFE98E828F8312566D1258C4850E7E
:1054A30082850F83A3A312563C125901125673121D
:1054B300563C1258F0125673A3A3E0C0E0EE241139
:1054C300127605D0E012567AA3A3A3E0C0E0EE243F
:1054D30012127605D0E0125957600AE50E2408F837
:1054E300E50F12591E8E828F83A3A3A3A3A3A3A3A5
:1054F300A3E060218E828F83A385820C85830D12A6
:105503005641EE2415127605125918850C82850D25
:1055130083E02408F08E828F83A3A3A3A3A3E06078
:105523000F12564D8E828F83A3A3A3A3A312568477
:10553300EE2418122992607C12564DC0E0EE241915
:10554300127605D0E0125684F8E50E28F582E50FB1
:10555300122995C0E0EE241A127605D0E012568483
:10556300125615E433FB12568F7002A3E060458E8A
:10557300828F83A3E0F8E50E28F508E50F12562283
:10558300120817EE2419122992C333FCE433FD7475
:1055930003120AAC12644B12532612084912561511
:1055A300850C82850D83E02A126765EE241B127633
:1055B300051259188E828F83A3E0FA8A08E50E2517
:1055C30008F8E50F340012562C12433EC39AC0E08C
:1055D300EE2417127605D0E0127CE4E06031EE246D
:1055E30017F508EF3400F509850882F583E024F206
:1055F300F0EE241DF8EF12760F240EFAA3E0340028
:10560300FB88828983EAF0A3EB125940C39AF00224
:1056130050AFEE2419F582EF125665C333FA2234E4
:1056230000F509750A00780822F9EE241D12563494
:10563300221272E6E8F0A3E922E0FA025330E0F81E
:10564300E50E28F8E50F3400F9228E828F83A385B7
:10565300820C85830DE0F8E50E28F582E50F1256DE
:1056630065221272E9E022A3A3A3F08A828B83222C
:10567300F0A3E912567A22F0850E82850F83025732
:1056830037F0850C82850D83E004F02212153685F0
:105693001082851183EAF0A3EB1256A0221256A5BD
:1056A300E022F08510828511832274F41203568A56
:1056B300088B09EA125749F0EA1313543F12574271
:1056C300A3A3A3F0EAC41313125749A3A3F0EB1245
:1056D3005727F08A0A8B0B7409780A120A4FE50AD6
:1056E300125727A3F08A0A8B0B740A780A120A4FFF
:1056F300E50A5401C0E0EC2418F582ED127608D0D7
:10570300E0F08A0A8B0B740B780A120A4FE50A122F
:10571300573CF0740C7808120A4FE50812573CA363
:10572300F002474A12572B2254018C828D83800347
:10573300A3A3A3A3A3A3A3A32212572BA3A32254DC
:105743000F8C828D832254038C828D83A3A322C06A
:1057530082C08379008A828B83A3A3A3A3A3A3E03C
:1057630090036A600FE070228A828B83A3A3E070A8
:1057730019098016E060138A828B831264429003B6
:1057830073E06A7003A3E06B70E78003120849D0EB
:1057930083D08202053374F31203568A0A8B0B8972
:1057A3000CECFEEDFF8A828B831258C4850A828536
:1057B3000B83A3A31258BB12590112592F1258BBC2
:1057C3001258F012592FA3A3E0C0E0EE2411127671
:1057D30005D0E0125936A3A3A3E0C0E0EE241212D1
:1057E3007605D0E0125957600AE50A2408F8E50B5C
:1057F30012591E8E828F83A3A3A3A3A3A3A3A3E003
:10580300601B8E828F83A31258D2EE241512760565
:10581300125918850882850983E02408F08E828F47
:1058230083A3A3A3A3A3E060248E828F83A3858293
:1058330008858309E0F8E50A28F582E50B12760866
:105843001258E4F0850882850983E004F0EEFAEF4C
:10585300FB120F5AE9705E8E828F83A3A3A3A3A3C7
:10586300A3123D3B7025E0FC8C08E50A2508FAE508
:105873000B3400FBEE241D125BAFE50CC39CC0E0B0
:10588300EE2417127605D0E0F0802A1258D2740E57
:1058930028F8E43912562C125940FCE50CC39C2419
:1058A300F2C39AFDEE2417127605EDF0AA0AAB0BAC
:1058B3007901120ADA0266FCE0FA850A82850B8313
:1058C300221258CE120F54221272E9E00229B18536
:1058D3008208858309E0F8E50A28F8E50B3400F926
:1058E300221258E822E08E828F83025736A3A3A3A5
:1058F300A3A3E0F9EAF8EE240B124C15E822A3A3C4
:10590300A3E0F9EA8E828F83A302573312670D8EC9
:10591300828F83A3A3E8F0A3E9F0223400F9EE24F5
:1059230013125634124329E02408F022F0A3E9129B
:10593300593622F0850A82850B83025737F01259B4
:10594300452290036BE0F9120AE0E9FA85088285A3
:105953000983E022F074088E828F83A3127CE8A36C
:10596300E022C082C0837AE57B0379E2121CB67A17
:10597300E57B03025792C082C08390037312644B8A
:10598300025792C082C08374FE1208DB85108285A1
:105993001183AA82AB83794B1259A102578F121C30
:1059A300B68510828511831258CE740222C082C03C
:1059B30083794A121CB602579274F6120356900367
:1059C300EDE0FE04F0EEF9120EFAEA7001EB70EE70
:1059D300EE60EBF9025C1674F012035674FE1208C3
:1059E300DB851082851183ECF0A3EDF08A0C8B0D1F
:1059F30089087413120AACE0F50F750900750E00DF
:105A0300851082851183E0FC1210DA8A0A8B0BAEB3
:105A13000AAF0BEE7001EF7018E50F6003025B48ED
:105A2300A908851082851183125BA71210FE025B01
:105A330097E5086020EE2402122992F885080AE50A
:105A43000A28F8E4340013E813F0700974018E8215
:105A53008F83A3A3F0E50F7003025B319003FAE099
:105A63007002A3E060099003FA125C6B121E777454
:105A730012120AACE070588E828F83E07003025BCF
:105A83009714F064026003025B97750E0190036D37
:105A9300E0A2E14003025B63AA0CAB0D125B9A70B8
:105AA30001E97003025B63E50E600D88828983A3BD
:105AB300A3A3A3A3E0C2E0F0E5097003025B978808
:105AC300828983A3A3A3A3A3E0D2E0F0025B679040
:105AD300036DE0A2E150439003FCE07002A3E06099
:105AE3000DEEFAEFFB9003FC125C6B121E778E82B5
:105AF3008F83E0C394045003E004F0E06403700A6E
:105B0300750901AA0CAB0D120E34E48E828F83A3A8
:105B1300F0E5096003025A90807A9003FEE004F0F6
:105B2300FA901A8BE06A706C750901025A90901A08
:105B3300A8E0C0E08E828F83A3A3E0FAD0E0C39AEB
:105B43005052025A8D7401650F7049E50860459003
:105B5300036DE0A2E1503DAA0CAB0D120E3480346C
:105B6300E509603090036DE0A2E15012AA0CAB0D81
:105B7300120B8EE96008AA0CAB0D79008013120F8B
:105B830072EA650C7003EB650D7009AA0CAB0D7915
:105B930001120CF00250AF120BA08A0A8B0BA80A59
:105BA300A90BE822123366AA0CAB0D22F582EF345F
:105BB30000F583EAF0A3EBF02274F612035675089E
:105BC3005F750903780812081B7C6E7D007A217BC0
:105BD3000012159C7402120849E9F508120B1CE91E
:105BE3004208120BCAE9420890033BE07002A3E0AB
:105BF300600C90033B125C6B121E77E94208121D86
:105C0300A6E9420812188AE94208A9088005740D1A
:105C13001208497F020205AD74F6120356121C8660
:105C230075085F750903780812081B75086E7509F6
:105C330000780812081B7C007D007A217B00121576
:105C4300A27404120849120B22120BD090033DE0F8
:105C53007002A3E0600990033D125C6B121E771281
:105C6300144080AF8E828F831263BB2274F61203BB
:105C73005674FF1208DB7E0075085F750903780808
:105C830012081B7C6E7D007A217B0012159C740226
:105C9300120849E96003025D34780812081B75088D
:105CA3006E8E09780812081B7C007D007A217B0028
:105CB3001215A87404120849E97076900373E0641E
:105CC300FE7004A3E064FF60680E900382E0640842
:105CD3006005E064047056EE125D717A8A7B037985
:105CE30043121CBC7A877B037947121CBC7A787BEE
:105CF30003794A123F787A807B037950121CBC7A6D
:105D0300737B037953121CBC7A887B037954121C6E
:105D1300BC7A757B0379E1121CBC90036DE0A2E3AE
:105D23005004D2F08002C2F0125D578004121C8628
:105D33001E120B28120BD690033FE07002A3E06003
:105D43000990033F125C6B121E77120ABCEEF974C2
:105D530001025C13A2F0E492E0125D657952121C19
:105D6300BC22851082851183F0AA82AB8322125D47
:105D7300657942121CBC2274F6120356E9FEA2E0B6
:105D8300502675085F750903780812081B75086E9D
:105D9300750900780812081B7C007D007A217B00BE
:105DA3001215A27404120849EEA2E35003120B2E3B
:105DB300EEA2E15003120BDCEEA2E250139003417A
:105DC300E07002A3E06009900341125C6B121E773E
:105DD300025C1674F412035674EC1208DB7401129D
:105DE3000AAC125EC490877F7808120A6D7583032C
:105DF30075828B78081208F160097405120AAC7475
:105E03000180067405120AACE4F090877F780812CB
:105E13000A6D75830375828F78081208F16009741F
:105E230007120AAC740180067407120AACE4125E0E
:105E330087120AAC125E767407120AACE0700B7418
:105E430005120AACE07003E48002740185108285B8
:105E53001183F0901A30E0901A2FFAE05AFA851065
:105E630082851183E05A125D6B7941121CBC741454
:105E7300024747AA82AB83120EB27AD07B037945DD
:105E8300121CBC22125EB974012274F712035674F9
:105E9300ED1208DBE9FE9003CC1256A5125EC47422
:105EA30012120AACEE125EB9851082851183125E5E
:105EB300767413026898F0901A34E0F97CD07D036D
:105EC30022AC82AD83901A34E0F97AD07B03120EB0
:105ED300B82274F41203568A088B09901A36E064C8
:105EE300FE7004A3E064FF70597A161237F3700151
:105EF300EF604F74018E828F831261E0A3E0600430
:105F03007402800274018E828F83A3F0E508241D3E
:105F1300F582E509125F48125F56A31260E6FCA3FF
:105F2300E0FDEE24020A0A123D30EE241312760538
:105F3300E4125F5D1275FBE509127608126713120E
:105F4300591802474A124C18125F4F22E0F81263A5
:105F5300C1A3221258E8A3A3A322F0125F6222EE88
:105F6300FAEFFB9003CDE0F91214D02274F212037E
:105F73005674FD1208DB8A088B09890C8C0D740199
:105F8300120AAC74041262177001EF7003026016F8
:105F9300126701740788828983F0A3A882A983E525
:105FA300082408FAE5091260291260378A828B8374
:105FB300126036850882850983A3A3A3A3A3A3A3A1
:105FC300A3A3A3E088828983123D6B7401F0EE24BE
:105FD30018127605127C5812621DEE241312602FDC
:105FE3007403650C60067401650C700712602174FC
:105FF300048004126021E4F0901A3612590F7401E0
:10600300650D7006EE2411124E7DEEFAEFFB120CB5
:106013007880027910901A3612604B0224D2124C07
:10602300127440F0A3223400FB02566EF582EF1285
:10603300623322A3E088828983F0A308A98322A381
:10604300A3A3A3A3A3A3A3A374FEF0A374FFF022AB
:1060530074F41203568A088B097A007B041224DE37
:106063001260DC1259187409900382F0120F668AC9
:106073000A8B0BAC0AAD0BE5082413F582E5091274
:10608300760812644B1268636401704A1237F17028
:1060930001EF604274028E828F83F0E508241DF8BD
:1060A300E5091250C312644B8A828B83A3E0FC8AF6
:1060B300828B83A3A3E0FBEC8E828F83A3A3F0A345
:1060C300EB1260F41242511260E6FAA3E0FB794A44
:1060D300121CBC125F6202474A90034612670D907E
:1060E3001A8822A3F0E5082415F582E509125665FE
:1060F300221260FB1260FF22F00250C6E0F8A312E6
:1061030063C2A3A3A32274F412035674FD1208DB23
:106113008A088B097401120AAC74021262177001A7
:10612300EF70030261D9126701740488828983F0D6
:10613300E4A3126209A3A3E06401700874208882B7
:106143008983A3F0850882850983A3A3A3A3A3E07E
:106153006401700988828983A3E0D2E6F08508820E
:10616300850983A3A3A3A3A3A3E06401700A888280
:106173008983A3E0D2E78008EE2413127605740125
:106183001261E0E06401700AEE24161261FC241827
:106193008008EE24171261FC241A1256301261F69D
:1061A300E064017009EE240F12602FA3E4F0850868
:1061B30082850983126312600812298F44041261D5
:1061C300F112621D85088285098312590FEEFAEFD9
:1061D300FB120C788002791074030247471261E4C2
:1061E3002212620DA3A3A322124C12E04420F0A3B7
:1061F300E0F0221261E4A3A322124C15740112628F
:106203000912670DEE2212620D22F08508828509BC
:1062130083A3A3221274A60237F8EE241712623066
:10622300120F66EE241A124C15EA025BB7F582EFE1
:106233001272E97401F02274F612035674F3120811
:10624300DBEAFEEBFF7C0D7D007900851082851172
:1062530083AA82AB831214ACEE241DF582EF125F86
:1062630048E0F854206008740C120AAC7401F0E89A
:1062730054806008740B120AAC7401F0E854406057
:106283000A740A120AAC7401F0800A740A120AAC86
:10629300E064017005EE24138003EE2415124C0B09
:1062A3007402120AACAA82AB83121CA412760212E5
:1062B30063AA125918740A120AACE064017033120B
:1062C3006305703B120F728A088B09A808A909EEAF
:1062D300240B122992687003A3E0697022120F66DF
:1062E300EAFCEBFD7402120AACAA82AB8312686368
:1062F300600D851082851183AA82AB83120CEA029A
:106303005C118E828F83A3A3A3A3A3A3A3A3A3122E
:10631300631622E0FAA3E0FB120FF6E92274F612E9
:10632300035674F31208DB8A088B09ECFEEDFF7C3D
:106333000D7D007900851082851183AA82AB8312BB
:106343007890A3A3A3A3A3A3A3A3A31263AAE8F090
:10635300A3E91263B0A3E0FAA2E55008740B120A92
:10636300AC7401F0EAA2E75008740A120AAC740193
:10637300F0EAA2E6EE5004241380022415124C0B1B
:106383007402120AACAA82AB83121CA4850882850C
:106393000983A3A3E0C0E0740C120AACD0E0126836
:1063A30069120CE4025C1112670D0256A6F0EE248A
:1063B3001D124C151263BB22E0F81263C122A3E045
:1063C300F58388822274F712035674E11208DBEA1C
:1063D300FEEBFF8E828F831243DDA2E0505E8E823E
:1063E3008F83A3E0F9E8FAE9FB8A828B83A3A3A353
:1063F300A3A3A3E054FE1261F1851082851183AC3F
:1064030082AD838A828B8312644FF98A828B83E005
:10641300241CFAA3E012602912644B120F60E97086
:106423001B741D120AAC12645670118510828511FB
:1064330083AC82AD83EEFAEFFB120FCC026896A316
:10644300A3A3A3A3A3A3A3A31258CE22E0241B12A6
:106453006D49221226E5640422E9FA790074046A7C
:10646300600A740A6A600574036A700109020533DD
:1064730074F612035674208A828B83F07401A3A3EB
:10648300F0120C7E8A088B09AE08AF09EE7001EF9B
:10649300600774018E828F83F09003C0E070031253
:1064A300621DEEFAEFFB025C16C082C083901A35C0
:1064B300024410C082C083E9901A35F0025792C09B
:1064C30082C08374019003E2F0E9A2E350037403F2
:1064D300F0E9A2E15004E0D2E2F002579274F6121E
:1064E300035679007C008A088B097808120567F83F
:1064F300FF07136511651165116511650A650E6561
:10650300136507650C80097C0480050C80F67C0804
:106513009003E2E05C6003098003EC600109025C24
:106523001674F4120356EAFEEBFF8908120BA68ACF
:106533000A8B0BA80AA90BE87001E96041888289DC
:1065430083A3A3A3A3E06036C3940550317401650C
:1065530008601A88828983A3A3A3A3E06401600D62
:1065630088828983A3A3A3A3E06402700A88828933
:1065730083126588121E77EEFAEFFB120BB2024705
:106583004A8E828F831258CE90035C1263BB2274AF
:10659300F61203568A828B83E07014A3E07002A381
:1065A300E0600C8A828B8312644A121DE880047AAD
:1065B300007B00025C16C082C0839003BFE06402CC
:1065C300700B900382E06408700312100E0257925E
:1065D30074F312035674DD1208DB8A088B09750CF9
:1065E30000900373E065087004A3E065097025EA71
:1065F3007001EB70030266E89003EEE07002A3E023
:1066030070030266E8750C019003EE125C6B121EB8
:10661300770266F5120BA08A0A8B0BAE0AAF0BEE5C
:106623007001EF70030266E88E828F83A3A3A3A396
:10663300E0640160108E828F83A3A3A3A3E06402AE
:1066430060030266E8E485108285118312671AF8F5
:10665300A3E0F9740B120AAC12676A120B64E970B7
:10666300030266E88E828F8312671312591879002A
:10667300120D7A8E828F83126720120AACAC82AD20
:1066830083740D120AACAA82AB83121CA48E828F70
:10669300831267097415120AAC1259187417120A77
:1066A300ACE4F07C028E828F83A3A3A3A3E0F974EE
:1066B3000D120AACAA82AB83120FB48E828F83129F
:1066C30067097401120AAC12676A120B6A750C012E
:1066D30090877F7808120A6DEE240C1276057808ED
:1066E300120A5E800D900380124C0EAA08AB0912A9
:1066F30010C2A90C74231208497F050205ADEE12DE
:1067030075FDEF124C1812670D22E0F8A3E0F92291
:1067130012670D901A3622124329A3E022EAF0A34E
:10672300EBF0740322C082C08374FE1208DB79018C
:10673300900358125C6B121E77851082851183EAD1
:10674300F0A3EB12676590037312676A7953121C07
:10675300BC85108285118312644B1216E074020209
:10676300578F1256A080A4E8F0A3E912686D227433
:10677300F512035674F31208DBEAFEEBFF8C088D67
:1067830009750A12EE7001EF7005790002685490E2
:106793000373E06E7003A3E06F7018120F66EAFCD8
:1067A300EBFDAA08AB091268637005750A01800343
:1067B300750A00E4851082851183F07401120AAC16
:1067C300EEF0A3EF126869120B58E9602B74031201
:1067D3000AACAA82AB83120B3AE96401701A750AF8
:1067E300017403120AACAC82AD83AA08AB09126828
:1067F300636021750A00801C7412650A7016900389
:10680300BFE06402700EAC08AD09EEFAEFFB120BA9
:1068130088E970DFAC08AD09EEFAEFFB1210E0E98E
:10682300FA740A6A7005750A01801D74A06A7012F1
:10683300AC08AD09EEFAEFFB1210F2EEFAEFFB1221
:10684300110A7401650A7007EEFAEFFB121020A912
:106853000A740D1208490248AD2421FAE93417FBE2
:10686300121C9EE922E412686D2212687122F085DF
:106873001082851183025D6C74F7120356EAFEEBF6
:10688300FF12100E790DEEFCEFFD7AFC7BFF121068
:106893002C8005741F1208497F010205AD74F7129D
:1068A3000356EAFEEBFF7508008E828F83A3A3A332
:1068B300A3A3A3A3A3E06017EE24151276361276E2
:1068C3000312644B12101AE9640170037508018EF8
:1068D300828F83A3A3A3A3A3A3A3E06018EE24132F
:1068E3001276051268FCFAA3E0FB12101AE96401A0
:1068F3007003750801A908809F126902023D61E0D7
:10690300FCA3E0FD02469374F212035674FD1208D1
:10691300DB8A088B09ECFEEDFF890C750D01740110
:10692300120AAC74041274A17001EB602B1269603B
:1069330012760812696688828983F0A3E50CF0EE6B
:1069430088828983A3A3F0EF8882898312566A120F
:106953007C56120C78E9F50DA90D0224D2EA1275C2
:10696300FDEB2212670D74032274F7120356EAFE3D
:10697300EBFFEE241D1276051269D7FC888289830A
:10698300A3A3A3E0FBECFA88828983A3E012072286
:10699300010002A169020CAD690DA869B069790112
:1069A300120CF680081210088003121704126305F4
:1069B300601DEE2411122992C39402401212760232
:1069C300126FC27003A3E0696005120F7E80027923
:1069D3000002689B12762BA3E02274F01203567414
:1069E300F31208DB7403120AACECF0A3EDF08A0E89
:1069F3008B0F890B741D120AACE0F50A7E01EE12AF
:106A03000AAC740AF0E97007E50AC333240AF08577
:106A13001082851183AA82AB83120FDE8A088B0949
:106A2300EA7001EB7003026AD81250CB7409126C3E
:106A33006C450A126C79120AAC126C4FE50B70307C
:106A43007A008026EAC333F8E433F9741E120AACE1
:106A5300E028F8A3E039F988828983126AE58882FD
:106A6300898312424BA30EAF830AEAC3950A40D42B
:106A7300E5082417F582E509126032120F66E5086E
:106A8300241AF582E509125BB27405120AACAC82D2
:106A9300AD83AA0EAB0F120B40E96021E508126A21
:106AA300E0E5091260327405120AACA882A983E5F5
:106AB300082418F582E50912760812591885088208
:106AC300850983A3A3E50EF0A3E50FF0AA08AB099C
:106AD300120C78E9FEEEF9740D0250B1E82416F5B4
:106AE3008222124251F0A3AE82AF832274F01203CA
:106AF3005674F81208DB8A0E8B0F126B86FA741F1A
:106B03005AF50A74E05A126CB76073E508706FE5C2
:106B13000AC333FA7B00126FA57001EB60607C003F
:106B230080288E828F83E0FAA3E0F9E42AE9FBEC64
:106B330033F8E433F9E50828F582E50939125BB443
:106B4300EE24020E0EEF3400FF0CECC3950A40D284
:106B5300780812081B780A12081F7403120AACACD7
:106B630082AD837900E50E1275FDE50F12760812EA
:106B73006FAE7403120849AA08AB0912153C7408D6
:106B83000250B1EA241DF582EB1256652401FEA3DF
:106B9300E03400FF02433F74F012035674FE120800
:106BA300DB851082851183125BB689088C0E8D0FED
:106BB3007412120AACE0F50B90122AE07002A3E003
:106BC3006075E50BC333F8E433F9740E28FAE4393E
:106BD300FB1214C48A0C8B0DAE0CAF0DEE7001EFDB
:106BE300605574D48E828F831267651259128E8218
:106BF3008F83A3A3A3A3E508F0AC0EAD0FEE24058A
:106C0300123D2FEE240D127605E50BF07413120AD4
:106C1300AC126C47120817E50BC333FCE433FDEEEB
:106C2300240EFAEF126C40120849EEFAEFFB9012B1
:106C33002A125C6B121E770250AFFAE50D3400FB8B
:106C4300025326A3E0F508A3E0025624123366EEAE
:106C5300FAEFFB126C5A22121CA4EE2408FEEF3446
:106C630000FF229003800233668E828F83F0A3E5B8
:106C73000BC43354E022F0A3AE82AF8374032274B7
:106C8300F712035674F81208DB126B8654E0126C89
:106C9300B7601CE50870188E828F83A3E0FA8E829A
:106CA3008F83A3A3E0FB8E828F83E0F912105C74C1
:106CB30008026898F508A3AE82AF83EEFCEFFD856A
:106CC3001082851183AA82AB83126C5A8510828548
:106CD3001183AC82AD837A947B0302686374F712E9
:106CE300035674E11208DBEAFEEBFF126D3E7002FD
:106CF300A3E060448E828F8312644B8510828511DA
:106D030083126D507409120AAC126FC27003A3E0B0
:106D1300696025125C6712069D741A120AACE0F9C9
:106D2300740B120AAC124C0E740D120AAC12644BA3
:106D3300120E2E7402120849026896126D42228EB8
:106D4300828F83E0241CF8A3E012761722AC82AD75
:106D530083EA241BF582EB122ABEEA241CF582EB9C
:106D63001258CB120F4E2274F7120356E9FE7C0021
:106D73007D0078007900800C126E3A2CFCA3E03D74
:106D8300FD1277A5127BDE5037E8FAE9FBEA75F0CE
:106D930012A4FAAFF075F012EBA42FFBEA24A9F5C5
:106DA30082EB3415F583E064FF60D6126E3A70020D
:106DB300A3E060CDEE60C1126E3FE4F0A3F080C1AA
:106DC30078007900800C126E192CFCA3E03DFD12B3
:106DD30077A5127BD15038E8FAE9FBEA75F017A4DE
:106DE300FAAFF075F017EBA42FFBEA127BCCEB1292
:106DF3007A077004A3E064FF60D5126E197002A3D2
:106E0300E060CCEE60C0126E1EE4F0A3F080C0EC34
:106E1300FAEDFB02689B126E1EE022E8FAE9FBEA38
:106E230075F017A4FA75F017EBA42FFBEA2434F5D9
:106E330082EB3417F58322126E3FE022E8FAE9FB76
:106E4300EA75F012A4FA75F012EBA42FFBEA24B54D
:106E5300F582EB3415F5832274F7120356EAFEEB41
:106E6300FF9003CCE0C399501B120FA89003F012BC
:106E73006EEB900366E075F064A4FCADF07A007BE2
:106E8300021224E902689B74F6120356EAFEEBFF32
:106E93009003E3801388828983E06E7003A3E06F1D
:106EA300603F88828983A3A31249C27001E970E518
:106EB3007A047B001215368A088B09A808A909E809
:106EC3007001E9601C88828983126EEB9003E312E0
:106ED300644B88828983A3A3125BB69003E31259A0
:106EE30018025C16A3A3A3A3EEF0A3EFF02274F49D
:106EF3001203567E009003E380070E88828983A3E2
:106F0300A31249C27001E970F1EEC333FAE433FB13
:106F1300126FA57001EB7003026F9F7F009003E374
:106F2300802488828983124C0EEFC333FAE433FB47
:106F3300E5082AF582E5093BF583ECF0A3EDF00FB4
:106F430088828983A3A31249C27001E970D4900394
:106F5300C8126FC27003A3E0697808701912081B86
:106F6300EEF50A780A12081F7C947D0379009003DA
:106F7300C8126FAE801A12081BEEF50A780A1208BF
:106F83001F7C947D0379009003C812644B12103860
:106F93007403120849AA08AB0912153C120C8A02A1
:106FA300474A1215368A088B09EA221258CE121064
:106FB30044228E828F83A3A3A3A3A3A3A3A3A31279
:106FC300670D900373E06822C082C08380128A82B7
:106FD3008B83A3A31267099003E312591812153C7C
:106FE3009003E31249547001EB70E302579274F675
:106FF3001203569003801250D49003F012380212F9
:1070030059187AF07B037950121CBC9003F0127666
:107013003CFAEFFB1211049003F01250D490122C9F
:10702300E07002A3E0602D7A067B001214C4EA70BC
:1070330001EB602074D58A828B83F0E4A3A3F07400
:10704300018A828B8312566A126EE790122C125CAD
:107053006B121E77025C16C082C0839003F27486A3
:10706300F0A37410F09003F47480F0A37410F09004
:1070730003F6749EF0A37410F0025792C082C0838B
:10708300900373E064FE7004A3E064FF600E90035A
:107093006DE0A2E150061210E612108C1210860267
:1070A300579274F61203569003C1E060281214BE7F
:1070B3008A08A8089003C1E0FA75F0E8A4CAACF006
:1070C30075F003A42CFB747F582AFCE43BFD7A0083
:1070D3007B011224E9025C1674F012035674FE124B
:1070E30008DB750F00851082851183E4F0A3F0128D
:1070F3000BE87A047900120B76EAFE7A0279011220
:1071030072BF7A0379031272BF1210BCEAF50E2E16
:10711300FF8E0AEA250AF8E43400F9E87001E97001
:107123000302721F8F08750900740278081209DAC6
:10713300AA08AB0912568F7002A3E0700302721DF6
:107143008F08750900740278081209DAAC08AD09D2
:1071530079FF851082851183E0FA1214AC7508005B
:107163008056A908120BE28A0C8B0DEA7001EB60C2
:10717300458A828B83A3A3A3A3E0600464047036CF
:10718300050F8A828B83A3A3A3A3A3A3A3A3A3A370
:10719300E0F91210F885108285118312069DEFFD28
:1071A300850C82850D83A3A3A3A3A3A3A3A3A3E019
:1071B3001272C8120849050885080A90229BE493B5
:1071C300F8740193F9C3E50A98E4995006E50FC3EF
:1071D3009E408F750800E508C3950E503FAA087BB3
:1071E300001210C88A0C8B0DEA7001EB6028851021
:1071F3008285118312069DEA240EF582EB122995EE
:10720300FEEA240FF582EB122ABA1210F8EFFDEE14
:107213001272C8120849050880BC7F0075096A907C
:10722300036BE0600CF9120AE0E9FA745CC39AF5A7
:107233000975F003E50984F50A851082851183E059
:10724300F50EA3E0F50F750B00E5096006750B203D
:10725300750900E50AC39F5004AE0A8008EFFEE5F6
:107263000BD2E6F50BAC0EAD0FAA0BEEF91210988C
:10727300E9F50CE50BA2E6401F1E750800800EE53C
:107283000E2404F50EE50F3400F50F0508E508C3D9
:107293009E40ECEECFC39FFFE97006E50BA2E650DC
:1072A300A5851082851183E07002A3E06009851033
:1072B300828511831272DBA90C0250AF120B76EA9E
:1072C300CEC39EFE22FC850C82850D831258CE12FE
:1072D30010927402221272DF1272EE22EE240C124A
:1072E30072E622F582EF3400F58322E0FAA3E0FB95
:1072F30012153C2274F2120356EAFEEBFF8908745E
:107303000E120AAC12644B750A00750B0075090066
:10731300800E8A0A8B0BEA2404FAEB3400FB05097E
:10732300E509C39D50218A828B83E064FF7004A327
:10733300E064FF70158A828B83126EEBEC8A828B7A
:10734300831273DBE508F00224D7E50A7002E50B2C
:10735300600E850A82850B83C3E09EA3E09F50B233
:107363008A828B83126709C3EE98EF9950A4EAF8D7
:10737300EBF988828983E064FF7004A3E064FF6013
:1073830010E82404F8E93400F90509E509C39D4030
:10739300E1880A890BE824FCF8E934FFF98882893B
:1073A30083E0F50CA3E0F50D850A82850B83E50CDC
:1073B300F0A3E50D1260FB1273CF12535F1273CF6C
:1073C300A3F0C3EA98EB9940C8027338A3A3E085FE
:1073D3000A82850B83A3A322A31273E022A3F08A5C
:1073E3008202425E74F312035674FD1208DB8908AD
:1073F3008A09ECFEEDFF750C0175F003E9A4240284
:10740300C0E07401120AACD0E01274A17001EB6009
:107413007C12696012760812749B88828983F074E7
:107423001F55084509A3F01275E9750900803D8EC3
:10743300828F83E088828983F0A3A882A9838E82C6
:107443008F831260368E828F83A3A3E05407C4C058
:10745300E08E828F83A3A3A3E05407FCD0E04C12F9
:107463006038EE2404FEEF3400FF0509E509C395F7
:107473000840BC8A828B83A3A374FC12604DEA2468
:1074830013F582EB126032120C78E9F50CA90C7437
:10749300030266F98E828F8312670D7408221274B9
:1074A300A6EA22126871120FDE2274F11203568AC1
:1074B3000A8B0B7508007AFE7BFF7CFE7DFFE50AD5
:1074C300241DF582E50B127608127627E0F5097480
:1074D3001F5509F50C1275E9E50C600B8882898349
:1074E300E0FEA3E0FBEEFA750D008030888289830D
:1074F300E0FCA3E0FFECFEE824020808E912760FA3
:107503005407F50EA3A882A983EFFD900373E06EE1
:107513007003A3E06F7003850E08050DE50DC39599
:107523000C40C9E508700BA9091210A4E970030205
:1075330075E61275F31276208A0C8B0DA80CA90D33
:10754300E87001E9600EE488828983127A21E508F4
:10755300F00275E67CFF7DFF1275F3127608126464
:107563004B1210B08A0C8B0DAE0CAF0DEE7001EF09
:107573007033127CD77001EF60697C177D0079004E
:107583001214AC1275F3127608123D40125918907A
:107593000380127641A3125916EE240F127CF0EEEB
:1075A300240E12602FEE240E127605E508F0EE2469
:1075B3000C124E7DEE2402FAEF3400FB120B3AE973
:1075C3007021850A82850B83A3A3A3A3A3A3A3A3EB
:1075D300E06010E50A2415F582E50B1276392402E2
:1075E300123D2F02467CE824020808E93400F92200
:1075F300E50A1275FDE50B22E508240BF58222EE60
:10760300240BF582EF124C1822F8E50912761322A7
:10761300127617223400F988828983E0221258CB2C
:10762300120BA02212762B22E0F8A3E0F9888289BC
:1076330083A322F582EF124C18123366EE22123D19
:1076430044025734C082C08374FE6A700374FF6BB4
:10765300700479018034746059646060F5E9A2E5CF
:10766300500F900373126709C3EC98ED994019808A
:10767300E1A2E69003735008C3E09AA3E09B80ED78
:10768300C3E09AA3E09B50DA790002579274F71291
:1076930003567E0080041276AB0E9022A6E493FA82
:1076A300EEC39A40F102689BEE75F017A4241FFA0B
:1076B300E5F03417FB1210CE2274F712035678004C
:1076C300790080031277A59022A6E493FEC3E89E77
:1076D300E994005064E8FEE9FFEE75F017A4FE8517
:1076E300F00875F017EFA42508127C4BE06A7003CD
:1076F300A3E06B70CFE8FEE9FFEE75F017A4FE750B
:10770300F017EFA42508FFEE2429F582EF3417F5CF
:1077130083E06C7003A3E06D600A74FF6C70037404
:10772300FF6D70A0E875F017A4F8AAF075F017E9DB
:10773300A42AF9E812786280047A007B0002689B2D
:1077430074F61203567CFF7DFF7AFE7BFF1210B0A6
:10775300EA7001EB704978007900803EE8FCE9FDAE
:10776300EC75F017A4FCAEF075F017EDA42EFDEC4C
:10777300242EF582ED3417F583E0701BE8FAE9FB5C
:10778300EA75F017A4FAACF075F017EBA42CFBEA3A
:10779300241FFAEB3417FB1277A51277F040BD02D2
:1077A3005C16E824010275ED74F71203567A007B28
:1077B3000078007900802EE8FCE9FDEC75F017A451
:1077C300FCAEF075F017EDA42EFDEC127BCCED12A0
:1077D3007A077004A3E064FF6008EA24010AEB342B
:1077E30000FB1277A51277F040CD02689B9022A68A
:1077F300E493FCC3E89CE994002274F41203568AD0
:10780300088B09ECFEEDFF800B1210CEEEFCEFFDB2
:10781300AA08AB091210B0EA7001EB70EC02474AF8
:1078230074F61203567E007D0080020E0D9022A690
:10783300E493FCEDC39C501CED1279FF7004A3E0AC
:1078430064FF60E88E08EA65087001EB70DDED12F5
:10785300785E80047A007B00025C1675F017A4241E
:107863001FFAE93417FB2274F7120356EAFEEBFF03
:10787300EE7001EF600E12788A12604B8E828F8356
:10788300A312604202689B7C177D0079001214AC3E
:10789300023D4974F7120356EAFEEBFF75080080B8
:1078A30018A808E875F017A4A9F0127D647003A363
:1078B300E06F6003127D6A05089022A6E493FAE55F
:1078C30008C39A40DC02689B74F41203568A088B3F
:1078D30009ECFEEDFF900380E06E7003A3E06F7090
:1078E30012125B9A7001E9600AE82408FAE934008D
:1078F300FB8022EEFCEFFDAA08AB091210B08A0848
:107903008B09A808A909E87001E96005E8240D803E
:10791300DB7A007B0002474A74F4120356EAFEEB5B
:10792300FF8C0A8D0B7508007509008036E5097513
:10793300F017A42421FAE5F03417FB120B3AE9609F
:1079430020A809127DA87003A3E06F700375080ACD
:10795300AC0AAD0BE875F017A412685C600343082A
:10796300A005099022A6E493FAE509C39A5004E519
:107973000860BA022AAA74F61203567E008024EE27
:10798300F9120BE2EAF8EBF9EA7001EB6014E82470
:1079930007127A0F500CE488828983A3A3A3127A77
:1079A30021F00E8E0890229BE493F8740193F9C39F
:1079B300E50898E49940C87E0080321279FE70048D
:1079C300A3E064FF6026EE75F017A4241FF8E934E2
:1079D30017F9E8240C127A0F5012E8240FF582E904
:1079E300124E80E8240EF582E9124E800E9022A6F4
:1079F300E493FAEEC39A40C3025C16EE127BC6E927
:107A0300127A07223417F583E064FE22F582E91225
:107A13005665FA74012AF09003C2E0C39A22A3A325
:107A2300A3A3A312535D02573374F41203568A08B7
:107A33008B09ECFEEDFF750A007C007D01801012BE
:107A430014BEE50AF5F0EA84ACF0750A007D00780F
:107A530000790080031277A5127BD14003027AE4F8
:107A6300E8FAE9FBEA75F017A4FA85F00B127BB389
:107A730064FE7004A3E064FF60DB127BA9650870F9
:107A830004A3E0650960CE127BA96E7003A3E06FC7
:107A930060C3E8FAE9FBEA75F017A4FA75F017EB8F
:107AA300A4250BFBEA242DF582EB3417F583E06064
:107AB300A4C39407509F74016D050A6098E50AC337
:107AC3009C4092E875F017A4F8AAF075F017E9A4A2
:107AD3002AF9E8127BCCE93417F58312644B027B55
:107AE300887800790080031277A5127BDE507DE849
:107AF300FAE9FBEA75F012A4FA85F00B127B9564A0
:107B0300FE7004A3E064FF60DE127B8B65087004E3
:107B1300A3E0650960D1127B8B6E7003A3E06F60F5
:107B2300C6E8FAE9FBEA75F012A4FA75F012EBA4C1
:107B3300250BFBEA24AEF582EB3415F583E060A751
:107B4300C3940750A274016D050A609BE50AC39CA8
:107B53004095E875F012A4F8AAF075F012E9A42A8A
:107B6300F9E824A5F582E93415027ADCE50A601107
:107B7300EC700E7401650A6003027A427C01027A9A
:107B83004D7AFE7BFF02474AE8FAE9FBEA75F012F9
:107B9300A4FA75F012EBA4250BFBEA24A5F582EBFE
:107BA3003415F583E022E8FAE9FBEA75F017A4FA45
:107BB30075F017EBA4250BFBEA127BCCEB3417F51E
:107BC30083E02275F017A4A9F0241FF582229022E6
:107BD300A6E493FAC3E89AE994002290229BE493E3
:107BE300FA740193FBC3E89AE99B2274F4120356D7
:107BF3008A088B098C0A8D0B7E007F008008EE2497
:107C0300010EEF3400FF9022A6E493F8C3EE98EF41
:107C130094005031AC0AAD0BEEF8EFF9E875F017AC
:107C2300A4F8AAF075F017E9A42AF9E812685C60D1
:107C3300CDEE75F017A4FEAAF075F017EFA42A1283
:107C43007C4B127C5802474AFFEE127BCCEF341771
:107C5300F58322A3A3E508F0A3E509F022E9FA7965
:107C630007C3940D400479018019EAC394074004C3
:107C73007903800FEAC39403400419198005EA705D
:107C830002790002053374F01203568A0E8B0F8CAF
:107C93000A8D0B8908127CD77001EF603412788A41
:107CA300E50EF0A3E50F127CE4A3A3A3A3E50AF07A
:107CB300A3E50BF0E508600AEE240F127605E5084C
:107CC3008008EE240F1276057401F0EE240E127C68
:107CD300F00250B41210B68A0C8B0DAE0CAF0DEE41
:107CE30022127CE822F08E828F8302573512623093
:107CF300EE240D124C157402F02274F51203568A09
:107D0300088B09ECFEEDFF750A008014E875F01787
:107D1300A4127D647003A3E06F6003127D6A050AF9
:107D23009022A6E493FAE50AC39A5024A80AE875B8
:107D3300F017A4A9F0127D56E065087004A3E0656E
:107D43000970C9E875F017A4127D56126EEB80CE48
:107D53000248AD127D5A222429F582E93417F583AE
:107D630022127D5AE06E22E812785E1210CE22743F
:107D7300F7120356EAFEEBFF7508008019A80812F4
:107D83007DA87003A3E06F700BE8127DE07005E53A
:107D9300081276AC05089022A6E493FAE508C39A84
:107DA30040DB02689BE8127BC6E93417F583E06E7B
:107DB3002274F71203567E0080151279FE7004A315
:107DC300E064FF6009EE127DE070031276AB0E9063
:107DD30022A6E493FAEEC39A40E002689B75F0177B
:107DE300A42421FAE93417FB120B3AE922C082C01A
:107DF300839003F8741CF0A37411F09003FA7422B7
:107E0300F0A37411F09003FC7428F0A37411F00232
:107E1300579274F4120356EAFEEBFF1243DA7035FD
:107E23008E828F83A3A3A3A3A3A3A3A3A312069DBD
:107E3300900344125C6B7808120A6DAA08AB09AC74
:107E43000AAD0B8E828F83A3E0F9120CFC7402122D
:107E53000849120C8A02474AC082C0839003CA129F
:107E63007F0CF09003CAE07002A3E0700579011261
:107E7300105602579274F612035674FC1208DBEA8A
:107E83002408F8EB1250C3127F0C1246A17002A310
:107E9300E09003CA700BE4F0A3F07901121056804E
:107EA30063C3E09415A3E09400405979001210567F
:107EB3008A088B09AC08AD09ECF8EDF9E875F064B4
:107EC300A4F8AAF075F064E9A42AF99003CA12642D
:107ED3004B12020DE8941AE994004028901224E012
:107EE3007002A3E0601E9003CA1263AA12591874A9
:107EF30002120AACECF0A3ED126869901224125C32
:107F03006B121E777404025C13E02401F0A3E034C7
:107F13000022C082C08374F81208DB8510828511A9
:107F230083AC82AD83758387758239740812079594
:107F3300851082851183AC82AD83126863640170FE
:107F430004790080027901740802578FD083D082AC
:107F5300020533C082C0838019198C828D83E08A25
:107F6300828B83F0A3AA82AB838C828D83A3AC82A2
:107F7300AD83E970E480D5C082C083801D198A82F5
:107F83008B83E08C828D83F08A828B83A3AA82AB5E
:107F9300838C828D83A3AC82AD83E970E080AD7462
:107FA300F7120356EAFEEBFF8908E970031218CCB7
:107FB3008E828F83E0F5D9A3AE82AF831508E508DF
:107FC30070EE7F010205AD74F7120356EAFEEBFF74
:107FD3008908E970031218CCE5D98E828F83F0A348
:0C7FE300AE82AF831508E50870EE80D672
:108000000000000000000000000000000000000070
:10801000000000F800000000000000333000000005
:1080200000100C06100C060000000000000000000C
:1080300040C07840C0784000043F04043F0404007E
:10804000007088FC08300000001820FF211E00008E
:10805000F008F000E018000000211C031E211E00A3
:1080600000F00888700000001E2123241927211029
:1080700010160E00000000000000000000000000CC
:10808000000000E018040200000000071820400073
:1080900000020418E0000000004020180700000063
:1080A000404080F0804040000202010F01020200C7
:1080B000000000F0000000000101011F01010100AB
:1080C000000000000000000080B070000000000010
:1080D0000000000000000000000101010101010199
:1080E0000000000000000000003030000000000030
:1080F0000000000080601804006018060100000005
:1081000000E010080810E000000F102020100F0001
:10811000001010F8000000000020203F2020000088
:1081200000700808088870000030282422213000E0
:1081300000300888884830000018202020110E00E8
:108140000000C02010F8000000070424243F240091
:1081500000F80888880808000019212020110E0066
:1081600000E0108888180000000F112020110E0078
:1081700000380808C83808000000003F0000000070
:108180000070880808887000001C222121221C0031
:1081900000E010080810E0000000312222110F005A
:1081A000000000C0C00000000000003030000000EF
:1081B000000000800000000000008060000000005F
:1081C0000000804020100800000102040810200078
:1081D00040404040404040000404040404040400C3
:1081E0000008102040800000002010080402010058
:1081F000007048080808F000000000303601000058
:10820000C030C828E810E0000718272423140B000A
:108210000000C038E0000000203C23020227382084
:1082200008F8888888700000203F202020110E0068
:10823000C03008080808380007182020201008005F
:1082400008F808080810E000203F202020100F0048
:1082500008F88888E8081000203F20202320180014
:1082600008F88888E8081000203F2000030000007C
:10827000C03008080838000007182020221E02001D
:1082800008F808000008F808203F210101213F20DC
:10829000000808F8080800000020203F2020000007
:1082A00000000808F8080800C08080807F000000F7
:1082B00008F888C028180800203F20012638200030
:1082C00008F8080000000000203F20202020300097
:1082D00008F8F800F8F80800203F003F003F2000B1
:1082E00008F830C00008F808203F200007183F00B9
:1082F000E01008080810E0000F10202020100F00E8
:1083000008F808080808F000203F210101010000DA
:10831000E01008080810E0000F18242438504F001F
:1083200008F8888888887000203F2000030C3020DF
:1083300000708808080838000038202121221C001D
:10834000180808F8080818000000203F2000000066
:1083500008F808000008F808001F202020201F004F
:108360000878880000C83808000007380E010000AF
:10837000F80800F80008F800033C0700073C030079
:10838000081868808068180820302C03032C3020DF
:108390000838C800C83808000000203F200000004E
:1083A00010080808C83808002038262120201800A6
:1083B000000000FE020202000000007F404040007A
:1083C000000C30C000000000000000010638C000B2
:1083D00000020202FE000000004040407F0000005A
:1083E000000004020202040000000000000000007F
:1083F000000000000000000080808080808080807D
:108400000002020400000000000000000000000064
:1084100000008080808000000019242222223F205A
:1084200008F8008080000000003F112020110E009D
:108430000000008080800000000E1120202011002C
:10844000000000808088F800000E112020103F20DE
:108450000000808080800000001F22222222130062
:10846000008080F0888888180020203F20200000AD
:108470000000808080808000006B94949493600062
:1084800008F8008080800000203F210000203F206D
:1084900000809898000000000020203F202000006D
:1084A000000000809898000000C08080807F00005D
:1084B00008F8000080808000203F24022D3020003A
:1084C000000808F8000000000020203F20200000E5
:1084D0008080808080808000203F20003F20003FFF
:1084E0008080008080800000203F210000203F200D
:1084F0000000808080800000001F202020201F00BE
:10850000808000808000000080FFA12020110E00EC
:108510000000008080808000000E112020A0FF80DD
:10852000808080008080800020203F21200001008A
:1085300000008080808080000033242424241900DF
:10854000008080E0808000000000001F20200000EC
:108550008080000000808000001F202020103F202D
:10856000808080000080808000010E3008060100BD
:1085700080800080008080800F300C030C300F0062
:1085800000808000808080000020312E0E3120008D
:10859000808080000080808080818E7018060100BD
:1085A00000808080808080000021302C22213000DB
:1085B00000000000807C020200000000003F4040FC
:1085C00000000000FF00000000000000FF000000AD
:1085D0000002027C800000000040403F00000000DC
:1085E0000006010102020404000000000000000077
:1085F000000000000000000000000000000000007B
:1086000000000000000000000000000000004E4DCF
:108610002D656E65726779206E6F74207570004FDE
:10862000727068616E20526573706F6E7365001AA8
:1086300013460EEA185A1ED61D621646172C1653FC
:1086400074617274446576696365204552520041D5
:1086500073736F6320436E66206661696C004173BB
:10866000736F6320527370206661696C004D617492
:10867000636820446573632052657100456E6572BE
:108680006779204C6576656C004D4F444520756ECA
:108690006B6E6F776E005A696742656520436F6F36
:1086A0007264004E6F6E204D617463686564004EA5
:1086B0006574776F726B2049443A000B050F010017
:1086C00000026B87026B875363616E204661696CA1
:1086D00065640000000000000000000000000000D1
:1086E000000000000000000053657269616C417079
:1086F000700000000000000000000000000000000A
:108700000000000000004173736F6320436E660039
:108710005273702053656E74005375636365737391
:1087200000526F757465723A00506172656E743AEA
:1087300000FFFFFFFFFFFFFFFF0000000000000041
:1087400000494545453A20004661696C6564000B67
:108750000C11BB860053656E740002050200010017
:108760000000FF3000000064000000010000001065
:108770002700000100000000E1F50500F8FF0700F8
:108780000000000058000000000C003A20003000FB
:108790000874F612035674FF1208DBE48510828514
:1087A0001183F0858208858309780812081B7508F3
:1087B00001750900780812081B12A0C31208497439
:1087C00001029EAC74F61203568C088D09780812CB
:1087D000081B75080B750900780812081B12A0C346
:1087E000029EAC74F61203568C088D0978081208A4
:1087F0001B75080B750900780812081B12A0CE1211
:108800009FD7029EACC082C0838A828B83E0D2E76E
:10881000F012170A02A79FC082C083790012889FB6
:10882000C082C08390033012B869D083D082C3E085
:108830009CA3E09D500C12ADCEFAA3E0128910600B
:10884000010902A79F74F712035612889F128A4BE0
:10885000AEF075F00BEDA42EFD900332E02CFEA3DC
:10886000E03DFF740169600574026970208A828BA3
:1088700083A312B9CB12C9A97402697018128CCBE8
:10888000128DDB7010E48E828F83F08008EA24035F
:10889000FCEB128DC3EEFAEFFB120AF8029A841277
:1088A000C070EB12BC6B2274F41203568A088B0959
:1088B00012B9D179008A828B83E0604E7E007F00FE
:1088C000804312890D703B128A97F50AA3E039F5AF
:1088D0000B850882850983E08C82850B8312A48234
:1088E000F8A3E0F98C82850B83128DE3FCE5091275
:1088F0008D59128DCB12BC70AA0AAB0B120AF8125A
:10890000BEFD129239128CD340B802A47DEEFAEF6C
:10891000FBEA75F00BA4FAACF075F00BEBA42CFBA2
:1089200090033212CD69F583E0540F2274F51203DF
:10893000568A088B09740B120AAC12BF02750A0121
:10894000EC7001ED6026EC128EB1ED12AAA4790153
:10895000120B04EE7001EF606E8E828F83A312B94A
:10896000D97902EEFAEFFB120B04805BEE7001EF97
:108970006031128EB0EF12AAA4EE2403FAEF128D2A
:10898000D5700CAA08AB09120B0AE9F50A80CAE5F2
:10899000082403FAE509128DD5702C7903AA08ABD7
:1089A0000980C48A828B83A3E064FE7004A3E06420
:1089B000FF7005128DD2700CAA08AB09120B0AE9E0
:1089C000F50A8003750A00029B0774F7120356909C
:1089D000033012AD61EA7001EB6031EA75F00BA46F
:1089E000FAACF075F00BEBA42CFBEAFEEBFF1215D2
:1089F0003690033212AD61900332E07002A3E06062
:108A000012EEFCEFFD79001214AC8007900332E403
:108A1000F0A3F0029A8474F61203567508007509E3
:108A200000780812081B900330128A4BAAF075F0E8
:108A30000BEDA42AFD7A237B0012159C7402120808
:108A400049E9FE6003120B22029E8C12B86DEC7590
:108A5000F00BA4FC2274F71203567E007F00800AFC
:108A6000EEFAEFFB120AE6129239128AEB40F1029B
:108A70009A8474F71203567E007F008012128A9740
:108A8000FCA3E039FDEEFAEFFB120AF21292391262
:108A90008AEB40E9029A84EEF8EFF9128AD8E028CE
:108AA0002274F71203567E007F008020128AD412AF
:108AB000BA3E88828983E0A2E7500EC2E7F0AC821A
:108AC000AD83EEFAEFFB120AEC129239128AEB40F8
:108AD000DB029A84EEF8EFF9E875F00BA4F8AAF03F
:108AE00075F00BE9A42AF99003322290033012AA00
:108AF000C5C3EE98EF9922C082C083EC7001ED608F
:108B000005121CA480097C087D0079001214AC02B7
:108B1000A79F74F61203567900EA7001EB60177C88
:108B2000008C08EA250812BEF6600479017C080C66
:108B3000ECC3940840EB029EAF74F712035674F333
:108B40001208DBECFEEDFFE4851082851183F074E2
:108B500001120AAC12A0FA120B587403120AACAC40
:108B600082AD83EEFAEFFB120B34EEFAEFFB120B41
:108B70003A029A7F74F712035674F31208DBECFE84
:108B8000EDFFE4851082851183F0EAFCEBFD7403B0
:108B9000120AAC12A1317401120AAC128EB512AADB
:108BA000AE74FE68700374FF696004790180027915
:108BB00000029A7F74F7120356EAFEEBFF128C0252
:108BC0007010128C0D64FFFC8A828B83E05CF012C3
:108BD0000AF802A3E774F7120356EAFEEBFF7508E2
:108BE000008E828F83E06017128C027012128C0D3F
:108BF0008A828B83FCE05C7006E04CF0120AF8027B
:108C0000A3E7120AFEE9F5087401650822EE12C016
:108C100071EF12AAC1128AD8E028FAA3E039FB8EBC
:108C2000828F83E02274F41203568A088B097C0039
:108C30007D00128CCB128DCBE508128EB1E50912A6
:108C4000B9D57900850882850983A3E064FE7004A4
:108C5000A3E064FF60727E007F00806712890D6070
:108C60005FEEFAEFFBEA75F00BA4FAACF075F00BCF
:108C7000EBA42CFB900332E02AF50AA3E03BF50BB2
:108C8000850882850983A312B9C0850A82850B8372
:108C9000A3E06A7003A3E06B7026E50A2403FAE5FB
:108CA0000B128DD57014E50A2403FCE50B3400FD8E
:108CB000E5082403FAE509128DCB12BC7012BEFD43
:108CC000129239128CD3409402A47DEA24030A0A3A
:108CD0000AEB2290033012B9C7C3EE9AEF9B2274BD
:108CE000F21203568A0A8B0B8A828B83A312B9D99C
:108CF00012B9D1750800128DD270597E007F0080A4
:108D00004E128AD412CD5AE0540F6040128A97F561
:108D10000CA3E039F50DE50C2403FCE50D128D598B
:108D20003400FB121C9EE964017021850C82850DC4
:108D300083A312B862850A82850B83A3E8F0A3E9B6
:108D400012B07612BC7B75080112BEFF1292391266
:108D50008AEB40ADA908029D1C3400FDE50A2403FE
:108D6000FAE50B2274F5120356EAFEEBFF8E828FB2
:108D700083A312B9D97C007D00EE24030A0A0A12EB
:108D80008DCAEEFAEFFB120AFEE9F50A7401650AD4
:108D9000702E12A3EC12B862128A9BF508A3E03978
:108DA000F509850882F583A3128EB5128DE3FAE5E5
:108DB00009128DD5700AE5082403FCE509128DC35C
:108DC000029B073400FDEE2403FAEF3400FB120B84
:108DD0003422128CCB128DDB6401223400FB120B87
:108DE0003AE922A3E8F0A3E9F0E50824032274F2AB
:108DF00012035674E61208DBEAFEEBFF128EB0EFA8
:108E000012B9D5750801750A00750B00750C00754F
:108E10000D00E4851082851183F0EE2403FCEF340D
:108E200000FD7403120AAC12A2D86401702D740BF9
:108E3000120AAC12AD10128EB1EF12AAAB7401126D
:108E40000AAC128EB5A3E0687003A3E06960538595
:108E5000108285118385820A85830B740D120AACFA
:108E6000128EC312B862740E120AAC12AAAE740D3E
:108E7000120AACAA82AB83120B58E96401700B741E
:108E80000D120AAC85820C85830D780C12081BAC80
:108E90000AAD0BEEFAEFFB120B107402120849E94F
:108EA000F508EEFAEFFB120B52A908741A029D198D
:108EB000EE12C07122128EB922E0F8A3E0F98E8280
:108EC0008F8322E4128EC822F08E828F83A322C069
:108ED00082C083128EF1EC75F012A4FCAAF075F03A
:108EE00012EDA42AFD79FF7AA57B151214AC02A716
:108EF0009F90229BE493FC740193FD2274F712036C
:108F000056E9FEEAFF7C007D0078007900802DE8BC
:108F1000FAE9FBEA75F012A4FA85F00875F012EB95
:108F2000A4250812936AC39E400FE0FAEFC39A404B
:108F300008EC24010CED3400FD12986C90229B1279
:108F400097F340CBECFAEDFB029A84C082C08378A1
:108F5000007900800312986C90229B1297F3500CBA
:108F600012935464FF70EE1293F880047A007B0031
:108F700002A79F74F012035674F31208DB8A0E8B5B
:108F80000F8C088D09890AEC7001ED6015AA08ABF9
:108F900009120BA68A0C8B0DAE0CAF0DEE7001EF13
:108FA000704B120B7C8A0C8B0DA80CA90DE8FEE906
:108FB000FFE87001E960367401851082851183F045
:108FC000120AACE50EF0A3E50FF0AC08AD0974038E
:108FD000120AAC12910D740B120AAC12A6C312AA9B
:108FE000AE129089AA0EAB0F1210C28006EE70016D
:108FF000EF60727A00E50A6007C3940550027A04B4
:109000008E828F83E50EF0A3E50F129A0CE50AF02D
:10901000EA8E828F83A3A3A3A3A3F074028E828F10
:1090200083A3A3A3A3A3A3A3A3F074018E828F831E
:10903000A3A3A3A3A3A3A3A3A312C5B6A3F0EE2443
:1090400010129082E4F0A312A50EA3A3F012A3ECD9
:10905000E4F090877F7808120A6DEE240C1290825B
:109060007808120A5E1292A4400EE4901A30F07A48
:10907000307B1A7941121CBCEEFAEFFB02C92FEECD
:10908000240DF582EF12BC6B22E48E828F83A3A3A2
:10909000A3A3A3A3F090038012B86D2274F212036D
:1090A0005674F31208DBEAFEEBFF8C088D09750A93
:1090B00000AA08AB09120BA68A0C8B0DA80CA90DEF
:1090C000E87001E9604088828983E06E7003A3E064
:1090D0006F603388828983A3A3A3A3E0C394055060
:1090E000258882898312BC7B740185108285118357
:1090F000F0120AAC12BC7BAC08AD097403120AACC6
:1091000012910D750A01A90A740D029D1912A13C54
:10911000120B6A2274F612035612B4C97001E96088
:109120001488828983A3A3A3A3E06009C394055094
:1091300004790180027900029EAF74F61203561280
:10914000B4C97001E9601488828983A3A3A3A3E052
:109150006009C394035004790180027900029EAF34
:1091600074F6120356120BA08A828B83E58270027A
:10917000E583600BA3A3A3A3E070047901800279C7
:1091800000029EAFC082C083EAFCEBFD7A007B0048
:10919000120BAC02A79FC082C0837C007D0080F0D0
:1091A00074F412035674F31208DB8A0A8B0B8C08D2
:1091B0008D097E007F00802112970B120AAC12925B
:1091C0003E60137403120AACAC82AD83AA0AAB0BE7
:1091D000121C9EE970381292391292305049129541
:1091E000A960F3E50A7002E50B70CD74FF650870A5
:1091F0000474FF650960DFEEF8EFF9E875F012A47A
:10920000F81296F465087004A3E0650970C8EE755D
:10921000F012A4FEAAF075F012EFA42AFFEE24A526
:10922000FAEF3415FB80047A007B00740D02A47AF7
:1092300090229B129DC2028AF2129595FF22E8F0BD
:10924000A3E912A156120B64E92274F412035674B6
:10925000F31208DB750800120BA68A0A8B0BAE0A04
:10926000AF0BEE7001EF602A7401851082851183C7
:1092700012A6F5F8A3E0F9740B120AAC12A14E1273
:109280000B4C7C127D0079FFEEFAEFFB1214AC75EB
:1092900008011292A450097401901A30F0120FA222
:1092A000A90880877A047900120B7690229B129D80
:1092B000C2EA98EB992274F7120356E9FE74FE6A2B
:1092C000700374FF6B780079007005805912986CF8
:1092D00090229B12985F504EE8FCE9FDEC75F0126D
:1092E000A4FCAFF075F012EDA42F12C941ED129558
:1092F000C160DAE8FCE9FDEC75F012A4FC75F0122F
:10930000EDA42FFDEC24A5F582ED3415F583E06A7C
:109310007003A3E06B70B6800A1293546005C39487
:1093200005401A12986C90229B1297F3501FEE7012
:10933000E812935464016005E0640370E6E875F098
:1093400012A4F8AAF01296FB12B9BE80047AFE7B32
:10935000FF029A84E8FAE9FBEA75F012A4FAACF08D
:1093600075F012EBA42C12936A22FBEA24A9F58271
:10937000EB3415F583E022120BB802A79FC082C020
:1093800083790180F274F01203568A0E8B0F7A04EF
:109390007901120B768A08AE08EE7001EB6044EAA0
:1093A000C333FAEB33FB1215368A0A8B0B8A088B10
:1093B00009EA7001EB60287AFE7BFF120BBE74FE97
:1093C0006A700374FF6B6021850A82850B8312AD7E
:1093D00061E50A2402F50AE50B3400F50B80DC7E1A
:1093E000008006750800750900EE850E82850F83E2
:1093F000F0AA08AB0902C934E875F012A4F8AAF083
:1094000075F012E9A42AF9E824A5FAE93415FB223B
:1094100074F6120356750800750900780812081BC7
:1094200090229B129EC0740378081209DA12959D4F
:109430007B0012159C7402120849E9FE6003120BAE
:10944000D0029E8C74F612035674FE1208DB129E34
:10945000ED029E9074F612035674DF1208DB7E0054
:109460008510828511838582088583097808120812
:109470001B7508028E09780812081B7C007D0012FB
:109480009FD5120849E960030295128079740F1282
:109490000AAC858208858309780812081B750808BC
:1094A000750900780812081B8E08740378081209E1
:1094B000DA74022508FCE43509FD129FD51208492B
:1094C000E970427402120AAC7401F07411120AAC11
:1094D00012B862740D120AAC12AAAE7402120AAC6F
:1094E000AA82AB83120B64E9601B7413120AACE00E
:1094F000F97405120AACAC82AD83740F120AAC1277
:10950000B9C0120B820E8E08129FC7E49950030255
:10951000948DEEF97421029EAC74F612035674FE1B
:109520001208DB851082851183E4F0A3F0FE804EE3
:109530001295A96046EEF8EFF9E875F012A4F875F7
:10954000F012E9A42AF9E824A5F508E93415F5098B
:10955000780812081B750808750900780812081B9E
:109560007404120AAC129D29740378081209DA12E5
:10957000959D12A0C612084912A0B3129595FF122C
:10958000923040AC851082851183858208858309DD
:109590007808029E90EE24010EEF3400227402251A
:1095A00008FCE43509FD7A2222EEF8EFF9E875F0BF
:1095B00012A4F8AAF075F012E9A42AF9E812C94336
:1095C000E912937164FF2274F71203567A007B004C
:1095D000800919EA24010AEB3400FB128EF1C3EA78
:1095E0009CEB9D503AEAFCEBFDEC75F012A4FCAE4E
:1095F000F075F012EDA42E12C941ED129371C394CF
:109600000550D0E970CCEA75F012A4FAACF075F010
:1096100012EBA42CFBEA24A5FAEB3415FB80047AA8
:10962000007B00029A8474F712035674F31208DB6D
:109630007E007F000296C3E50812BC4B12B9BEEE55
:10964000F8EFF9E875F012A4F8ACF075F012E9A49F
:109650002CF9E812C6F16A7003A3E06B6044E508D8
:1096600075F017A4F8AAF0EAF9E8241FF582E934A6
:1096700017F58312A253120AACE0687003A3E069E5
:109680006020E50875F017A4F8EAF9E82421FCE960
:109690003417FD7403120AACAA82AB83121C9EE934
:1096A0006011E50875F017A4241FFAE5F03417FBE4
:1096B0001210CE05089022A612BE3450030296372F
:1096C0001292391292305029EEF8EFF9E875F01243
:1096D000A4F8AAF01296F464FF7004A3E064FF609B
:1096E000DF12970B120AAC12923E60D4750800800C
:1096F000C4029A7F1296FBF583E02275F012E9A46A
:109700002AF9E824A5F582E934152274018510822E
:10971000851183F0EEF8EFF9E875F012A4F875F012
:1097200012E9A42AF9E824A7F582E9341512AAC39C
:10973000740B2274F6120356129EB4FC740193FD4E
:10974000EC8508F0A4CCAAF08509F0A42AFA8508D3
:10975000F0EDA42AFD79FF7AEC7B191214AC90038A
:10976000357400F0A3740CF090033774FAF0A3740E
:109770000BF09003397424F0A3740CF090033B7445
:1097800036F0A3740CF090033D743CF0A3740CF01D
:1097900090033F7442F0A3740CF09003417448F0BE
:1097A000A3740CF0E4900334F0029EAFC082C08337
:1097B00078007900800312986C1297F0501CE8FA38
:1097C000E9FBEA75F00EA4FAACF075F00EEBA42CF0
:1097D0001297E170E1129C5D80047A007B0002A781
:1097E0009FFBEA24ECF582EB3419F583E064FF2259
:1097F00090229DE493FA740193FBC3E89AE99B22BB
:1098000074F71203567A007B00780079008045E8EF
:10981000FCE9FDEC75F00EA4FCAEF075F00EEDA4C5
:109820002EFDEC24ECF582ED1297E86024E8FCE9CB
:10983000FDEC75F00EA4FC75F00EEDA42EFDEC24ED
:10984000F1F582ED3419F583E0FCEA2CFAEB3400F3
:10985000FB12986C90229D12985F40B3029A84E4A8
:1098600093FC740193FDC3E89CE99D22E824010860
:10987000E93400F92274F112035674FC1208DB7407
:1098800002120AAC12AD61890E8C088D0B7E007F2E
:1098900000120C607402120AAC12B9C0120C6612EB
:1098A000AD5B7402120AAC12B50A7007750A018E1C
:1098B0000980058E0A850809851082851183E06478
:1098C000FE7004A3E064FF70030299E28E08800238
:1098D000050885080C90229D12C9794003029975EC
:1098E000A808E875F00EA4A9F0129D54650E70E06A
:1098F000E875F00EA4129D21650A70D412B85CE5DB
:109900000875F00EA424EEF582E5F03419F583E035
:10991000687003A3E06970B8A808E875F00EA4A900
:10992000F024F0F582E93419F583E0650970A1E8C7
:1099300075F00EA424ECFEE93419FF750800E50863
:10994000C3950B40030299E2E508C333F8E433F909
:109950007413120AAC1299FB120C0CE97013E5088F
:10996000C333F8E433F97413120AAC1299FB120CE6
:1099700018050880C9120BF48A0C8B0DAE0CAF0DC4
:10998000EE7001EF605C8E828F83E50EF0A3E50A36
:1099900012A6DE8E828F83A3A3E8F0A3E9129A0CAD
:1099A000E509F09022AAE493C3950B5004E493F5E3
:1099B0000B8E828F83A3A3A3A3A3E50BF0741312D2
:1099C0000AAC129D29750A007808120817E50BC326
:1099D00033FCE433FDEE2406FAEF34001299F4125E
:1099E0000849EEFAEFFB7404800274121208497FF2
:1099F000070205ADFB1214A074032212CD5E129A69
:109A00000222E0FCA3E0FDEEFAEFFB22128EC8A3D7
:109A1000A3A322C082C08390229F128EF479FF12EA
:109A200014AC790102A79F74F7120356EA7001EB98
:109A300060498A828B83A3A3A3A3A3A3E5827002B8
:109A4000E58360377E0080010E8A828B83A3A3A307
:109A5000A3A3E0FFEEC39F5022EEC333F8E433F933
:109A6000EA28F582EB39F583A3A3A3A3A3A3E06CB3
:109A70007003A3E06D70D1790180027900800574D4
:109A80000D1208497F010205AD74F5120356EA7004
:109A900001EB605F8A828B83A3A3A3A3A3E060632F
:109AA000EA2406F8EB3400F98A828B83A3A3A3A3EC
:109AB000A3E0F509750800800DEA2405F582EB1294
:109AC000B9B3603F0508E508C395095026E50812BB
:109AD0009B4FE06C7003A3E06D60DE129B5512BFDC
:109AE000028882898312BC7BE824020808E93400DA
:109AF000F980D18A828B83A3A3A3A3A3E060047916
:109B000001800279008002A90A7F030205AD74F783
:109B1000120356EA7001EB60318A828B83A3A3A300
:109B2000A3A3E0C0E09022AAE493FED0E0C39E503D
:109B300019EA2405F8EB12CEC4129B4F12C9A9886A
:109B4000828983E004F0790180027900029A84C35B
:109B500033FEE433FF12CD7202C99274F41203563D
:109B60008908EAFEEBFF8C098E828F83A3A3A3A34F
:109B7000A3A3A3A3E0640170098E828F8312B86946
:109B80008003129D5F74FE6C700374FF6D70077A22
:109B9000007B00029C1D780079008014129C2064D8
:109BA00001700A129C3E7003A3E06D606D12986C08
:109BB0001297F050DAE8FAE9FBEA75F00EA4FA859C
:109BC000F00A75F00EEBA4250AFBEA24ECF582EB13
:109BD0003419F583E0650870D48E828F83A3A3A324
:109BE000A3A3A3A3A3E0640160B2129C2070BE12E1
:109BF0009C3E7003A3E06D70B4E8FAE9FBEA75F0EF
:109C00000EA4FA75F00EEBA4250AFBEA24F0F58207
:109C1000EB3419F583E065097093129C5D02A47D15
:109C2000E8FAE9FBEA75F00EA4FA75F00EEBA4254C
:109C30000AFBEA24EDF582EB3419F583E022E8FA19
:109C4000E9FBEA75F00EA4FA75F00EEBA4250AFB09
:109C5000EA24EEF582EB3419F583E06C22129C6164
:109C600022E875F00EA4F8AAF075F00EE9A42AF91E
:109C7000E824ECFAE93419FB2274F21203568A0A3A
:109C80008B0B8A828B83A3A3A3A3A3A3A3A3E064C8
:109C90000170098A828B83129D298007120C4E8ADB
:109CA000088B0974FE6508700474FF650960687E9E
:109CB000007F00805A850A82850B83A3A3A3A3A3F8
:109CC000A3A3A3E064017041EEF8EFF9E875F00E8C
:109CD000A4F8AAF075F00EE9A42AF9E8129D21640F
:109CE000017029EEF8EFF9E875F00EA4F875F00EA2
:109CF000E9A42AF9E824EEF582E93419F583E06550
:109D0000087004A3E065097003129D311292399026
:109D1000229D129233409E80031208497F0602055D
:109D2000AD24EDF582E9029C38E0F508A3E0F509E1
:109D300022EEF8EFF9129C61120C0622EEF8EFF910
:109D4000E875F00EA4F8AAF075F00EE9A42AF9E877
:109D5000129D542224ECF582E93419F583E0221295
:109D60000C4E8A0A8B0BAC0AAD0B2274F31203560D
:109D7000890CEAFEEBFF750A00750B00750800758B
:109D800009008029E50875F00EA4F8AAF075F00E18
:109D9000E509129D4C650C7011EEFCEFFDAA82AB3B
:109DA00083120C0CE96003129E47129DCB90229DFA
:109DB000129DC2E50898E5099940C9AA0AAB0B02B1
:109DC000A651E493F8740193F9C322E5082401F540
:109DD00008E5093400F5092274F1120356890EEAE8
:109DE000FEEBFF8C09750800750A00750B008005F5
:109DF0000508129E4790229D12C703E50B9950401B
:109E0000E50A75F00EA4F8AAF075F00EE50BA42A89
:109E1000F9E824ECF50CE93419F50D850C82F5838D
:109E2000E0650E70CDEEFCEFFDAA0CAB0D120C0C34
:109E3000E960BFE508C3950940B6AA0CAB0D8004E4
:109E40007A007B000299EFE50A2401F50AE50B345C
:109E500000F50B2274F61203567508007509007898
:109E60000812081B129EB412A09875832275829F57
:109E7000E49328FCA3E49339FD7A417B0012159CFE
:109E80007402120849E9FE6003120C3CEEF9801FCF
:109E900012081B750802750900780812081B7C005F
:109EA0007D007A2212A0C612084974021208497F66
:109EB000020205AD90229F129EC090229DE4932243
:109EC000E493F508740193F5092274F612035674AD
:109ED000FE1208DB129EED12081B750802750900C0
:109EE000780812081B7C007D007A4180B7851082BB
:109EF000851183E4F0A312A0E485820885830978A4
:109F0000082274F412035674E71208DB7E007F0007
:109F10008510828511838582088583097808120857
:109F20001B7508028E09780812081B7C007D007AD8
:109F300041129FD7120849E96003029FBE8E088034
:109F4000757402120AAC85820A85830B780A12089E
:109F50001B90229F1206CA12A086129FD712084990
:109F6000E970507410120AACAC82AD837404120A0A
:109F7000AC12B9C0120C54E960397408120AAC85ED
:109F8000820A85830B780A12081B7409120AACE056
:109F9000FD7408120AACE0FC7412120AACAA82AB7F
:109FA000837404120AACE0F9120C0074021208491E
:109FB000129239129DCB129FC7E509994083EEFAA0
:109FC000EFFB741902A47A85108285118312AAC549
:109FD000C3E50898227A227B001215A87404227423
:109FE000F512035674F01208DB851082851183E4A4
:109FF000F0A3F0FE8057129D3C64FF604D858208FF
:10A00000858309750A00780812081790229F128E1E
:10A01000F47405120AACAA82AB831299F5120849AE
:10A020007402120AAC858208858309780812081B1D
:10A0300090229F1206CA7404120AAC129D2912A023
:10A040008612A0C612084912A0B3129595FF90225D
:10A050009D12923340A085108285118385820885E8
:10A060008309780812081B75080275090078081220
:10A07000081B7C007D007A4112A0C61208497410AA
:10A08000120849029B0990229FE49312A09874023F
:10A0900028FCE439FD7A4122F8740193F9E8850837
:10A0A000F0A4C8AAF08509F0A42AFA8508F0E9A46A
:10A0B0002AF922851082851183E02401F0A3E0347F
:10A0C00000F02212A0CE7B001215A2740422EA75C1
:10A0D000F00BA4FAACF075F00BEBA42CFBEAFCEB54
:10A0E000FD7A232212A0E822F085108285118322B6
:10A0F000A3A3E508F0A3E509F022EAF0A3EB12A17F
:10A100005622C082C08374F31208DB12A2DD7012E3
:10A110008A828B8312A253120AAC12A14E120B58E0
:10A12000800CEAFCEBFD7403120AAC12A13102A709
:10A130009412A1352212A13C120B5E22AA82AB839B
:10A14000120B34851082851183AA82AB8322E8F03A
:10A15000A3E912A1562212A15A2212A0E880EA74A1
:10A16000F712035674F31208DBECFEEDFF7404855E
:10A170001082851183F0740B120AACEAF0A3EB1283
:10A180009242F508601D74038E828F83A3A3A3A35C
:10A19000A3A3A3A3F0120AACAC82AD83EEFAEFFB4B
:10A1A000121CA4A908029A7FC082C08374F312080B
:10A1B000DB7404851082851183F0740B120AAC12D3
:10A1C000A0FA120B64740102A79612B9C7740D228B
:10A1D00074F612035674F31208DB900334E0706EC9
:10A1E0007404851082851183F090037312A25312B8
:10A1F0000AAC12AAAE120F66EAFCEBFD7403120A57
:10A20000AC12910D120F728A088B09A808A9097463
:10A2100001120AACE0687003A3E069602B74FE6869
:10A22000700374FF6960217401120AAC12AAAE7443
:10A2300003120AACAA82AB83120F788510828511B3
:10A2400083AA82AB83120B6A7401900334F0740DFD
:10A25000029EAC12AAC5740122C082C08374F3129C
:10A2600008DB12A2DD8A828B83701E12A253120AAF
:10A27000ACE8F0A3E912BAA9705B8510828511835E
:10A28000AA82AB83120B6A804CA3A3A3A3A3A3A3AC
:10A29000A3E064037010EAFCEBFD7403120AAC1235
:10A2A000A2D8703180D48A828B83A3A3A3A3A3A353
:10A2B000A3A3E0640170128A828B8312B862740BCC
:10A2C000120AACE8F0A3E9800B740B120AAC74FE1E
:10A2D000F0A374FFF002A79412A135E9227404855B
:10A2E000108285118312C590A3A3A3E06402227497
:10A2F000F5120356EAFCEBFD7A007B008A088A0916
:10A3000078007900800312986C90229DE493FE748B
:10A310000193FFC3E89EE99F5038E8FEE9FFEE7520
:10A32000F00EA4FE85F00A75F00EEFA4250AFFEEEC
:10A3300024ECF582EF1297E860CCAE08AF09740107
:10A340002EF508E43FF509EC6E7002ED6F70B71260
:10A350009C5D029B09C082C0839003487488F0A36F
:10A36000740EF090034A7482F0A3740EF090034EC2
:10A3700074CCF0A3740CF002A79F74F7120356EA92
:10A38000FEEBFF900382E064086019E0640460144F
:10A390008E828F83E06401704412A3EC12B4DDE07E
:10A3A000640670398E828F83A3A3E064FE7004A3D9
:10A3B000E064FF60288E828F83A3A312C98270039A
:10A3C000A3E069700BEE2415F582EF12BEF9600868
:10A3D000120F2AE9F5088008120F3080F67508C2BE
:10A3E000EEFAEFFB12153CA908029A84EE240B1238
:10A3F000BC682274F41203568A088B098A828B8304
:10A40000E0F8A3E028FAE43400FB1215368A0A8B40
:10A410000BAE0AAF0BEE7001EF605985088285091B
:10A4200083E0FC7D0079001214AC8E828F83A3A39D
:10A4300012B9D9120F6C8E828F83A3A3A3A312BD6E
:10A4400028F8EE28F8EF3400F912A3ECE8F0A3E9BD
:10A4500012A482C0E012907FD0E0F0120F7EEE24B2
:10A460000E129082E912A6C9E0C0E0EE241112900B
:10A4700082D0E0F0EEFAEFFB80031208497F04027D
:10A4800005AD12A6CEE02274F412035674EB120846
:10A49000DBEAFEEBFF900344E07002A3E070687A11
:10A4A000077B0012153690034412AD61900344E01F
:10A4B0007002A3E0604D90034412B8698F838E82CE
:10A4C00074071207958E828F837808120A6D8510A3
:10A4D000828511837808120A5E8E828F83A3A3A3DC
:10A4E000A3E0C0E07405120AACD0E012A50EE0C0F3
:10A4F000E07404120AACD0E0F07407120AAC12A6A1
:10A50000568006791080027901741502A47A12A58A
:10A510001222F08E828F8302C992C082C083900380
:10A5200044E07002A3E0600D90034412BE3C90032F
:10A5300044E4F0A3F0120EA612106E02A79F74F36B
:10A5400012035674EB1208DBECFEEDFF7422120AC4
:10A55000AC7808120A6D7426120AACE0FC7427125B
:10A560000AACE0FD7428120AACE0F50C740F6C70B4
:10A5700005740F6D6012901A97E06402700579C13E
:10A5800002A64CECC39D40F69003837808120A5E45
:10A59000E9900389F0EC900387F0ED900388F0E5F3
:10A5A0000C90038AF074FF6A700374FF6B701F9045
:10A5B0001AA4E064FF7004A3E064FF70051214BEE7
:10A5C000800C901AA412A6D7E8F0A3E980079003A4
:10A5D00080EAF0A3EBF0EE7001EF6017EEFAEFFB0C
:10A5E00012112EE96401700BEEFCEFFD7A947B03EF
:10A5F000121CA4900373E4F0A3F0900376F0A3F090
:10A60000900393F0901A97E06402700A740F90031D
:10A6100087F0900388F07405900382F07404120AA6
:10A62000ACE4F09003837808120A6D8510828511DE
:10A63000837808120A5E900389E0C0E07405120A6C
:10A64000ACD0E0F07407120AAC12A65674151208CA
:10A65000497F050205ADE412A65B2212A15A121C25
:10A66000CE22C082C083900343E070031217CA1247
:10A670000C9C02A79FC082C083900343E07007E454
:10A68000901A2FF080317401901A2FF0900343E05C
:10A6900064FF60237C41E0C394415002E0FCECFA8B
:10A6A000E0C39AF0EC75F0E8A4CCAAF075F003A42E
:10A6B0002AFD7A8012C99E7A2F7B1A7941121CBC1E
:10A6C00002A79F128EB9A3A32212A6CEA322F085C1
:10A6D0000882850983A32212AAC59003802212C989
:10A6E000B4F8A3E0F922C082C083EB90038AF01291
:10A6F0000E9402A79F128EC8A3E02274F71203568D
:10A7000074F81208DBEAFEEBFF7900900382E06444
:10A7100008704085108285118374FD12B9DB120F19
:10A72000667402120AAC12AD617405120AAC128E84
:10A73000C3E0C0E07404120AACD0E012A758C0E035
:10A740007406120AACD0E0F07407120AAC12AAB474
:10A75000120FC07408029A81F0028C1FC082C0835D
:10A760009003547450F0A3740DF09003EE7414F041
:10A77000A37410F09003587480F0A3740DF090034C
:10A780005A7450F0A3740DF090035C7486F0A374B7
:10A790000DF0800B740B120AAC12A1CA120849D03A
:10A7A00083D08202053374F412035674F91208DB65
:10A7B0008A088B098C0A8D0B851082851183780895
:10A7C000120A5E7404120AACE9F07405120AACE4D1
:10A7D000F07406120AAC12AAB4120C84740702A414
:10A7E0007A74F41203568A088B098A828B8312BF0B
:10A7F00002EE7001EF700302A8FF900310E07002F8
:10A80000A3E060158A828B83A3A3E0F9EEFAEFFB45
:10A8100090031012B4DD121E778E828F83A3A3A340
:10A82000A3A3A3A3A3A3E06402707F8E828F83A35C
:10A83000A3A3A3A3A3E05402700302A8CE850882B9
:10A84000850983A3A3E064E9700302A8CE8E828FFA
:10A8500083A3A3A3A3A3A3A3A3A3A3E07014901A09
:10A8600099E0048E828F83A3A3A3A3A3A3A3A3A38E
:10A87000A3F08E828F83A3A3A3A3A3A3A3A3A3A3C5
:10A88000E014F074048E828F83A3A3A3A3A3A3A3D5
:10A89000A3A3F0901A9A12A6C3A3A3E8F0A3E91207
:10A8A000CB957001EB700312C5988E828F83A3A3A2
:10A8B000A3A3A3A3A3A3A3E0640260128E828F8349
:10A8C000A3A3A3A3A3A3A3A3A3E0640670318E82D2
:10A8D0008F83A3A3A3A3A3A3E0A2E05022850882B1
:10A8E000850983A3A3E0F9EEFAEFFB121D648E82C3
:10A8F0008F83A3A3A3A3A3A3E054FEF0A3E0F002DD
:10A90000A47D74F012035674DD1208DB8A0C8B0DE3
:10A910008C0E8D0F7433120AAC7808120A6D7F000A
:10A92000740E120AACAC82AD83120AC2740E120A03
:10A93000ACE0A2E5500D0F12B9B9121D70E9600329
:10A9400002AA57740E120AACE0A2E6500E740F125F
:10A950000AACE0540370047E0180027E00740E1283
:10A960000AACE05403FA74026A700912B9B9120A07
:10A97000D402AA5774016A7043EE600312AA8A7463
:10A980000E120AACA882A9837403120AACE8F0A3E1
:10A99000E912AAB985108285118312AAAE850C82AC
:10A9A000850D83A3A3A3A3A3A3E0C0E07402120AAE
:10A9B000ACD0E012AAB5121E4E02AA57EA600302FA
:10A9C000AA57740D120AAC740212AAB97405120ABD
:10A9D000AC12AAAEEE6008740E120AAC12AA8A7407
:10A9E0000E120AACE0540C64047071E50C240FF5EF
:10A9F00082E50D12BEF9C0E07420120AACD0E0F07E
:10AA0000900312E07002A3E0604D120F6C8A0C8B71
:10AA10000DA80CA90D7405120AACE0687003A3E040
:10AA20006970347808120813EFF508780812081FC7
:10AA3000780E12081BEEF97415120AACAC82AD83C5
:10AA4000740C120AACAA82AB8390031212B4DD120A
:10AA50001E777407120849742302C9317808120856
:10AA600013780E12081B90038012069DEFF9740DE7
:10AA7000120AACAC82AD837416120AACAA82AB8304
:10AA8000121D58740812084980CD12AA9712BC6B87
:10AA900012B9C7120AC822AC82AD83E50C240BF5AB
:10AAA00082E50D2212AAC112C070EB12BC6BE8F055
:10AAB000A3E9F022E412A15622F012AA9B12AAC125
:10AAC000223400F583E002A6E1C082C0831216C8DA
:10AAD00002A79FC082C0831216CE02A79FC082C069
:10AAE000831216D402A79FC082C0831216DA02A76F
:10AAF0009F74F71203567409120AACE0F50878083F
:10AB000012081F1216E67401029A81C082C08312D5
:10AB100016F202A79FC082C0831216F802A79FC038
:10AB200082C0831216FE02A79F74F7120356EAFE34
:10AB3000EBFF74016970107900120DC27C1E790060
:10AB4000EEFAEFFB120D44029A8474F41203567469
:10AB5000F91208DB8A088B098C0A8D0B7413120A10
:10AB6000AC12B9C0901228E07002A3E06027E9851A
:10AB70001082851183F07401120AAC7808120A5E03
:10AB8000EAF8EBF97405120AAC12A14E90122812E1
:10AB9000B4DD121E7702A7DCC082C08312172E021A
:10ABA000A79F74F7120356901A32E0F97F00800BCA
:10ABB00012ADEB540D64017001190F12ADE3500397
:10ABC000E970ED029A8474F7120356901A33E0F993
:10ABD0007F00800B12ADEB548D64817001190F1250
:10ABE000ADE35003E970ED029A8474F212035689C2
:10ABF0000AE975F006A4F8A9F0740C28FEE439FF00
:10AC0000EA2EFAE43FFB1215368A088B09EA700136
:10AC1000EB6029EEFCEFFD79001214AC12C065E583
:10AC20000AF0E5082EF8E5093FF9850882850983D1
:10AC3000A3A3A3A3A3A3A3A3A312AAAEAA08AB0989
:10AC4000029D1C74F61203568A088B09120D20907F
:10AC50001A31E0FAE9C39A400990035012B9C012C0
:10AC60000D26E5082402FEE5093400FF9003521288
:10AC7000C076F0900352E004F0AA08AB09120D2C44
:10AC80008E828F83E0029E8DC082C0837900900304
:10AC90005080010912B9C08A828B83E5827002E577
:10ACA0008370F002A79F74F7120356EAFEEBFFEEE3
:10ACB0007001EF6058900350E07002A3E0604E9086
:10ACC000035012B4F57A007B00800FAA82AB831286
:10ACD000B4F5E5827002E5836033EE65827003EFC0
:10ACE000658370E790035012AD10687002EF698EB3
:10ACF000828F83700812B862900350800312CB8950
:10AD000012AD15121E1EEEFAEFFB12153C029A84CC
:10AD100012AAC5EE22E8F0A3E9F0029A07C082C0A9
:10AD20008390035080048882898312B862E870019E
:10AD3000E9600B88828983E07002A3E070E88A8270
:10AD40008B83E4F0A3F0E87001E9600688828983D0
:10AD5000800390035012AD6102A79F851082851178
:10AD600083EAF0A3EBF02274F7120356E9FC900398
:10AD70005080048A828B8312ADDE7001EB60177EF7
:10AD80000080010E12ADCEFDEEC39D50E6EE12AE78
:10AD9000046C70EF80047A007B00029A8474F712CE
:10ADA0000356E9FD7F0080010F12ADCEFEEFC39E7A
:10ADB0005019EF12AE046D70EFEF75F006A4F8A90C
:10ADC000F012C0AF741112AE134CF0029A8412AD9F
:10ADD000D222EA240BF582EB3400F583E02212B98B
:10ADE000C7EA2212ADD2FCEFC39C22EF75F006A495
:10ADF000FCADF0EA2CFCEB3DFD74112CF582E43D3A
:10AE0000F583E02275F006A4F8A9F0EA28F8EB39FA
:10AE1000F9741028F582E439F583E02274F6120300
:10AE200056120E3A7A008011EA12BD7412B9E51278
:10AE3000AE9AF0A312C37FF00A9022AE12C96F40FF
:10AE4000E77A00801B8A08750900740378081209E4
:10AE5000DA12C34E12B9E1A3A3A3A3A3A3A3F00ADA
:10AE60009022AB12C96F40DD7A00801A8A087509FA
:10AE700000740378081209DAE5082477F582E509F9
:10AE8000341912B9D70A12C96C40E19022A5E49393
:10AE900090035EF012C998029EAFA312AE9F2212D9
:10AEA000C37F02C99374F112035674F51208DBEAEA
:10AEB000FEEBFF89088C09E9A2E050127EFC7FFFBF
:10AEC000A2E15005D2E402AF6FD2E302AF6F120EDF
:10AED0001C8A0A8B0BA80AA90B900373E068700305
:10AEE000A3E0697005790002B051AC087902EEFA6E
:10AEF000EFFB120E16E960EDE508F50A780A120874
:10AF00001F12B056120849E9600302B04FE508C2AB
:10AF1000E5F5089003C0E07058E508A2E6405274D9
:10AF200003120AACAC82AD83EEFAEFFB120B40E9E0
:10AF3000703912B866EEFAEFFB1210B08A0A8B0B6A
:10AF4000A80AA90BE87001E96027E824020A0AE9C7
:10AF5000128DDB601CE50A2402FCE50B3400FD7455
:10AF600003120AACAA82AB83121CA4E508D2E5F551
:10AF700008900353E0F50E90037312B873780A1229
:10AF8000081B7D017C00900353E0F9AA0AAB0B1269
:10AF90000DCE7402120849E9FA900353E004F0EA76
:10AFA000600302B04FE508A2E550047A0E80027AF1
:10AFB000067401120AAC12C08B8A0A8B0BEA70016C
:10AFC000EB700302B04B12B066E50A241AF582E575
:10AFD0000B129085EAF0A3EB12B07612A25388828E
:10AFE0008983F07478550812B144E50EF0EE88823A
:10AFF0008983A3A3A312C365F0E488828983A3A3F2
:10B00000A3A3A3F0E508A2E550147403120AACACA4
:10B0100082AD83E82406FAE93400FB121CA4850AF9
:10B0200082850B83A3A374FD12B9DBE5096013C30A
:10B03000941E500EE50A2413F582E50B129085E567
:10B0400009F0AA0AAB0B120C7880067910800279FD
:10B05000C7740B0299EC79027CFE7DFFEEFAEFFBE0
:10B06000120D8C740122EA2417F582EB12BC6B746A
:10B0700001F0120F6622F0E50A12C071E50B12BC56
:10B080006B2274F41203568A088B09E9FE120FF63C
:10B09000E960077AFF7BFF02B137901A97E06402FC
:10B0A000600302B12A7900AA08AB0912C21D8A0AFC
:10B0B0008B0BA80AA90BE87001E960588882898384
:10B0C000A3A3A3A3A3E06401701C12B13A12B1417F
:10B0D000E064FE7004A3E064FF602B88828983A390
:10B0E000A312B9C0805188828983A3A3A3A3A3E03C
:10B0F0006403602888828983A3A3A3A3A3E06404D4
:10B1000070047AFE808F88828983A3A3A3A3A3E01F
:10B11000640270089003BFE06402700E12C70A70E8
:10B1200001EB6006AA08AB09800DAA08AB099003E1
:10B130005412B4DD121E7702A47D900372E002B4B3
:10B14000FBA3A3A3A312C37AA32274F7120356EAA4
:10B15000FEEBFF120B8EE9700AEEFAEFFB120B9A70
:10B16000E96006EEFAEFFB80047AFE7BFF029A8428
:10B1700074F01203568A0A8B0B8C0E8D0FE9FE7544
:10B180000800120FF6E97900600302B255AA0AAB73
:10B190000B12C1F0A80CA90DE87001E960198882B2
:10B1A0008983A3A3A3A3A3E06402704F9003BFE02D
:10B1B0006402700302B253AA0AAB0B90035A12B492
:10B1C000DD121E77120BA08A0C8B0DA80CA90DE8BE
:10B1D0007001E9607E88828983A3A3A3A3A3E0A270
:10B1E000E050707F01A2E150247901AC0AAD0BAAB6
:10B1F0000EAB0F120D6EE97020805888828983A3F0
:10B20000A3A3A3A3E06403704A7F02800C88828911
:10B2100083A3A3A3A3A3D2E1F0900373E0650E7010
:10B2200004A3E0650F70107C1EEEF9AA0AAB0B12A6
:10B230000D44750801801CEFF9AC0AAD0BAA0EABEA
:10B240000F120D6EE9700C750801EEF9AA0AAB0B2E
:10B25000120DC2A90802C93474F112035674EE1219
:10B2600008DB12AD5B8C088D099003F4E07002A33B
:10B27000E0601212CD407002E5836004A3E0700527
:10B28000790002B4C6851082851183E0241DF50C77
:10B29000A3E03400F50D850C82F58312B4F5A3E02C
:10B2A000F50A12B679FA88828983A3A3A3A3E0F9E9
:10B2B000EAFEE9FFAA08AB09120DC8E9FA850C827B
:10B2C000850D8312C98BE02AF50B530A7878081292
:10B2D000081B7D00AC0BA90E7402120AAC12B52734
:10B2E000120849E9FA74036A6096EA7044741855C2
:10B2F0000A700302B3EDE50AD2E0F50AA2E45004B5
:10B30000D2E1F50AE50AF50C780C12081F7901ACB8
:10B3100008AD09E9120AAC12B520120849E970110A
:10B320007421120AAC12B4EE12C9AF12B500121693
:10B33000EC7421120AAC12B4DDE064FF7004A3E0E7
:10B3400064FF603B9003BFE06402700302B280853B
:10B350001082851183E012B50012B4DA121E77EA6A
:10B3600065087003EB6509600302B28012B4D6125F
:10B370001E777421120AAC12B4DDEAF0A3EBF07868
:10B380000812081B7D01AC0BA90E7402120AAC1244
:10B39000B527120849A90AEEFAEFFB120E1C8A081B
:10B3A0008B09A808A909900373E0687003A3E069FA
:10B3B000600302B4B9EEFAEFFB12B4C97001E960A0
:10B3C0006C88828983A3A3A3A3E06401600D8882B3
:10B3D0008983A3A3A3A3E0640270527402120AAC8F
:10B3E000AC82AD83EEFAEFFB120B40805390036CFE
:10B3F000E06019E50AF50C780C12081F7901AC0819
:10B40000AD09E9120AAC12B520120849E50AF50C9B
:10B41000780C12081F12B056120849E9600302B3F3
:10B42000317421120AAC12B4EEA302B37E120F667D
:10B43000EAFCEBFD7402120AACAA82AB83121CA4D4
:10B4400085108285118312B50A701C8510828511C2
:10B4500083E0241512B68BFCA3E0FD740A120AAC3B
:10B46000AA82AB83121CA412B514E04430F508780C
:10B470000812081F7403120AAC85820885830978B4
:10B480000812081B740D120AAC858208858309789E
:10B490000812081BE50EF508780812081F7900EE5F
:10B4A000FCEFFD7406120AAC12B6AB12B9C0120D55
:10B4B00068740612084902B28012B514A3A3A3A3AC
:10B4C000E50BF0120F7E0299EA120BA08A088B0995
:10B4D000A808A909E822EEFAEFFB90035612B4E19E
:10B4E0002212B4E522E0F8A3E0F58388822212B4A8
:10B4F000E174FFF02212AAC58001F98882898322B3
:10B50000240B12B69CFAA3E0FB2212C98FA3A3A3BB
:10B51000E064012212B693F8A3E0F5838882A322A7
:10B5200012B9C412B0602212B9C4120DCE74022234
:10B5300074F112035674EE1208DB851082851183B4
:10B54000EAF0A3EB12C9B0241D12B68BF8A3E0F900
:10B5500012B679FC88828983A3A3A3A3E0FBECF550
:10B5600008EBF50988828983A3A3A3A3A3E0FC8841
:10B57000828983A3A3A3A3A3A3E0FAE4CAFBECFEFE
:10B58000EBFF88828983A3A3A3A3A3A3A3E0F50A67
:10B5900088828983A3E05478F50BA2E4501912B68F
:10B5A0008F2408FCA3E03400FD740A120AACAA82BE
:10B5B000AB83121CA47A08E50BA2E5501D12B68FCE
:10B5C0002AF8A3E03400F9740828FCE439FD740279
:10B5D000120AACAA82AB83121CA4AC0AA90EAA0858
:10B5E000AB09120DD4E9FA74036A700302B67690BF
:10B5F0000373E065087004A3E065096064EA705AAB
:10B60000E50BF50C780C12081F7901E9120AAC124F
:10B61000B6A1120849E9705E780B12081F74031274
:10B620000AAC85820C85830D780C12081B740D12F0
:10B630000AAC85820C85830D780C12081BE50EF58B
:10B640000B780B12081FA90AEEFCEFFDAA08AB0944
:10B65000120D687406120849801C74046A70178001
:10B66000B7E50BF508780812081F7901E9120AAC52
:10B6700012B6A11208490299EA88828983A3A3E03D
:10B68000F50E88828983A3A3A3E02212B69C22121E
:10B69000B69322851082851183E0241D12C939E0FA
:10B6A0002212B6AB129A0212B0602212B6AF22E09A
:10B6B000240BFAA3E03400FB8A828B832274F012FD
:10B6C000035674F21208DB7402120AACE9F0EAFEC7
:10B6D000EBFF8C088D09741E120AACE0F50F742381
:10B6E000120AACE0F50EA90F120DDA12AD5B74046C
:10B6F000120AAC7408F0E50EA2E450037410F0E5F1
:10B700000EA2E55004E02408F07403120AACAA82E9
:10B71000AB83120FDE8A0C8B0DEA7001EB70030213
:10B72000B84812B066E50C241AF582E50D12908532
:10B7300012AD617406120AACAC82AD8385108285AD
:10B74000118312B9C0120B40E9600E12B84D740695
:10B75000120AACA882A9838020E50EA2E4502585B8
:10B760001082851183E06E7003A3E06F701612B82B
:10B770004D741F120AAC12B862E50C2418F582E56C
:10B780000D12AAABE50C128EB1E50D12908512B820
:10B79000737402850A82850B83F0A3E50E12B87BD1
:10B7A000E50FF0EE850A82850B83A3A3A3F0EF8556
:10B7B0000A82850B83A3A3A3A312B87BA3A3A3E54B
:10B7C00008F0E509850A82850B83A3A3A3A3A3122E
:10B7D000C9AFFAA3E0FB120DC87402120AACE9FA71
:10B7E000E02A850A82850B83A3A3A3A3A3A3A3F0C6
:10B7F000750800E50EA2E45018741F120AAC12B8C6
:10B8000069E50A2408FAE50B3400FB121CA475084C
:10B8100008E50EA2E5501C7421120AAC12B869E5C5
:10B820000A2508F8E50B3400F9740828FAE439FB16
:10B83000121CA412B85C850C82850D83A3A312AAE6
:10B84000AEAA0CAB0D120C78740E02C931E50C24B3
:10B8500016F582E50D12BC6B7401F022851082850D
:10B86000118312AAC52290038012B86D22E0FCA3B6
:10B87000E0FD22E0F50AA3E0F50B22F0850A8285BF
:10B880000B83A3A32274F2120356EAFEEBFF8C088B
:10B890008D09890A7900120E1C8A0C8B0DA80CA93F
:10B8A0000D900373E0687003A3E06979016019905B
:10B8B0000373E06E7003A3E06F600DA90AAC08ADDE
:10B8C00009EEFAEFFB12102C029D1C74F4120356C1
:10B8D0007ED77F1712C99890035EE014F0700C9029
:10B8E00022A5E49390035EF0120E28750800805E96
:10B8F0008E828F83A3A3A3A3E06049EE2404F58284
:10B90000EF12B9B3703E8E828F83A3A3A3A3A3E0EB
:10B910006403701079028E828F8312B9CBA312B99F
:10B92000C0120D6E8E828F83A3A3A3A3A3E0640134
:10B9300060128E828F8312B9D9E48E828F83A3A383
:10B94000A3A3A3F00508EE2407FEEF3400FF12BE08
:10B9500031409D750800803A85080A750B00740314
:10B96000780A1209DAE50A2437F8E50B3419F9E800
:10B970002407F582E912B9B3701685080A750B0021
:10B980007403780A1209DAE50A2437F812B9E1F0EB
:10B9900005089022AB12BE3440BE75080080091223
:10B9A000BE1F600214F005089022AE12BE3440EFB4
:10B9B00002A47D12ADD814F02212AA973400F583A8
:10B9C00012B9C72212B6AFE002B50512B86D028EE9
:10B9D000C912C070EB3400F58374FEF0A374FFF05D
:10B9E000228882898312B9E922A374FEF0A374FF2E
:10B9F000F0E402B4FB74F6120356E9702479009067
:10BA0000035812B4DD121E778A088B09AE08AF09FD
:10BA100074FE6E700374FF6F701A9022A8E4936036
:10BA200013790190035812B4DD121E778A088B092E
:10BA3000AE08AF09120FA2EEFAEFFB029EAFE028AC
:10BA4000F8A3E039F92274F612035674F31208DBF6
:10BA50001214BE8A088B09AE08AF09900373E06E1A
:10BA60007003A3E06F60E9120F72EA6E7002EB6F71
:10BA700060DEEEFAEFFB120FF6E970D4EE7001EF24
:10BA800060CEE4851082851183F07401120AACEE59
:10BA9000F0A3EF12BAA970B874FE6E700374FF6F52
:10BAA00060AEEEFAEFFB02A24E12A156120B58E95D
:10BAB00022C082C083120FA202A79F74F212035603
:10BAC000EAFEEBFF8C0C8D0D8908740E120AACE0B7
:10BAD000F50974FC6E700374FF6F70057900029DA8
:10BAE0001C7900120E1C8A0A8B0BAE0AAF0B900356
:10BAF00073E06E7003A3E06F7006E509A2E650DC08
:10BB0000A90912BC3E7001E9701279007AFE7BFF30
:10BB100012BC3E7001E97004790280C28882898378
:10BB200012BC7B74FE650C700474FF650D600D889B
:10BB3000828983A3A3E50CF0A3E50DF088828983B5
:10BB4000A3A3A3A3A3A3E509F0A2E0500D888289D3
:10BB500083A3A3A3A3A3A3D2E2F074016508702674
:10BB6000740188828983A3A3A3A3A3F012B13A121C
:10BB70009090AA0CAB0D1210DAEA7001EB60030290
:10BB8000BADC7E00801F88828983A3A3A3A3A3E0DD
:10BB90006401700302BADC12C35912AE9AA3E5081D
:10BBA000F002BADC0E9022A6E493FAEEC39A4003A8
:10BBB00002BADC7D0080010D9022A3E493FAEDC36C
:10BBC0009A40F4ED75F007A424D9F582E5F0341716
:10BBD000F58312AD1012BC4BF583E0687003A3E04F
:10BBE00069700302BADC9022A3E4936D70B6EE751F
:10BBF000F017A4241FFEE5F03417FF7C177D0079B1
:10BC000000EEFAEFFB1214AC8E828F83E50CF0A3EA
:10BC1000E50D12BC588E828F83A3A3A3A3A3A3A375
:10BC2000A3A3A3E8F0A3E912BC607401F0EE240E14
:10BC3000F582EF12B85512907F740202BBA0120E6B
:10BC4000108A0A8B0BA80AA90BE82275F017A42406
:10BC50001FF582E5F0341722F090038012AAC52266
:10BC6000F0EE240F12BC6822F582EF3400F5832237
:10BC7000E50812C071E5093400F583EEF0A3EFF09A
:10BC80002274F21203568A088B09890B8C0C8D0DD5
:10BC9000120D9E9022A3E493FE7001E460097AFEE7
:10BCA0007BFF120D9EE9FE9022A3E493F8C3EE9869
:10BCB000E49400C365D033506AEE12BD7912A0F04F
:10BCC00088828983A3E50BF09003C512B13DF0E8AB
:10BCD0002404F508E93400F509E50BC333FAE4332D
:10BCE000FB12153685088285098312BD287002A3D0
:10BCF000E06030850C08850D09750A007808120887
:10BD000017E50BC333FCE433FDEE75F006A424F312
:10BD1000F582E5F0341812B9BE1299F51208497986
:10BD20000080027907029D1CEAF0A3EBF0850882EF
:10BD3000850983E02274F61203568C088D09740A73
:10BD4000120AAC12BF02120D9EE9F89022AEE493E3
:10BD5000FAC3E89AE49400C365D0335014E812BDE6
:10BD600074E085088285098312AE9B128EB512AAF3
:10BD7000AE029EAF12BD79A32275F006A424EFF89F
:10BD8000E5F0341802B4FA74F7120356750800800F
:10BD90001BE50875F006A424F1F582E5F03418F5EA
:10BDA00083E06A7003A3E06B607205089022AEE442
:10BDB00093FCE508C39C40D9E4936508705E74FE6B
:10BDC0006A700374FF6B7054750800800205089058
:10BDD00022AE12BE34500512BE1F70F112BE315099
:10BDE0003BA808E875F006A4A9F024F3F582E9342D
:10BDF00018F583E07002A3E06022E875F006A42441
:10BE0000EFF8E93418F9740428FEE439FF8E828FC4
:10BE10008312BE3C8E828F83E4F0A3F002A3E7E599
:10BE20000875F006A424EFF582E5F03418F583E0F8
:10BE3000229022A3E493FAE508C39A2212B9C7120A
:10BE4000153C2274F61203567C007D00EA241DF591
:10BE500082EB12908512B4DDA3E0F9600EEA241D96
:10BE600012BEF62402FCA3E03400FD8A828B83A379
:10BE7000A3A3A3A3A3A3A3A312BF02900373E06E83
:10BE80007003A3E06F700DEA128EB1EB12B9BC1211
:10BE90000D92805CEA241112BEF66054FE74FF2EEF
:10BEA000F0750801780812081F8C088D09780812AF
:10BEB000081BE9F508780812081F12BEF3F5087888
:10BEC0000812081FEA2415F582EB12908512069DD0
:10BED000EEF912889F12B8698A828B83A3A3A3A369
:10BEE000A3A3A3A3A312B9C0120DAA7407120849F1
:10BEF000029EAFEA2412F582EB12ADD822790190AE
:10BF00000330E0FEA3E0FF2274F012035674F9122E
:10BF100008DB7405120AAC12AD617403120AAC128C
:10BF2000C9A9E9FF7419120AACE0FE741A120AAC2E
:10BF3000E0F50C741B120AAC12CD7C741D120AAC15
:10BF4000E0F50D6009E50CC3332404FA80027A029F
:10BF50007401120AAC12C08B8A088B09EA7001EBDB
:10BF6000700302C0607405120AAC12C07A12AAAE45
:10BF70007403120AAC12C07AA3A312AAAEEA241365
:10BF8000F582EB129085EFF0EA2414F582EB129023
:10BF900085EEF0EA241712BEF664017050120F6CA1
:10BFA0008A0A8B0BA80AA90B850882850983A3A39B
:10BFB000A3A3E0687003A3E06960327417120AACAF
:10BFC000E07002A3E060197417120AAC12B862E5BF
:10BFD00008241AF582E509129085E8F0A3E9800C9F
:10BFE000E5082417F582E509129085E4F012C06592
:10BFF00012BF0274058E828F83F0A3E50D7004E5F5
:10C000000C80557401250C12C084780079008028BA
:10C01000850E82850F83E012C080850E82850F8396
:10C02000A312C076F0E50E2402F50EE50F3400F5FC
:10C030000FA30EAF8312986C850C0AC3E8950AE92A
:10C040009400A2D265D03340C7120F6CEA12C080B0
:10C05000120F6CEB8E828F83F0AA08AB09120C785A
:10C06000740702C931E50812C071E50912BC6B22E0
:10C07000EA240BF58222E0028EBE12CB8DA3A3220E
:10C080008E828F83F0A3AE82AF8322EA12A1561272
:10C090000FDE22C082C083E9C333F8E43312C0AE9E
:10C0A00074FE28F58274FF3912B9BE02A79FF9EA1F
:10C0B00028F8EB39F92274F312035689088A09EC3F
:10C0C000FEEDFF750C008002050CE50CC3950850D1
:10C0D0002AE50CC333F8E433F9EE28F582EF39F59D
:10C0E00083C082C083120F6C8A0A8B0BD083D082EC
:10C0F000E0650A7004A3E0650B70CDE509650C707E
:10C100000479018002790002A65174F0120356747A
:10C11000F31208DB8A0E8B0F8C088D09E9FE750A75
:10C1200000120FF6E97900600302C1EDAA0EAB0F11
:10C1300012C1F0AE0CAF0DEE7001EF700302C1EB57
:10C140008E828F83A3A3A3A3A3A3E0A2E240030252
:10C15000C1EB120F6CEA65087003EB650970077894
:10C160000A12081F8032AA08AB09120B94E9640175
:10C17000705A7404851082851183F07401120AAC20
:10C18000E508F0A3E50912BAA96401703F750A0138
:10C19000780A12081F750A00750B00780A12081B2E
:10C1A000780A12081F780A12081F7408120AAC8550
:10C1B000820A85830B780A12081B791EAC08AD0928
:10C1C000AA0EAB0F120DAA74071208498E828F8334
:10C1D000A3A3A3A3A3A3E0A2E1400D8E828F83A318
:10C1E000A3A3A3A3A3C2E2F0750A01A90A02C92F5F
:10C1F00012C2218A0C8B0D2274F6120356E912C268
:10C200001A8A088B09A808A909E87001E9600612D2
:10C21000CFE6F980027904029EAFFE790012C221B6
:10C2200022120E1CEEF9120E102274F61203567E24
:10C2300007900367E0704412B8661210DA8A088B20
:10C2400009A808A909E87001E9603090036CE0646E
:10C250000188828983A37016E0C0E088828983A365
:10C26000A3E0FAD0E0C39A888289835001A3A3E0B7
:10C27000F91210F8E9FEEE70027E07029E8C74F04F
:10C280001203568A0A8B0BE9FEECFF8D087410121C
:10C290000AACE0F50CA3E0F50D120E0AE9F50E125A
:10C2A000C3C0504F890A750B007403780A1209DA6B
:10C2B000E50A243DF582E50B3419F583E0FAEFC376
:10C2C0009A502CE5086023750F007403780E12094C
:10C2D000DAE50E2437F8E50F3419F9EF88828983FF
:10C2E000A3A3A3A3A3A312C36EF0790002C9347958
:10C2F0000380F979007AFE7BFF120E0AE9F50E90B1
:10C3000022ABE493650E7004790280E0E50860DA00
:10C310008908750900740378081209DA12C34E8877
:10C32000828983A3E50AF0A3E50B12C36E12C365ED
:10C33000A3A3F074FF88828983A3A3A3A3A3F0EE31
:10C3400088828983F012C359A3A3A3A3809BE50825
:10C350002437F8E5093419F922900371E0888289BD
:10C3600083A3A3A322F0EF8882898302C99312C317
:10C370007AA3A3E50CF0A3E50D2212C37FA322F05C
:10C3800002B4FB74F4120356ECFE120E0A12C3C080
:10C390005029890A750B007403780A1209DAE50A34
:10C3A000243CF582E50B3419F583E0FAEEC39A508C
:10C3B00006EEF07900800679038002790402A47DFC
:10C3C0009022ABE493FAE9C39A2274F6120356EA78
:10C3D000FEEBFF120E0AE9F50812C3C050197509E9
:10C3E00000740378081209DAE508243AF582E509B1
:10C3F000341912B9BE8016900356E07002A3E060B3
:10C400000812B4D6121E7780047AFE7BFF029EAF1C
:10C4100074F61203568A828B83E4A3A3A3A3A3F02A
:10C42000FB80010B9022A7E493FAEBC39A501F8B79
:10C430000812C94AFA8C828D83A3A3A3A3A3A3A342
:10C44000A3E06A70DEECFAEDFB120F1E801EE4938F
:10C450006B701974068C828D83A3A3A3A3A3A3A3DB
:10C46000A3A3F07A008C828D8312C5AB029EAF74B9
:10C47000F41203568A088B098A828B83A3A3E014E3
:10C4800012C590E0F9120EFA8A0A8B0BAE0AAF0BB6
:10C49000EE7001EF700302C58D850882850983A3C4
:10C4A000A3E070288E828F83A3A3A3A3A3A3A3A337
:10C4B000A3E06402600312C5A574068E828F83A375
:10C4C000A3A3A3A3A3A3A3A3F002C58D850882857C
:10C4D0000983A3A3A3A3A3A3E0700302C5708508E7
:10C4E00082850983A3A3A3A3E0700302C58DE50899
:10C4F0002403F582E50912B9B3600302C58D8508EE
:10C5000082850983A3A3A3A3E01412C5B6E0640344
:10C510007051850882850983A3A3A3A3E0700DEE63
:10C52000FCEFFDAA08AB09120DE0803774048E827F
:10C530008F83A3A3A3A3A3A3A3A3A3F01214BE8AD0
:10C540000A740F550AF87401288E828F83A3A3A35F
:10C55000A3F0A3E4F07A20FB12CB9E7001EB7003F2
:10C5600012C598900360E085088285098302C4C5DE
:10C570008E828F83A3A3A3A3A3A3A3A3A3E0640397
:10C58000700BEEFCEFFDAA08AB09120DE002A47DD2
:10C59000F08A828B8302C9927A207B009003CDE0DF
:10C5A000F91214FA227AF08E828F83E0240C12B6EC
:10C5B0009CF9120E522212A51202C99374F61203AC
:10C5C000567C007E0080258E08750900740378086B
:10C5D0001209DAE5082477FAE5093419FB8A828B17
:10C5E00083A3A3E06005120DE67C010E9022A7E470
:10C5F00093FAEEC39A40D074016C70097C647D009C
:10C600007A4012C99E029EAF74F41203568C088DB4
:10C61000097E777F197C0080378E828F83A3A3A346
:10C62000A3A3A3A3E0FD12BEF36D701B8E828F83C4
:10C6300012B86212ADCE687003A3E06970098E82F1
:10C640008F83A3A3E0701E0CEE2408FEEF3400FFDE
:10C650009022A7E493FDECC39D40BEE4936C70056B
:10C66000790002A47D8E828F83A3A3A3A3A3A3E05A
:10C670007004790180EC12C70A7001EB600D8E82A4
:10C680008F83A3A3A3A3A3A3E014F07C0080010CD9
:10C690008C0A90229B12C703E4995025EC12C6F62F
:10C6A00060EDEC75F012A412C6F165087004A3E009
:10C6B000650970DB8E828F83A3A3A3A3A3A3E014D9
:10C6C000F09022A6E493F890229BE49328F8A3E448
:10C6D000933400F98E828F83A3A3A3A3A3A312CDC7
:10C6E000D5508FE48E828F83A3A3A3A3A3A3F0804E
:10C6F0008112C962E02275F012A4A9F012C943E9BF
:10C700000295C1129DC2E50A982212CD4D1210B0B9
:10C71000EA2274F012035674F71208DB7401120A4D
:10C72000AC12AD617403120AAC12C9A9E98510827A
:10C73000851183F07E777F197508017509009022B5
:10C74000A6E49378081209DAE5093395E0F50AF5CD
:10C750000B90877F780C120A6D7405120AAC780C66
:10C76000120A5E7A0080128E828F83A3A3E0601883
:10C770000AEE2408FEEF3400FF12C96C40E9E4938E
:10C780006A7005790002C92B1290897403120AACF1
:10C7900012B9C01210B0EA7001EB600D8E828F8367
:10C7A000A3A3A3A3A3A3E004F07A008032640160F2
:10C7B00005E0640370217401120AAC12C98BA3A3B3
:10C7C000A3A3E064FF7004A3E064FF700A74051281
:10C7D0000AAC78081209A10A740178081207F48AD1
:10C7E0000C12C9765055EA75F012A4F8ABF012C9D4
:10C7F0005B12B8627403120AACE0687003A3E069CC
:10C8000060D5EA75F012A4F812C95B12C9827003F0
:10C81000A3E06960C2EA75F012A4F8EBF9E812C966
:10C8200043E912937164046003E070818E828F8308
:10C83000A3A3A3A3A3A3E004F0809C8E828F83A371
:10C84000A3A3A3A3A3E0600F7401120AACE0241118
:10C8500012B68B64017003E48005900361E0048EDE
:10C86000828F83A3A3A3A3F090036612C076A3A331
:10C87000F090036012C076A3A3A3F07401120AAC77
:10C88000E0240B12C939128EB5E8F0A3E912C9B041
:10C890008E828F83A3A3A3A3A3F07401120AACE03A
:10C8A000241212B68B8E828F83A3A3A3A3A3A3A368
:10C8B000F07405120AACC082C08390877F7808129A
:10C8C0000A6DD083D08278081208F160497A00801E
:10C8D000010A12C96C503F8A0812C94A600BFB85D5
:10C8E0001082851183E06B70E875090085108285E0
:10C8F0001183E0C0E0E50812C951D0E0F0740512E0
:10C900000AAC780C120A6D740278081209DA12CB9C
:10C910007C780C120A5E7A4012CB9C7001EB700995
:10C920007C647D007A4012C99E790174098002748A
:10C930000D1208497F080205ADF8A3E0340002B4E7
:10C94000FAFDEC24A9F582228E08E50812C951E00F
:10C950002224BFF582E43419F58322EBF9E812C9E9
:10C96000622224A5F582E93415F583229022A7E4FA
:10C9700093FBEAC39B2290229B129DC2E50C98E494
:10C98000992212AAC5900373E0682212C98F22125D
:10C99000B4E5A3A3A3A3A3227CE87D037A107B00C4
:10C9A0009003CDE0F91215D822ECF0A3EDF022A30C
:10C9B00012C9B42212A0E8E02274F41203567508DA
:10C9C00000800205089022A712BE34500D85080A87
:10C9D000E50A12C94C6970EBE4F002A47D74F01210
:10C9E000035674FC1208DB8A0E8B0F8A828B83A39A
:10C9F000A312B9C0120F00EA7001EB600302CB1260
:10CA000090877F7808120A6D85108285118312A0A5
:10CA1000F2A3E50AF0A3E50BF07508017509009093
:10CA200022A6E49378081209DAE5093395E0F50ABD
:10CA3000F50B7E0080080E740178081207F48E0C46
:10CA400012C976502DEE12C6F660EBEE75F012A408
:10CA500012C95E12B862850E82850F83A3A3E068B7
:10CA60007003A3E06970CF85108285118378081266
:10CA70000A5E7E0080057A007B000E9022A7E49378
:10CA8000FCEEC39C400302CB1212C94860EC75094E
:10CA900000740278081209DA12CB7CC082C0838548
:10CAA00010828511837808120A6DD083D0827808AD
:10CAB00012097B90877F78081208F160BD12C9487F
:10CAC000F9120EFAEA7001EB60AC8A828B83A3A3A1
:10CAD000A3A3A3A3A3A3A3E06405709A85108285F2
:10CAE00011837808120A6D7808120A2F8E0C750DC2
:10CAF000007402780C1209DAE50C24C8F582E50D01
:10CB00003419F58378081209B49022A7E493FE0241
:10CB1000CA7AEA7001EB60128A828B83A3A3A3A373
:10CB2000A3A3A3A3A3E06405601D850E82850F83E4
:10CB3000A3A3A3A312B869850E82850F83A3A312B2
:10CB4000B9C0121CF88030850E82850F83A3A31212
:10CB5000CB89E0FCA3E0F5838C8212AAAE74018A33
:10CB6000828B83A3A3A3A3A3A3A3A3A312CB957098
:10CB700001EB700312C598740402C931E50824C89A
:10CB8000F582E5093419F5832212CB8D22E0F8A352
:10CB9000E0F902B6B8F07A2012CB9C227B00900319
:10CBA000CDE0F91215E4EA2274F6120356E9FC7995
:10CBB000008001099022ABE493FDE9C39D503D89BB
:10CBC00008750900740378081209DAE5082438F5B5
:10CBD00082E5093419F583E06A7003A3E06B70D332
:10CBE0008908750900740378081209DAE508243702
:10CBF000F582E5093419F583E06C70B7029EAF74D5
:10CC0000F7120356E95440F97E007F008057EEFC8E
:10CC1000EFFDEC75F007A4FCA8F075F007EDA42873
:10CC2000FDEC24D7F582ED3417F583E06A7003A399
:10CC3000E06B702E74FE6A700374FF6B700302CC9D
:10CC4000DBEEFCEFFDEC75F007A4FC75F007EDA43E
:10CC500028FDEC24DDF582ED3417F583E0544069BE
:10CC600060791292399022A3E493FCC3EE9CEF9476
:10CC700000409BE4936E7001EF707974FE6A70035C
:10CC800074FF6B706F7E007F0080031292399022D8
:10CC9000A3E493FAC3EE9AEF94005058EEFAEFFB38
:10CCA000EA75F007A4FAACF075F007EBA42CFBEAE8
:10CCB00024DBF582EB3417F583E070CFEEFAEFFB5F
:10CCC000EA75F007A4FA75F007EBA42CFBEA24D769
:10CCD000F582EB341712B9BE120DC2EE75F007A43F
:10CCE000FEAAF075F007EFA42AFFEE24D7FAEF347E
:10CCF00017FB80047A007B00029A8474F4120356B6
:10CD00008A088B09E9FFEC12C21A8A828B83E582BA
:10CD10007002E583600DA3A3A3A3A3E06F70047961
:10CD200000801A74016F701312CD407002E58360A9
:10CD30000AE0C394035004A3E070E4790102A47DE7
:10CD400012CD4D1210DA8A828B83E5822290038005
:10CD5000E0FCA3E0FDAA08AB092212CD5E22E02888
:10CD6000FAA3E0398A82F58322E02AFCA3E03B8C17
:10CD70008222EA2EF582EB3FF583A322E0F50EA393
:10CD8000E0F50F2274F6120356EAFEEBFFE9A2E685
:10CD9000501A79FF121DB8EA7001EB600990037315
:10CDA000E0FAA3E0802B7AFE7BFF802612B4C970E4
:10CDB00001E9601A88828983A3A3A3A3E0640160C8
:10CDC000DC88828983A3A3A3A3E0640260CFEEFA88
:10CDD000EFFB029EAFE0FAC3E89AE994002274F5F3
:10CDE000120356EAFEEBFF8C088D09740B120AAC95
:10CDF000E0F50A74026970127C1EA90AEEFAEFFBD4
:10CE0000120D44E9703379018031740169702AACE4
:10CE10000A7901120E16E96020E5087002E5096042
:10CE2000D7EEFAEFFB120D9E9022AE12C3C350C88C
:10CE30007401850882850983F07900029B0974F6E4
:10CE40001203567C0079057A007B0080638E828F06
:10CE500083A3A3A3A3E07002A3E0604CEE2404F834
:10CE6000EF12CEC424FFF0A3E034FF12C37FE070C2
:10CE700002A3E0703374068E828F83A3A3A3A3A3BF
:10CE8000A3A3A3A3F012C5A58E828F83A3A3A3A3FC
:10CE9000A3A3E0540460118E828F83A3A3A3A3A352
:10CEA000A3A3A3E0F9120DFE7C007905EEFAEFFBD7
:10CEB000120EF48A088B09AE08AF09EE7001EF700C
:10CEC0008C029EAF3400F988828983E02274F012CC
:10CED00003568A088B09ECFEEDFF7410120AAC129F
:10CEE000CD7CE96004790B80547900EEFAEFFB12F7
:10CEF0000E108A0A8B0BEA7001EB60448A828B83E6
:10CF0000A3A3A3A3A3A3E0A2E05035AC08AD09AA54
:10CF10000EAB0F1210EC8A0C8B0DA80CA90D74FE31
:10CF200068700374FF696018850A82850B83A3A368
:10CF300012AAAE790CAC08AD09EEFAEFFB12102C78
:10CF400002C93474F712035678D779177C007D0034
:10CF5000804488828983A3A3A3A3A3A3E0A2E04083
:10CF60002A88828983A3A3E06A7003A3E06B701B05
:10CF700088828983A3A3A3A3A3E06401700D740333
:10CF800088828983A312B14112B9D9EC24010CED36
:10CF90003400FD12CFA79022A3E493FEC3EC9EEDD4
:10CFA000940040AE029A84E82407F8029870C08288
:10CFB000C08378D779177A007B00801912CFE68872
:10CFC000828983A3A3A3A3A3A3F0EA24010AEB34D9
:10CFD00000FB12CFA79022A3E493FCC3EA9CEB943E
:10CFE0000040D902A79F8882898374FEF0A374FF52
:10CFF00012C37A12B9E9A3A3A3A312AE9FA3F0228E
:10D00000C082C083901262E4F0A3F07C037D037AB7
:10D01000ED7B11121CA4120C727900121E6002DF4B
:10D020007C74F5120356EAFFEBFEE9704374026F5D
:10D030007053901A7E7408F0750A00780A12081F5F
:10D04000ECF50A780A12081FEEF50A780A12081F92
:10D05000901A8C120699901A90E0F97CC57D129076
:10D060001AA412DAB7120C907407120849E960107A
:10D070007CE87D037A017B009011F5E0F91215D868
:10D080007F030205AD74016F7010901A7E7408F072
:10D090007B00EEFAF9120CA280D37C897D867A3F60
:10D0A0007B8612193E80C974F412035689089004D5
:10D0B000B812DA17120F6C9011E312DA9E120F6693
:10D0C00080308E828F8312DA10601B7A027B00120E
:10D0D00014C4EA4B60108A828B8374D1F0A3E508F4
:10D0E00012E56312D7DA8E828F83A3A3A3A3A312C0
:10D0F000DA17EE4F70CC7F040205AD74F0120356C0
:10D10000E9FD8A0E8B0F7410120AAC12DA17741232
:10D11000120AAC12D1D47A007B008051E50CC333E3
:10D12000F8E433F9EE28F582EF39F58312D7D2EB24
:10D13000C333F8E433F9E50E28F582E50F39F583BA
:10D14000E0650A7004A3E0650B7019EAC333F8E4E4
:10D1500033F9E50828F582E50939F583E50AF0A3F6
:10D16000E50BF00A050CE50CC39C40B00BEBC39D2E
:10D170005005750C0080EFEAF902DA7A74F41203B4
:10D1800056E9FEECFF740C120AAC12DA88750B003B
:10D190008002050BE50BC39E5033750A0080020523
:10D1A0000AE50AC39F50EBE50BC333FCE433FDEA09
:10D1B0002CF582EB3D12D1D2E50AC312E7C4E0653B
:10D1C000087004A3E0650970D67901800279000235
:10D1D000D0F6F58312E09B2274F612035612D26643
:10D1E0007003A3E06D70177508F8750911780812BF
:10D1F000081BEEFA12183C7402120849801A7508CE
:10D2000002750980780812081B8C088D09780812AD
:10D21000081B12D281120849800574021208497F46
:10D22000020205AD74F612035612D2667003A3E033
:10D230006D7017750805750912780812081BEEFA4B
:10D240001218427402120849801A75080375098081
:10D25000780812081B8C088D09780812081B12D256
:10D260008112084980B9EAFEEBFF12D27BEF12DA95
:10D27000D7FCE439FD9011E3E06C22EE2413F58233
:10D2800022EE240E12E0C3FD7C8012D9FF12E0C30F
:10D29000F912185474042274F612035674FE12081C
:10D2A000DBEAFEEBFF851082851183E4F0A3F01228
:10D2B000D27BEF12DB00FA88828983A3A3E0F975A1
:10D2C00008007509006005C394F140057509828066
:10D2D000299011E3E06A7003A3E06B701A85108255
:10D2E000851183AA82AB8312146AE9F50812DF83E1
:10D2F0007008750983800375098185108285118303
:10D3000012DA7FA909EEFAEFFB121848E508600867
:10D3100012DF83600312DA3502D21A74F212035656
:10D320008A0C8B0D75080075090012DACC120F6C8F
:10D33000EA6E7002EB6F7012121476E914F5087938
:10D34000017A2E7B1212147C8003750980E50C246F
:10D350000E12DAC4F50A780A12081F750A2E750B28
:10D3600012780A12081B780812081F8E0A8F0B7891
:10D370000A12081BE509F508780812081F12DAEAF4
:10D38000F582E50D12DA0B7A057B8012184E02E861
:10D39000BA74F6120356E9FE7F00802F8A828B83CF
:10D3A00012D9C0F9E5082400E439F509EF33F8E4AF
:10D3B00033F9EC28F582ED39F583E508F0A3E509AA
:10D3C000F0EA24020A0AEB3400FB0FEFC39E40CCC4
:10D3D00002D21F74F012035674F51208DB740312A4
:10D3E0000AAC12DA9E7402120AACE4F07409120A52
:10D3F000ACE4F0A3F07407120AACE4F0A3F07403F9
:10D40000120AACE0241312DEBB12D7D2850A82F5D1
:10D410008312E5402400F508E439F509850A828580
:10D420000B83A3A3E0FA850A82850B83A3A3A3E061
:10D43000F9EAFEE439FFE50A2404F50AE50B3400B5
:10D44000F50BAA08AB09120FF6E96401703C7403EE
:10D45000120AAC12D7E512081FE4F508F50978089E
:10D4600012081B780812081F9011E312069D750818
:10D4700080780812081F740A120AAC12D7C6120A62
:10D48000AC12D7F012084902D7A7AA08AB09120FAD
:10D49000F6E9700E9011E3E065087004A3E06509F9
:10D4A00070AC12D7AC880F602EC333FAE433FB1292
:10D4B00015367409120AAC12DA9E7409120AAC12FB
:10D4C000DF8960137409120AAC12D7BCA90F1217B6
:10D4D000B28A0A8B0B8003750F0012D7AC880E60DE
:10D4E0002AC333FAE433FB1215367407120AAC125E
:10D4F000DA9E7407120AAC12DF89600F7407120AF1
:10D50000AC12D7BCA90E1217B28003750E0090049E
:10D51000B8804DE4F0A3F0AA0CAB0D7405120AAC70
:10D5200012DA10F8A312D7DA85108285118312DA85
:10D5300010C0E07402120AACE0F8742E28F5827470
:10D540001212E683D0E0F07402120AACE004F0E5B7
:10D550000BA2E0500312DA357405120AAC12E87718
:10D5600012DA887405120AAC12DA507405120AAC89
:10D5700012DF89700302D7277405120AAC12DA2170
:10D58000E8FAE9FB8A828B83E060CD7405120AAC6D
:10D5900012E86BA3E0A2E050BF7405120AAC12DAE5
:10D5A0001D12DA85E8FCE9FDEC4D8A828B83601957
:10D5B000E0FA79018C828D83121E778510828511A5
:10D5C0008312DA9E750B01800F12DA858510828531
:10D5D000118312DA50750B0012DF83700302D54FEE
:10D5E00085108285118312DA1DA3E06E7003A3E01B
:10D5F0006F600302D54FE50F7004E50E605B851088
:10D600008285118312E879A3A312069D7402120A7F
:10D61000AC12E881E0FC740B120AAC12DAB7A90F65
:10D620001217947402120849E9702E851082851130
:10D630008312DA3012069D7402120AAC12E898E0E6
:10D64000FC7409120AAC12DAB7A90E12179474020C
:10D65000120849E9700302D54FE50E250FC33324A4
:10D660000AFA7B001214C48A0C8B0DEA450D700374
:10D6700002D5288A828B8374D2F07403120AAC120A
:10D68000E37C8A828B8312DA4E8A828B83A3A3A3E4
:10D69000A3E50F12E74DA3A3A3A3E50EF0EA24052B
:10D6A000FAEB3400FBE50F6033E50C240AF8E50DD6
:10D6B0003400F98A828B8312DA507409120AAC1290
:10D6C000E8A7120817E50FC333FCE433FD8A828B09
:10D6D0008312DAB712E08712084980088A828B83A6
:10D6E000E4F0A3F0E50C2408F582E50D12E683E5ED
:10D6F0000E700302D513E50FC333F8E433F9E50CDC
:10D7000028F8E50D39F9E8240AFAE93400FB12DAC1
:10D710009E7407120AAC12E8A7120817E50E12E071
:10D720008112084902D5177402120AACE0604974EC
:10D7300003120AAC12D7E512081F75082E750912DC
:10D74000780812081B7405120AAC12DA9812081F26
:10D750009011E312069D750800780812081F740ADC
:10D76000120AAC12D7C6120AAC12D7F0120849E955
:10D7700070117C107D8780047CA37D867A6D7B860A
:10D7800012193E7409120AAC12DF8960087409127A
:10D790000AAC12DA3B7407120AAC12DF8960087413
:10D7A00007120AAC12DA3B740B02DA56850A82853C
:10D7B0000B83E0F8A385820A85830B22E0FCA3E0BB
:10D7C000FDAA0AAB0B22E02402FCA3E03400FD74A6
:10D7D0000A22E0F50AA3E0F50B2212E87212DA74CD
:10D7E000F91214D022E0240E12E3B2F508780822D0
:10D7F00012DA6B7A067B8012184E74072274F012CC
:10D80000035674F41208DB8A0A8B0BECFEEDFF74EE
:10D810000B120AAC7403F0120AACAA82AB83121C7E
:10D82000A4120F66EAFCEBFD7403120AACAA82ABE9
:10D8300083121C9EE9600E12D9B8F8740368601058
:10D84000740168600B851082851183748402D96726
:10D850008E828F83A3A3A3A3A3A3A3A3E0F9602134
:10D86000C394F1501CEE2414F508EF12E70F740373
:10D87000687019850882850983E06005C394F140CA
:10D880000B851082851183748202D967EE240BF513
:10D890000EEF3400F50FE50A240CF582E50B12DAE1
:10D8A000C864217002A3E0600302D9338510828529
:10D8B00011837487F0120BFA90229DE493F874019F
:10D8C00093F9C3EA98EB99400302D96812DA9212ED
:10D8D000081FAC0EAD0F8E828F83A3A3A3A3A3A3B7
:10D8E000A3A3A312DAB78E828F83A3A3A3A3A3A3B8
:10D8F000A3A3E0F9121E067401120849E9706985B4
:10D900001082851183E4F012172812D9B8640370CD
:10D91000577401120AACAC82AD83AA0EAB0F121D74
:10D92000EEE970447D007C007900AA0EAB0F12185E
:10D9300024803512DA9212081FAC0EAD0F8E828F42
:10D9400083A3A3A3A3A3A3A3A3A312DAB7121E00C6
:10D950007401120849E98510828511837007E4F08B
:10D9600012172880037488F012E674E50B12E68320
:10D9700012DA9812081F7401120AAC858208858396
:10D9800009780812081BE50A240CF582E50B12D968
:10D99000BD4480F509780812081B7901E50A2402C4
:10D9A000FCE50B3400FDE50A240FFAE50B12DAF969
:10D9B000120849740C02DA5612DAA4E02212DA4292
:10D9C000E0F508A3E022C082C08374F31208DB856F
:10D9D0001082851183E4F004120AAC12DA9E7403FB
:10D9E000120AACAA82AB83120B3485108285118394
:10D9F000AA82AB83120B6A740D12084902DF7CEE17
:10DA00002402FAEF3400FBEE240F2212E0C6F922C2
:10DA100012DA742212E726E0FEA3E0FF2212DA29CE
:10DA20002212DA2912DA8C22F8A3E0F58388822206
:10DA300012E89CA32285108285118312DABB12158D
:10DA40003C223400F58322EE240412E55822A3A3DD
:10DA5000E8F0A3E9F022120849801F2406F8A3E0A9
:10DA60003400F9740122F812E3B322E0240FF81213
:10DA7000E3B7F922E012DA28E0227F080205ADE0E0
:10DA8000FCA3E0FD22A3A3A312DA8C22E0F8A3E01A
:10DA9000F922850882850983E0F508780822EAF0F2
:10DAA000A3EBF02212D27BEF3400F58322AC82ADDF
:10DAB0008385108285118312DABB22E0FAA3E0FB92
:10DAC00022020533F582E50D12E0C62212E6A41209
:10DAD000DAD7FEE439FF2212E6AEFAA3E0F9EA242F
:10DAE0000022F085108285118322E50C2402FCE5DA
:10DAF0000D3400FDE50C240F223400FB12E36C22F0
:10DB000012E6AAFCA3E0FBEC2274F612035674E0C2
:10DB10001208DBEAFEEBFF851082851183AC82AD33
:10DB20008312180C1211107402120AAC12DAAD1220
:10DB3000101AE96401700302DC8A740B120AACAAA1
:10DB400082AB83120F787402120AACAC82AD83747C
:10DB50000B120AACAA82AB83121C9EE96032120F30
:10DB6000728A088B09A808A909851082851183E0AB
:10DB7000687003A3E069601885108285118312DA4A
:10DB80008890037612DA507A767B03794B121CBCAC
:10DB9000EE2411F582EF12E683C082C083120F6C6F
:10DBA0008A088B09D083D082E065087004A3E06501
:10DBB0000960327402120AACAA82AB83120BA68AE5
:10DBC000828B83E5824583601CA3A3A3A3E0F87442
:10DBD00001686005740268700C7402120AACAA82B3
:10DBE000AB83120BB2120F6C8A088B09A808A90923
:10DBF000851082851183E0687003A3E069601C745E
:10DC000002120AAC12DAAD120B88E9600E7402122D
:10DC10000AAC12DAAD1210F21217287413120AAC01
:10DC2000E412E3F0F8A3E0F97414120AAC12DA502B
:10DC30007413120AACAA82AB83120B58E9604B7CB6
:10DC4000087D007900740B120AACAA82AB8312140F
:10DC5000AC7416120AACAC82AD83740B120AACAA77
:10DC600082AB83121C9EE960217402120AACAC8262
:10DC7000AD837416120AACAA82AB83120B347413F0
:10DC8000120AACAA82AB83120B6A742002D21C3433
:10DC900000F50B850A82F5832274F012035674F6A0
:10DCA0001208DB8A0E8B0F7E0090126412DF8970DF
:10DCB000457A377B0012153690126412DA9E901264
:10DCC0006412DF8960197C377D0079001214ACACD6
:10DCD0000EAD0F90126412DAB71217E2E9700B85DD
:10DCE0001082851183748802DE0112DEBF7401F098
:10DCF00012E35002DEA412DEBF7402F0AC0EAD0FD0
:10DD000012E3431217E2E9700A85108285118374C9
:10DD100088F00E75082E750912780812081B9012EB
:10DD200064E0242912DEBB12069D901264E02428D0
:10DD300012DED8241512DEEB241412DEE11208499B
:10DD4000E9C0E0901264E0243112DEBBD0E0F012B2
:10DD5000E3A8750A00602512DEA9243212DEFD60F8
:10DD600010780812081712E3A812E08112084980FF
:10DD70000B8510828511837488F07E01750C2E75D9
:10DD80000D12780C12081B901264E0241212DEBBF4
:10DD900012069D901264E0241112DED8242C12DEAB
:10DDA000EB242B12DEE1120849E9C0E0901264E096
:10DDB000243412DEBBD0E0F012DEF3601812DEA9CC
:10DDC000243512DEFD6029780812081712DEF312DE
:10DDD000E081120849EEA2E0401F12E3A87005128C
:10DDE000E38F60157B007A0079001217E802DEA449
:10DDF0008510828511837488F08510828511837463
:10DE000086F07409120AAC7402F0850E82850F83C5
:10DE100012DA867401120AAC12DA50850E82850F6E
:10DE200083A312DA9812081F7401120AAC858208C3
:10DE3000858309780812081B750820750980780801
:10DE400012081B79017406120AACAC82AD83AA0ECB
:10DE5000AB0F12E36C12084912E39C704474091270
:10DE60000AAC740212E3E7F583888212DA86740141
:10DE7000120AAC12E40B12081F7401120AAC85825C
:10DE800008858309780812081B75082075098078B1
:10DE90000812081B79017406120AAC12E35E12081C
:10DEA000491217DC740A02DA56C333FAE433FB1260
:10DEB00015368A0C8B0D901264E02212DEC9229076
:10DEC0001264E0242E12DEC922F8A3E012DED02272
:10DED0003400F9888289832212E3B2FC901264E054
:10DEE000221812DA6F12178E74042212DF95901224
:10DEF00064E022901264E0243412E3B22212E3DCE4
:10DF0000E50CF0A3E50D12E51D12DABBEA4B22C0C9
:10DF100082C08390126412DF896061901264E024F1
:10DF20003512DF8F600312153C901264E024321228
:10DF3000DF8F600312153C901264E0241212DF8F11
:10DF4000600312153C901264E0241512DF8F600309
:10DF500012153C901264E0242912DF8F6003121521
:10DF60003C901264E0242C12DF8F600312153C9069
:10DF7000126412DA3B901264E4F0A3F0D083D082F2
:10DF800002053385108285118312DA8CE84922124A
:10DF9000DF95EA4B22F812E3B7FAA3E0FB2274F014
:10DFA0001203568A0C8B0D8C0E8D0F7E018C088D02
:10DFB00009750A0078081208177C177D0012E0879F
:10DFC000120849E50C2412F582E50D12E683E4F00F
:10DFD000A312E0CCE4F0A3F0E50E2411F582E50FE6
:10DFE00012DAC86039C333FAE433FB121536E50C94
:10DFF0002412F582E50D12E68312DA9EE50C241256
:10E0000012DAC4FA4B6016E50E241212E08D1208E3
:10E0100017E50E241112E0B012084980011EE50E2A
:10E020002414F582E50F12DAC86030C333FAE43302
:10E03000FB121536E50C2415F582E50D12E52312C9
:10E04000E0CCE0FA4B6036E50E241512E08D1208A4
:10E0500017E50E241412E0B0120849EEA2E04018B1
:10E06000E50C241212E0A3600312153CE50C241504
:10E0700012E0A3600312153CEEF902DA7A7E00800A
:10E08000DFC333FCE433FD1214A0740322F582E5F0
:10E090000F340012E099780822F583E0F508A3E038
:10E0A000F50922F582E50D12DA4212DABBEA4B22BB
:10E0B000F582E50F12E0C6C333FCE433FD1214A071
:10E0C000740322F582EF3400F583E022F0E50C249E
:10E0D00015F582E50D12DA422274F012035674EA45
:10E0E0001208DB7403120AACEBF0890E8A0F750A72
:10E0F00000750B00851082851183E412E3E7F9E8CF
:10E10000497005790002E33E7403650E60067402EF
:10E11000650E700E7403120AACE0FA12E372E06A44
:10E1200070E17CEE7D177A007B00121E547401654D
:10E130000E700B8510828511837485F0803E9012DD
:10E1400064E0242F12DEBBE50E60067403650E70DA
:10E15000157401F07403650E701EE50F601E8510C6
:10E160008285118380D57402650E7010E50F7004EE
:10E17000740180C7740280C3E50E601912E38370D6
:10E1800014901264E02431080812DA67700512E373
:10E190008F600214F012E3A8F8901264602212D784
:10E1A000D2E8C333F8E433F9901264E0243212E386
:10E1B000C2241D12DA5D120AAC12E3FD2425802F61
:10E1C00012DEF6F8602E901264E02417F50AA3E040
:10E1D0003400F50BE8C333F8E433F9901264E0241B
:10E1E0003512E3C212DA5B120AAC12E3FD240E12FE
:10E1F000DA66F50D740C120AAC740212E3F06003D7
:10E2000002E2B0E50A450B700302E2B012E383704C
:10E21000047E2280027E21850A82850B8312DA86A3
:10E220007404120AAC12DA50901266E0C0E012E3F5
:10E2300072D0E0F07415120AAC7403F07401120A83
:10E24000AC12DA7F740D120AACAA82AB83121CA442
:10E25000850A82850B83A3E0F50C780C12081FE574
:10E260000DF50C780C12081F740F120AAC85820C85
:10E2700085830D780C12081B780812081BE50A2408
:10E2800006F508E50B12E70F780812081B12E67472
:10E29000E50B12DA0B740C120AACAC82AD83EEFA09
:10E2A0007B00121860740812084912E35002E33C24
:10E2B00090126412E37C7404120AAC12E40B12088C
:10E2C0001F7401120AAC8582088583097808120838
:10E2D0001B750820750980780812081B79017409DC
:10E2E000120AAC12E35E12084912E39C704B9012C2
:10E2F00064E0241912DEBB12DA887404120AAC122C
:10E30000E3FD241812D7E812081F7401120AAC8525
:10E310008208858309780812081B75082075098012
:10E32000780812081B79017409120AACAC82AD831B
:10E3300012E34312E36C1208491217DC79017416D8
:10E3400002DA56901264E02417FAA3E03400FB22AC
:10E350007CEE7D1790030112DABB121E5422AC82B0
:10E36000AD8390126412DABB12E36C2212181E7491
:10E370000522901264E0243012DEC92212E88912CC
:10E38000DA8C22901264E0242F12E3B2640122900E
:10E390001264E0243408080812E3B322901264E007
:10E3A000242E12E3B2640222901264E0243112E3BC
:10E3B000B222F812E3B722A3E03400F988828983FD
:10E3C000E02212E3DCE028F8A3E039F9E824FEF5C6
:10E3D00082E934FF12E099901264E022FAA3E0345B
:10E3E00000FB8A828B8322F0901264E0F8A3E02283
:10E3F00012E3F42212E3F82212DAE2E02212E4013C
:10E4000022E8F0A3E9F0901264E02212E40112E89D
:10E4100070E0F508780822C082C0837B007A857995
:10E42000011217E802DF7C74F11203568C088D0983
:10E43000EA240F12E7DC12E51D12DA868C828D8346
:10E4400012DA4EEA240E12E7DCA312E8B0FEA3E0D3
:10E4500012E53B8C828D83A3A3A3A312E85A240662
:10E46000FAE50912E547C0E0E508240E12E67FD080
:10E47000E012E804F8E508240F12E67FE812E66EE1
:10E480002412F50AE50912DC8FE4F0A312E56AE430
:10E49000F0A312E5630EAF83E508241112E52B60AB
:10E4A0002412E7E8FCA3E0FDEC4D6019EEFAEFFB67
:10E4B000850C82850D83E0F91217B28A0A8B0BAEA8
:10E4C0000AAF0B8008850C82850D83E4F08E828F65
:10E4D00083E0F8A3AE82AF83E508241412E52B6035
:10E4E0002FC333FAE433FB121536E5082415F58201
:10E4F000E50912E52312E56A12DA7FEC4D6011EEB0
:10E50000FAEFFB850C82850D83E0F91217B28008C3
:10E51000850C82850D83E4F07F070205ADF08A82C9
:10E520008B832212DA42EAF0A3EB22F50CE50934E0
:10E5300000F50D850C82F583E8F022FF8E828F8333
:10E54000E0FAA3E0F9EA223400FB12E54E22121CA5
:10E55000A4EE240812E55822FEEF3400FF8E828FCD
:10E5600083E02212E714E0F8A322F0E5082415F571
:10E5700082E50912DA422274F61203568C088D09DC
:10E5800012DA1412E75E7014EEFCEFFD12E849C0D7
:10E59000E0E508241412E67FD0E0800312E73FF0A4
:10E5A00002D21F74F2120356EA2413FEEB3400FF6A
:10E5B000EA2410F582EB12DAC8C3940C400E8E8266
:10E5C0008F83E0240B12DA66F50A8003750A00E5F2
:10E5D0000AC333F8E433F9E8240DFAE912E8648A4F
:10E5E000088B09EA450960758E828F8312E7228ABB
:10E5F000828B8312E6F67065EEFCEFFDEA24030AD7
:10E600000A0AEB12E54712E93C12E66E240BF8E524
:10E61000093400F9E8FAE9FB8A828B83E4F0E50A21
:10E62000603BE508240D0808E5093400F9AC0A8EC2
:10E63000828F8312E66812E71AC0E012E67BD0E010
:10E6400012E7528E828F83E0F50AA3E0FBE50A8889
:10E6500082898312E68712E6641CEC70E6AA08AB96
:10E660000902E8BF12E7BA22E08A828B832212E70E
:10E67000AEE50822E50A240EF58222E508240CF511
:10E6800082E50912DA4222F0A3EBF012E68F22E8CB
:10E6900024020808E93400F92212E69EE022F088FC
:10E6A00082898322EA12D27CEB2212E6AE22340067
:10E6B000F583E0F8A3E0F988828983E0227F0102F4
:10E6C00005AD74F7120356EA2413F8EB12DED0E01E
:10E6D000FAA3E0F5838A8212E7E212E699F8A3E052
:10E6E000F988828983A3E0FA88828983A312E7D21A
:10E6F00012DA5102E6BD12E6FA2212E6FE22F08E8E
:10E70000828F83A3AE82AF832212E51DA3A322349E
:10E7100000F50922F08E828F832212E756E0221242
:10E72000E72612E7342212E72A22EA12D27CEB34DF
:10E7300000F58322E0FEA3E0FF8E828F83E022E0DB
:10E74000FCA3E0F9EC8A828B83F0A3E92212E709AB
:10E75000A32212E7562212E714A30EAF8322EEFC87
:10E76000EFFDAA08AB0912E54E850882850983A34F
:10E77000A3A3A3A3A3A3A312E80885088285098302
:10E78000A3A3A3A3A3A3A3A3A312E7AE8E828F8305
:10E79000E0F8E50812D27CE50912DA42E812E75601
:10E7A000E508240BFAE5093400FB74036822F0A3A2
:10E7B000E912E7B522F012E7BA22EE24020E0EEFBC
:10E7C0003400FF2233FCE433FDE82CF582E93DF50B
:10E7D0008322A3E0F9EA8C828D83A322F582EB12D7
:10E7E000DA42E08C828D8322C333FAE433FB1215C4
:10E7F00036850A82850B83EAF0A3EBF0850A8285D1
:10E800000B83E02212E8082212E6FEE0FAA3E0F908
:10E81000EA2274F61203568C088D0912E71FFAA338
:10E82000E0F9EA8C828D8312E85A2402FAE5093471
:10E8300000FB12E849850882850983A3A3A3A3A34B
:10E84000A3A3A3A3A3F002D21F121CA48E828F83C2
:10E85000A3A3A3A3A3A3A3A3E02212E7AEEEFCEF1E
:10E86000FDE508223400FB12153622E012E8702282
:10E87000F8A312DA2AA322E0F812E871A3A3A3A353
:10E880002212E889A3A3A3A32212E88D22E0F8A311
:10E89000E0F5838882A3A32212E89C2212E88DA3CC
:10E8A000A3A3A3A3A3A32212E09B750A00780822C6
:10E8B000F012E8B52212E72AE02274071208497F15
:10E8C000060205AD74F61203568C088D0912E91C78
:10E8D000850882850983120A9512DA47FAE5082429
:10E8E00004F8E5093400F9EA8882898312E6F6C360
:10E8F0009406500512E949801F74FE6A600574FF92
:10E900006A701612E949A312E75288828983E0F4FB
:10E91000700712E92DF0A3E9F002D21F12E8B5FE4C
:10E92000A3E0FF7904EEFAEFFB1214B2228E828F7D
:10E9300083E012E93CA3A3A3A3A3A322FAA3E0F9D3
:10E94000EA850882850983A322E0850882850983F8
:10E95000A3A3A3A3A32274F212035674F41208DB38
:10E960008A0C8B0D8C0A8D0B8908741A120AAC1252
:10E97000F5957C0C7D007900851082851183AA8233
:10E98000AB831214AC7409120AACE412EA8EA3A38E
:10E99000A3A3A3A3A3E0C0E07408120AACD0E0F0E4
:10E9A000850A82850B8312EB18F0901A86E024FF0B
:10E9B000F50AA3E034FFF50B850C82850D8312F474
:10E9C0008975091E780912081F780C12081B780A2D
:10E9D00012081B85080AE50A2401F50AE43400F54B
:10E9E0000B780A12081B8E0A8F0B780A12081B90EC
:10E9F00012B7E0F97C807D1A7409120AACAA82ABC6
:10EA0000831214587409120849740C02F78374F2C3
:10EA10001203568908740E120AAC12FA68741012A6
:10EA20000AAC12EBF9120AACE0F509901A8612F260
:10EA3000D4AE088023850A82850B83E0850C82850D
:10EA40000D8312EA8E85820A85830B850C82850DE3
:10EA500083A385820C85830DEEFF74FF2F1E047047
:10EA6000D4E5096005750A408003750A00E50A448B
:10EA70001E9012B7F0880A890B780A12081BA908A1
:10EA800012F2CE1208499012B7E4F002F786F08530
:10EA90000A82850B83A32274F412035674F71208BA
:10EAA000DB8A088B09890B8C0A901A8612F595ACC3
:10EAB00008AD097AE57B03121C9EE9700A740812FE
:10EAC0000AAC12EC6C800E7408120AAC7402F0905E
:10EAD00011E312EB18F0AC08AD09EEFAEFFB121CD3
:10EAE000A48A088B09AE08AF098E828F83E50BF0EC
:10EAF000A3E50AF0E4F508F509780812081B790A7D
:10EB00007402120AACAC82AD837A667B1212F2CE2A
:10EB1000120849740902F5AA12FA6C85108285114F
:10EB200083E8F0A3E9227402120AACAC82AD837AC6
:10EB3000667B1212F2CE1208497409800312F2CEDB
:10EB40001208497F020205AD74F01203568A0E8B3B
:10EB50000F8C088D09E9FE7410120AAC12EBF91241
:10EB60000AAC12F2D47414120AACE0FB7415120A47
:10EB7000AC12F58412FA65EE2BC3332406FAC39463
:10EB80004F40047910806F88828983E508F0A3E5FF
:10EB900009F0A3E50AF0A3E50BF0A3EE12EFEC6099
:10EBA000197F00EFC333F508E433F509E50C2508B8
:10EBB000F50AE50D12EBFF9E40E9EB88828983128E
:10EBC000EFEC60177F00EFC333F508E433F509EC91
:10EBD0002508F50AED12EBFF9B40EB750806750959
:10EBE00000780812081BEAF9AC0EAD0F7A667B12AA
:10EBF00012F2CE12084902F5D612F47874122235B8
:10EC000009F50B850A82F58312F60FA882A9838580
:10EC10000A82850B8312EC1C0FEFC322A312EC2196
:10EC20002212F60F08A9832274F612035674F71203
:10EC300008DBE9FE7408120AAC12EC6712EC7CEAFD
:10EC400012EC90EBF0901A86E02402FAA3E0340074
:10EC500012F5B2A3A3EEF075081375090078081237
:10EC6000081B790B02EB2612EC6CF022740FF08576
:10EC7000108285118374FDF0A374FF22901A86120E
:10EC8000EC832212EC8722E0F8A3E0F5838882224D
:10EC9000F012EC9522901A8612EC87A32274F012DF
:10ECA000035674EE1208DB7401120AAC12F5FD75FE
:10ECB0000A00750B007401120AACE0240CF50EA3D7
:10ECC000E03400F50F850E82F58312F84E70047C57
:10ECD0000880027C027401120AACE02413F8A3E05D
:10ECE0003400F97403120AAC12F8487403120AAC27
:10ECF00012EC7F12FA68E82CF582E912F5EBF50CBC
:10ED0000EA4B704D880A890BAC0AAD0B7AE57B03A0
:10ED1000121C9EE960099011E312F59502EDC3AA59
:10ED20000AAB0B120BA6EAF8EBF9EA4B700302EF01
:10ED30003688828983A3A3A3A3E06401600302EF62
:10ED4000368882898312F595E50C6077750CFF8013
:10ED50007288828983E0FAA3E0F9EA2400FEE439AC
:10ED6000FF9011E3E06E7003A3E06F7008750AE591
:10ED7000750B03804EEFFB120BA0EAF8EBF9EA4BA0
:10ED8000604188828983A3A3A3A3E06401703474E3
:10ED900005120AACE412F842A3A312FA6874101226
:10EDA0000AAC12F8487405120AACAA82AB83120BA3
:10EDB00064E9600B7408120AAC85820A85830BE54E
:10EDC0000C708974FE6E700374FF6F700302EF366F
:10EDD000E50A450B700302EF36901A8612F49A7515
:10EDE0000D0BE50C60177401650C60117402650C65
:10EDF000700E850E82850F8312F8547003E4800232
:10EE0000748085088285098312EF3BAC0AAD0BAA9A
:10EE100008AB09121CA4EE8A828B83F0A3EF12EFD9
:10EE20003B7401650C600302EF049011E3E06E7027
:10EE300003A3E06F600302EF04851082851183E471
:10EE4000F0AA82AB83120BC48A0A8B0BAC0AAD0BFF
:10EE5000850882850983A3A882A983EC4D700302EB
:10EE6000EEF9850E82850F8312F84E70047E0880BD
:10EE7000027E027403120AACE0FAA3E0F5838A82F0
:10EE8000E02EFAA3E034008A82F583A3E0FEC333C8
:10EE9000FAE433FBEC2AFAED3BFB85108285118303
:10EEA000E0FFEEC39F500CE0C39EF0C333240BF58C
:10EEB0000D8002E4F012EF4FEE8882898312EF3B5F
:10EEC000050D050D80218A828B8312EF448A828B87
:10EED00083A312EF44EA24020A0AEB3400FB8510F4
:10EEE00082851183E014F0851082851183E070D64D
:10EEF000ECFAEDFB12153C800B850882850983E452
:10EF0000F0750D0C9012B77410F0850E82850F838A
:10EF1000E0F508A3E04480F509780812081BA90D64
:10EF20007403120AAC12F1F7120AAC12F2031208BF
:10EF3000499012B7E4F0741202F5D3F0A385820869
:10EF40008583092212EF4FA385820885830922E079
:10EF5000850882850983F02274F6120356740A121A
:10EF60000AAC12F59512FA658882898312EFE412D1
:10EF7000EFEC8E828F83E0541F88828983F0A30890
:10EF800012F61BA312EFF312EFF4A312F00312F028
:10EF90000312F62112F6292408FCEF3400FD8C82BE
:10EFA0008D8312F6178C828D8312EFF312F62924CB
:10EFB0000B12FA5312F630240CF582EF12F5EB889F
:10EFC000828983F0750802750980780812081B7918
:10EFD00010EA2402FCEB3400FDEA240FFAEB3400C3
:10EFE000FB02EB3DE4F0A3ECF0A3ED22F0A3A8823A
:10EFF000A98322A312EFF82212EC218E828F83A321
:10F00000A3A32212EFF8A3A32274F6120356EAFE7A
:10F01000EBFF740A120AAC12F2DC12F1E912F79952
:10F0200012F7A78882898312F49A540FF9740C7826
:10F0300008120A4FE508C4498A828B83F0750803D9
:10F04000750980780812081B7905EE2402FCEF345C
:10F0500000FDEE240FFAEF808574F012035674FD64
:10F060001208DB7401120AAC12F5FDE985108285E5
:10F070001183F012F1E6EC2409F50CED3400F50DE6
:10F08000EC2406F50AED3400F50B8510828511831A
:10F09000E0702BEC4D6027850C82850D83C082C00B
:10F0A00083850A82850B83E0D083D082F8E028C371
:10F0B00033240CF9C3944F4007791002F1E379042B
:10F0C00085108285118312F64C9011E312F7AB90F4
:10F0D00011E412F63BE9C39405500302F1C574FC38
:10F0E00029F0A30A0AAB838C828D8312F7AB8C8242
:10F0F0008D83A3AE82AF8312F212EC2403FEED34B3
:10F1000000FF8E828F8312F2128C828D83A3A3A3C1
:10F11000A3A3E0C454F08A828B83F0A30AAB838557
:10F120000A82850B8312F7AB850A82850B83E06028
:10F13000427800EC2407F50EED3400F50F8027E847
:10F14000C333FEE433FF850E82850F83E02EF5087E
:10F15000A3E03F12F647850E82850F83E02EF50867
:10F16000A3E03F12F1ED850A82850B83E0FEE8C340
:10F170009E40CC850C82850D8312F64C850C8285D1
:10F180000D83E060427800EC240AFCED3400FDECD5
:10F19000FEEDFF850C82850D83E0FCE8C39C5027C3
:10F1A000E8C333FCE433FD8E828F83E02CF508A3A3
:10F1B000E03D12F6478E828F83E02CF508A3E03DF8
:10F1C00012F1ED80CEE4F07508047509807808121C
:10F1D000081B7403120AAC12F1F7120AAC12F20304
:10F1E00012084902F5D1901A8612F5CB22850882C1
:10F1F000F58312F21D0822E02402FCA3E03400FD96
:10F20000740322E0240FFAA3E03400FB12181874F0
:10F21000022212F21E8E828F8312F21D22A3E08A36
:10F22000828B83F0A30AAB832274F012035674FF1F
:10F230001208DBE9851082851183F0EAFEEBFF8C72
:10F240000E8D0F7411120AACE0F87412120AAC128F
:10F25000F5847414120AACE0F97415120AACE0F5E6
:10F2600008A312F5C1750C0474066E700374806FE8
:10F270007005750B108003750B00E88A828B831272
:10F28000EFE5F0A3E912F7A06017740429F50C75F7
:10F290000A0078081208178908AC0812F7B5120896
:10F2A00049E50B9012B7F08E088F09780812081BF9
:10F2B000A90CAC0EAD0F7402120AAC12F2CA1208FD
:10F2C000499012B7E4F00402F5D3AA82AB83121876
:10F2D00018740222E0F50CA3E0F50D2212FA6C90EE
:10F2E0001A862274F612035674FF1208DBE98510A1
:10F2F00082851183F0ECFE740B120AAC12FA68746A
:10F300000D120AAC12F49A12F337EEF012F337A38F
:10F31000E8F012F34312EC91A3A3E4F0780812088A
:10F320001B7904EAFCEBFD7402120AAC12F2CA1259
:10F330000849740102EB40901A86E0FCA3E0F583D3
:10F340008C822212EC95A3E9F02274F01203567419
:10F35000FC1208DB7402120AAC12F5FD7401120AE9
:10F36000ACE9F0ECFEEDFF7414120AAC12F49A74DE
:10F3700016120AACE0F50E7419120AACE0F50F9003
:10F380001A8612F478E50E250FC333240F851082F8
:10F39000851183F0C3944F4005791002F473120F66
:10F3A0006CEA6E7002EB6F6005790202F473EE8511
:10F3B0000A82850B83F0A3EF12F480120F66EAFC39
:10F3C000EBFDAA0AAB0B121CA47401120AAC12F6D4
:10F3D0003BE508F0A3E509F0A3E50E12F4807C00FC
:10F3E0008029ECC333FAE433FB7417120AACE02A29
:10F3F000FAA3E03BFB8A828B8312F4898A828B8397
:10F40000A312F60B85820A85830B0C850A82850B75
:10F4100083A3A882A983ECC3950E40C6850A828582
:10F420000B83E50FF0880A890B7C008023ECC33343
:10F43000F8E433F9741A120AACE028F8A3E039F9B9
:10F440008882898312F4A288828983A312F4A20C91
:10F45000ECC3950F40D7750820750900780812088D
:10F460001B7402120AACE0F97404120AAC12F59B88
:10F47000120849740402F5D3E0F50AA3E0F50B2263
:10F48000F0A385820A85830B2212F48D22E0850A7F
:10F4900082850B83F0223400F583E0F508A3E0F5C4
:10F4A000092212F48DA385820A85830B2274F0123F
:10F4B000035674FD1208DB7401120AACECF0A3EDE4
:10F4C000F0E9851082851183F08A088B0974131284
:10F4D0000AAC12F5847415120AAC12F59574171261
:10F4E0000AAC12F4787419120AACE0F50F12F1E6C6
:10F4F000750E0C850A82850B83A3A3A3A3A3A3A3E4
:10F50000A3E0F87403687005750E1580087401682F
:10F510007003750E0E121CA412F635EEF0A3EF1256
:10F52000F7A0850A82850B83A3A3A3A3A3A3A3A308
:10F5300012F58AA3A3A3A3A3A3A3E0F8740368709E
:10F540000FAC0AAD0B121CA48A828B83E50F8013CB
:10F55000740168700F850A82850B8312F58AE08A30
:10F56000828B83F09012B77410F0780812081BA9F0
:10F570000E7403120AAC12F59B1208499012B7E4FC
:10F58000F002F5D1E0FCA3E0FD2212F21E850A8212
:10F59000850B83A322E0FEA3E0FF22E0FCA3E0FDB5
:10F5A0007A667B121218187402221208497F04022C
:10F5B00005ADFB121CA412EC95A3A3A3A3A3A3A3C4
:10F5C00022E0F50912F5C822901A86E0FAA3E0FBC2
:10F5D0002274031208497F080205AD3400F98882BD
:10F5E000898322E50E2410F582E50F3400F583E0CF
:10F5F00022F02401FAE43400FB12153622EAF0A3CB
:10F60000EBF022EAF0A3EBF074022212F60F22E0F4
:10F6100088828983F0A32212EC1D22A9838E828F17
:10F620008312EC1C8E828F8322A3A3A3A3A3A3A384
:10F6300012EC1DEE2285108285118312F63F22E026
:10F640008A828B83F0A322850882F58312F63FAA73
:10F6500082AB832274F212035674F61208DB74052F
:10F66000120AACE9F07408120AAC12F5FD74041227
:10F670000AACECF0ED851082851183F07418120A43
:10F68000AC7808120A6D741C120AAC12F2D4741E03
:10F69000120AAC12F595851082851183E0240AC008
:10F6A000E07401120AACD0E012F5F17402120AAC57
:10F6B00012F603120AAC12F8547005791002F781A1
:10F6C0007402120AACE0240108A3E03400F97406C5
:10F6D000120AAC12F8487406120AAC12F1E974046A
:10F6E000120AAC12F64C780812081312151874049A
:10F6F0001208498A828B83E50CF0A3E50DF0A3EE96
:10F70000F0A3EF12F7A085108285118312F7AB8565
:10F710001082851183E0601B7420120AAC12F49AE7
:10F72000750A0078081208177403120AAC12F7AFB2
:10F730001208497406120AAC12F2DC12F84874225C
:10F74000120AACE09012B7F0750838750980780895
:10F7500012081B7403120AACE0F9740A120AAC1204
:10F76000F5847407120AAC12F2CA120849E9FE7451
:10F7700002120AAC12F1E912F78B9012B7E4F0EE24
:10F78000F9740A1208497F060205AD12153C901A59
:10F79000867468F0A37412F0228A828B8312EFE4DD
:10F7A000F0A3AA82AB83228882898312F21E22E010
:10F7B000FC12F7B5227D001214A074032274F21219
:10F7C0000356890AEAFEEBFF9012B8800888088980
:10F7D000098882898312F854601F88828983A3A3D1
:10F7E000E0650A70E888828983A3A3A3E06E7003B2
:10F7F000A3E06F70D8790080467A057B0012153639
:10F800008A0C8B0DA80CA90DE84960318882898388
:10F81000A3A3E50A12F842A3A3A3EEF0A3EF12F804
:10F8200042E4F0A3F09012B812F84E600B85088203
:10F8300085098312F84880BD9012B880F6791002CD
:10F84000F786F08882898322E8F0A3E9F02212F596
:10F85000CBEA4B2212FA6CE8492274F01203568A62
:10F860000E8B0F7508009012B802F911850C828575
:10F870000D83A3A3A312FA68E50E240C12F5E76822
:10F880007003A3E069600302F90B12F5E32415FA93
:10F89000E43400FB1214C48A0A8B0BAE0AAF0BEEE1
:10F8A0004F6068850E08850F09750A0078081208F0
:10F8B000177C1512F7B512084912F5E36032EE24F1
:10F8C00015FAEF3400FBEE241312FA5312F5FDE59E
:10F8D0000E2413F582E50F12F4967808120817E546
:10F8E0000E2410F582E50F12FA5612F7AF120849EE
:10F8F0008E828F8374D3F0EEFAEFFB850C82850D38
:10F9000083A3A3E0F91214D0750801850C82850D3C
:10F910008312F2D4E50C450D600302F86CA90802CD
:10F92000F5D674F612035674EB1208DB7E00740AE7
:10F93000120AAC740212FA5BA3A312FA68740212E0
:10F940000AAC12F848EA2415F582EB12F5EBC0E098
:10F95000740B120AACD0E012FA5B12FA68740C1243
:10F960000AAC12F848EA2419F582EB12F5EBC0E074
:10F97000740E120AACD0E0F0EA241FF582EB12F507
:10F98000EB14C0E07410120AACD0E0F0EA2421F8C5
:10F99000EB12F5DBE02401FCA3E03400FD7413124C
:10F9A0000AACECF0A3ED12F84212EC7FE0C0E07478
:10F9B0000F120AACD0E0F0EA2412F582EB12FA56EC
:10F9C00012FA687411120AAC12F848851082851177
:10F9D00083AA82AB83121872E9FC80010E8E08752F
:10F9E0000900740278081209DA74262508F87421CF
:10F9F0003509F988828983E493C0E0740193F58323
:10FA0000D082AA82AB8374FF6A700374FF6B602E8E
:10FA1000740C120AACE06A7003A3E06B70BE851030
:10FA200082851183AA82AB8388828983A3A3E4930E
:10FA3000C0E0740193F583D082121E778010EC70C1
:10FA40000D851082851183AA82AB8312171074155D
:10FA500002EB40F582EF3400F58322F08A828B833B
:10FA6000A3A3A3A322901A8612FA6C22E0F8A3E0C3
:10FA7000F922C082C083E9F87402686009740368DF
:10FA8000600879E8803C7B1880027B0CEBC39A50BD
:10FA90000679E8EBFA80027900906180E0D2E0F02C
:10FAA000906189E0D2E5F0906182E0D2E0F0E0D2AE
:10FAB000E1F09015707401F0EA901571F0E8901A79
:10FAC000A6F002FD9F74F012035674EF1208DB7467
:10FAD00001120AACEAF0A3EBF0ECFEEDFF740112A8
:10FAE0000AACE0F8A3E0F9E849601C7401120AAC22
:10FAF000A3E0F5838882A3A3A3A3A3A3A3A3E0F811
:10FB0000901AA6E068600579E802FD117401120AF6
:10FB1000ACE0FA121A2EE9F46005791E02FD11120A
:10FB20001A3A740D120AAC120A95901AA6E06402F1
:10FB30008510828511837041E412FD29507E740D79
:10FB4000120AACC082C08375080175090085108255
:10FB5000851183E078081209DA12FEDED083D082A4
:10FB6000780812097BE5084509450A450B6063855D
:10FB70001082851183E00480C0E4803B740D120A7A
:10FB8000ACC082C08375080175090085108285119B
:10FB900083E0C33378081209DA12FEDED083D08204
:10FBA000780812097BE5084509450A450B6073850D
:10FBB0001082851183E00412FD2940C0E0F8901501
:10FBC00071E0687005791A02FD11901AA6E06402CE
:10FBD00070507406120AACEEF07407120AACEFF023
:10FBE0007401120AAC12FEE8E0C0E07408120AAC1C
:10FBF000D0E0F07401120AAC12FEE8A3E0C0E07499
:10FC000009120AACD0E0F079047406120AACAC8296
:10FC1000AD83851082851183E0F5087509007402B3
:10FC2000801A79087401120AACE0FCA3E0FD85108B
:10FC300082851183E0F508750900740378081209BC
:10FC4000DA2508FA74613509FB121B06901AA6E042
:10FC500064027903700D740A120AACAC82AD837A27
:10FC600067800B740A120AACAC82AD837A647B6144
:10FC7000121B0C7903740A120AACAA82AB83121409
:10FC8000B28A088B098C0A8D0B901AA6E064027563
:10FC90000C01750D008510828511837030E0780CA1
:10FCA0001209DA12FD1B1209C7780812081374072B
:10FCB000120AACAA82AB8312151E74041208497989
:10FCC00003E9120AACAC82AD837A678030E0C333BB
:10FCD000780C1209DA12FD1B1209C77808120813F2
:10FCE0007407120AACAA82AB8312151E74041208A0
:10FCF000497903E9120AACAC82AD837A647B611264
:10FD00001B067A01851082851183E0F9121A347975
:10FD10000074111208497F080205ADE50D3395E026
:10FD2000F50EF50F7808790C22F0901571E0F88542
:10FD30001082851183E0C39822C082C083EA4B60A1
:10FD4000158A828B83A3A3A3A3A3A3A3A3E0F89004
:10FD50001AA6E068600479E8800F121A2E74FF6911
:10FD600060F47A00121A3479008034C082C083743F
:10FD70000169901572700B7401F090618AE0D2E213
:10FD80008008E4F090618AE0C2E2F08012C082C094
:10FD900083901572E06401700479FE800279FFD0CF
:10FDA00083D082020533C082C083901572E0600464
:10FDB00079018009906163E0F8744058F980E0743B
:10FDC000F012035674F11208DB901AA6E064027078
:10FDD000447403120AACECF07404120AACEDF08A1D
:10FDE000828B83E0C0E07405120AACD0E0F08A8216
:10FDF0008B83A3E0C0E07406120AACD0E0F0740379
:10FE0000120AACA882A9837401120AACE8F0A3E933
:10FE1000F07F04800C7401120AACEAF0A3EBF07FCF
:10FE2000087E0080010E901571E0F8EEC398400343
:10FE300002FED7EE851082851183F0901AA6E06449
:10FE400003700A851082851183E0C333F0121A3AD9
:10FE50008A0C8B0D8C0E8D0F7508017509008510AD
:10FE600082851183E078081209DA12FEDE780C79B7
:10FE700008120968E50C450D450E450F60A7EFF91E
:10FE80007407120AACAC82AD83EE89F0A4FAA8F034
:10FE9000E428FB74613BFB121B0C7407120AACA92B
:10FEA00082AA8389088A09750A0078081208178FC0
:10FEB00008AC087D007404120AAC12FEE8A982AAFC
:10FEC000837B001214A67403120849E964016003DD
:10FED00002FE25EEF9800279FF740F02FD13E50999
:10FEE0003395E0F50AF50B22E0F8A3E0F58388826C
:10FEF0002274F0120356E9FEEAFF121A3A8A088BBE
:10FF0000098C0A8D0B750E01750F00EEC333780E48
:10FF10001209DA850E0C850F0D750E01F50FEE78BE
:10FF20000E1209DAA80EA90F046F901AA67021E02C
:10FF300064027014880CE9F50D12FD1D1209C778D2
:10FF4000081208137A83803512FD1B1209C7802618
:10FF5000E064027010E8F4F50CE9F4F50D12FD1DF3
:10FF600012096880DAE50CF4F8E50DF4880CF50D5B
:10FF700012FD1D12096878081208137A867B611237
:10FF8000151E740402FD13C082C08374FD1208DBC9
:10FF9000901AA6E064027903851082851183AC82F1
:10FFA000AD8370047A8380027A867B61121B0C79A0
:10FFB00003851082851183AA82AB831214B2740365
:10FFC00012084902FD9F74F7120356EAF8EBF98014
:10FFD00005A3AA82AB838A828B83E070F48C828D26
:10FFE00083E0A3AC82AD838A828B83F0A3AA82AB29
:0CFFF0008370EAE8FAE9FB7F010205AD2E
:020000040001F9
:1000000088828983A3E01313543F540322F582EBC3
:1000100012A8FDA2E2229004081296F51211A6225F
:10002000E0F508750900750A00750B0022740912C5
:1000300008497F040205AD12A209EF12A8FDA2E54E
:100040002234FFF5832212B3ACE82290047DE0FA5B
:10005000900462E022EE2412FAEF3400FB12133E09
:10006000E922790512134A740222E0FAA3E0F9EAC0
:100070002274021208497F060205ADF0900462E086
:10008000640F2212142E90048212B3AC7A147B00F7
:1000900022C082C083900408E07002A3E0600312D3
:1000A0008B8E9004051294667408900407F09004F7
:1000B00008E4F0A3F0900458F090040A028D27742D
:1000C000F712035674F71208DBEAFEEBFF1288D131
:1000D00074051296077403F0EE24020A0A12816B6B
:1000E00012822F8A828B8312A6F7EE2421FCEF3432
:1000F00000FD8C828D8312A212128171600BEE249E
:100100001F1288D474FFF0A3F0EE241FEF34001CFC
:100110001CFD8C828D83A3E0C0E0129287D0E01298
:10012000817188828983F074038E828F83A3A3A355
:10013000A312A6DC851082851183AA82AB83121CD0
:10014000A47408120AAC7403F090047712069D742C
:1001500002120AACAC82AD831295DD120849E97037
:1001600007EEFAEFFB12123C028869EF3400029EA0
:10017000AF12A21612A3618C828D83E02274F0125A
:100180000356EAFEEBFF890C7410120AAC1296F1CA
:100190007412120AAC12823DEE2402F508EF34000C
:1001A000F509850882F58312822FEB128245EA1247
:1001B0008257E50C12824990047CE012824590043B
:1001C0007BE0128257E50B12825BE50AF0E8FA85C4
:1001D0000882850983E0C39A8E828F83A3A3A3A399
:1001E000F085088285098312A6F78C828D83A3A3EC
:1001F000A3A3A3A3A3A3E0640370071288D174018F
:100200008009EE240EF582EF129BE812960774091E
:10021000F07508FF7509FF780812081B1295DD12AA
:100220000849E97007EEFAEFFB12123C028604124D
:10023000823322E024FFF8A3E034FFF922E0F50A3C
:10024000A3E0F50B228882898312824D22F0E824F4
:10025000FF18E934FFF9228882898312824D88824F
:1002600089832274F01203568A088B09890A8C0E3E
:100270008D0F750C00A2AFE492E0F50BC2AF9004B5
:100280000B803C12833C50341283426403702DE592
:100290000824F9F508E50934FFF5098E828F83A358
:1002A000A3E02405FCA3E03400FDAA08AB09121C5E
:1002B000A412835D7410250CF50C150A1287071221
:1002C000B064E50A6006EE7001EF70B7E50BA2E0DE
:1002D00092AFA2AFE492E0F50BC2AF90040B80198D
:1002E0002402FA12816B12918012834C12928712AF
:1002F000834C050C150A12870712896C7001EF6098
:100300001F128342640270EE12833CEE40D21280D0
:100310003750E37401850E82850F83F0E50A70D6AD
:10032000E50BA2E092AF850882850983E50CF0E534
:100330000824FFFAE50934FFFB028604128559A25E
:10034000E6228E828F8312928F028004A3A3A3A33E
:10035000A3E0850882850983F012835D22E50824E5
:10036000FFF508E50934FFF5092274F0120356740D
:10037000F51208DB7401120AACE9F08A0F8B0EE467
:10038000851082851183F0900411E0C39408400524
:10039000750B078003E0F50BE50B33333354F8900E
:1003A0000461FAE02A2433FEFA7B001214C48A0C9A
:1003B0008B0DEA7001EB70030284B812A6E790047B
:1003C00061E0FAFCC3E49CFCE49400FDE82CFEE947
:1003D0003DFF90045F1284D37808120817EA12B028
:1003E00058120849851082851183AC82AD83A90B10
:1003F000EE24FFFAEF34FFFB1211528A088B09AE8C
:1004000008AF09E41284DFE50EC454F0C0E09004A4
:1004100059E0C4333354C0C0E090045BE0A2E0E490
:1004200092E013135480FAD0E04AFAD0E04A440F25
:1004300012A23C120AACE50FC454F0FAE04A8E82D4
:100440008F83F0EEFA850C82850D83A3A3E0C39A17
:10045000850C82850D83A3A3A3A3F0850C82850D53
:1004600083A3A3EEF0A3EFF0E50C240E1284C9E5FC
:100470000C240D1284C9740A120AACE4F0F508F5D4
:1004800009780812081B7404120AACAE82AF8312FA
:10049000132CEEFCEFFDAA0CAB0D1295E3120849EC
:1004A000851082851183E06009850C82850D831299
:1004B0008611AA0CAB0D80047A007B00740B8003BC
:1004C0001294E1120849028604F582E50D12961293
:1004D000E4F022E0F508A3E0F509750A0022E08EB9
:1004E000828F831284E722F01284EC22EE24FF1E16
:1004F000EF34FFFF2274F21203568A0C8B0DA2AF69
:10050000E492E0F50AC2AF75080075090090040B8B
:100510008024128710501C850C82850D8312856201
:100520001296EB121332E9600A128555C2E6F08E7C
:10053000088F0912870712896C7001EF70D4E508E3
:100540007002E509600612926FD2E6F0E50AA2E0B9
:1005500092AF02807612855922EE12A2E9EF12A222
:100560005522A3A3E0FCA3E0FD2274F01203568AF7
:100570000E8B0F8C0C8D0D750800A2AFE492E0F588
:1005800009C2AF7E007F0090040B8019AE0AAF0B4A
:10059000128609128FEFD2E7F0E50A24FBF582E517
:1005A0000B34FFF58312823DE50A7002E50B6037DC
:1005B00012A2DDA2E750E2850A82850B83A3A31273
:1005C000069DAC0CAD0DAA0EAB0F121338740212BF
:1005D0000849E960C4EE7001EF60B11289607007EC
:1005E0008E828F83128611E509A2E092AFEE700130
:1005F000EF6006121236750801A9088007EEFAEFBF
:10060000FB12141C7F080205AD128559D2E4F0EEEE
:100610002212928FE0D2E4F02274F212035674FE9A
:100620001208DB750C00750D00851082851183E4BE
:10063000F0A3F0A2AF92E0F50AC2AF90040B12B0A3
:1006400064802C12870712927A780C12081B12868B
:10065000F5120849EEFCEFFD851082851183AA8210
:10066000AB831214DCAE08AF09900411E014F0EE75
:100670007001EF60271287105019EE240B128F566D
:1006800024FFF0A3E034FFF088828983E07002A3A6
:10069000E060B08E0C8F0D12870780A2E50AA2E001
:1006A00092AF900411E0602F900462E0640F600646
:1006B000900458E070217AFF7B0312142E90876318
:1006C0001206997AFF7B031294E1120849800812FE
:1006D000115E74F0129319851082851183AA82AB82
:1006E000831214E28A088B09AE08AF09EE7001EF9D
:1006F00070DD028071EEFCEFFD7A0B7B041214EECC
:100700007402228E0A8F0BEE24FBF582EF028041E9
:10071000128559A2E72274F7120356EAFEEBFF1284
:10072000115E901A6212928B121E77E96401900496
:100730007E700AE02401F8A3E034008004E0F8A30E
:10074000E0F9EE240B1288D412A6F7900411E070A1
:100750001F900462E0640F70177AFF7B0312142E5F
:100760009087631206997AFF7B031294E11208497D
:10077000A2AFE492E0FAC2AF9004111287CB0297C5
:100780004A74F7120356EAFEEBFF1287BAF0121111
:100790005EEEFCEFFD7A0B7B041214E8A2AFE4924C
:1007A000E0FAC2AF9004111287CB900462E0640FAC
:1007B000700579081212EA02974A128559C2E4229A
:1007C000A2AFE492E0FAC2AF900412E004F0EAA211
:1007D000E092AF2274F712035674EA1208DBEAFEC5
:1007E000EBFF90045BE0602A740185108285118321
:1007F000F0120AACE4128871120AAC128816C0E03A
:10080000740A120AACD0E012A59A740B120AAC1248
:10081000994A74168055AA82AB83121CA48E828FCB
:1008200083A3A3129291E022C082C08312114602D8
:1008300093B874F712035674EB1208DBEAFEEBFF71
:100840007406851082851183128871120AACAA82FF
:10085000AB83121CA4EE2407FCEF3400FD740A12D3
:100860000AAC12994A741580027409120849029759
:100870004AF0128C5374022274F712035674F71262
:1008800008DBEAFEEBFFEE2421128FF1604112A695
:10089000E1851082851183AA82AB83121CA474089F
:1008A000120AAC7403F090047712069DEE241F1216
:1008B00088D412069D90048AE0F97404120AACAC44
:1008C00082AD83EEFAEFFB12114C740412084980DA
:1008D00098EE240EF582EF1296122274F21203564D
:1008E0008A0C8B0D750A00750B007508E7A2AFE442
:1008F00092E0F509C2AF90040B80031287031289BE
:100900006C7001EF602F12871050F012896070EB4D
:10091000EE242EF582EF12A92A850C828B83A3A3E5
:10092000E06A70D7780A12081B1286F512084990FF
:100930000411E014F0E509A2E092AFEE7001EF605F
:1009400013EEFAEFFB12115E79F0EEFAEFFB1212E2
:10095000F0750800A908AA0CAB0D1212F0028076FF
:10096000EE240DF582EF12A8FD640122E0FEA3E063
:10097000FFEE2274F412035674F71208DBEAFEEB62
:10098000FF1211A0E9F508704FEE240E128FF160EE
:10099000477A0079091211E8EA7001EB603A7408AD
:1009A000120AAC12AE85128B4212069D7508FF75B5
:1009B00009FF780812081B8E828F83A3A3A3A3A329
:1009C000A3A3A3E0F97404120AACAC82AD831211A4
:1009D0004C7404120849800D8E828F83A3E508129F
:1009E00093251211AC02802D74F1120356EAFEEB2E
:1009F000FF7508008E828F83A3A3A3A3A3A3A3A341
:100A0000E0C3940B40128E828F83A3A3A3A3A3A35E
:100A1000A3A3E0C3941D40037508E88E828F83A3CF
:100A2000A3A3A3A3A3A3A3A3A3E0C394104005750A
:100A300008E880138E828F83A3A3A3A3A3A3A3A3F9
:100A4000A3A3E0640F600B90042FE05408700375BB
:100A500008E88E828F83A3A3A3A3A3A3A3A3A3A326
:100A6000E0C0E0EE240BF582EF12A92AD0E0C39A91
:100A70005008E0640F60037508E890047BE064FFB1
:100A80007004A3E064FF70037508EC7A237B001206
:100A90001536900408129E33900408E07002A3E01B
:100AA00060288E828F83A3A3A982AA83890C8A0DD2
:100AB000750E00780C1208177C237D009004081234
:100AC00096F1129CD6120849800375081AA9087F6E
:100AD000070205AD74F7120356EAFEEBFF8E828F14
:100AE00083A3A3A3A3A3A3A3A3E090046212ADAF27
:100AF00090047DF0EE240B128FF190045D128B4276
:100B0000A3A3A3A3E0900459F0F9121B3090045959
:100B1000E0600CEE24041295E9EE2406128B377483
:100B20000190045812807B60047A0180027A00EA06
:100B300090040AF002974AFAEF3400FB79E11213AD
:100B4000C222128B462212984BA3A3A3A3A3227402
:100B5000F7120356EAFEEBFF8E828F83A3E0700349
:100B600012801612AE8F02974A74F7120356EAFEED
:100B7000EBFF900408E07002A3E0600A128B8E90F5
:100B80000408E4F0A3F07408128F5D02974A900401
:100B9000081296F512153C2274F61203569004586A
:100BA000E0601290040AE0700C128BB8EA7001EB5E
:100BB000600312123C029A0F90045DE0FB12804B1E
:100BC000F91211582274F712035674FA1208DBEA6C
:100BD000FEEBFF8E828F83A3A3A3A3A3A3E0A2E2D5
:100BE000506CEE242A1288D4128564EE2412FAEF97
:100BF0003400FB121164E9705590875EE064017067
:100C000032EE241A129601702A7410851082851112
:100C100083F0EE241212B3A27402120AAC12A6F7E9
:100C2000EE242A12B3A27404120AACE8F0A312B1A3
:100C30008F801B12132CE9FAEE242A1288D4120694
:100C40009D7B30128C53790112806412084974061E
:100C500002886BEE2412FCEF3400FD22C082C083B8
:100C6000900459E0600312139E0293B8C082C083BF
:100C70009004507493F0A37422F0900452740FF017
:100C8000A37422F0900454747DF0A37422F0901A9F
:100C90006E74C5F0A3741FF090043A7440F0A3740E
:100CA00011F0901A587470F0A37411F0901A5A74DD
:100CB00076F0A37411F090042FE04402028D24C05A
:100CC00082C08312A92079030299D4C082C0831202
:100CD000A92079050299D4C082C083790802A9BFEE
:100CE000C082C083800A7A0B7B041214E21214CAF9
:100CF00090040BE07002A3E070EC90040DE0700231
:100D0000A3E0600C7A0D7B041214E21214CA80EA8C
:100D100090040BE4F0A3F0900411F0900412F09012
:100D200004138003F0A3E0F00293B874F4120356A6
:100D30008908E92432F582E43422F583E493FEFA4B
:100D40007B001214C4EA7001EB600F12A6E7E48A7C
:100D5000828B83A3A3A3A3F080297A027B001214C1
:100D6000C4EA7001EB6018E5082453F582E43422EC
:100D7000F583E4938A828B83F0741AA31290B07A7D
:100D8000007B00028032C008740629FBEAA2E05012
:100D90001EEB75F00A84AAF0EA6014740A2BC39A59
:100DA000FBEAC394054004740A2BFB740B2BFBE98C
:100DB000C394134004781480027806E82BFB8B0858
:100DC00074092508F8E43400F97A0A7B0012020558
:100DD000E8F9D008020533C082C08390042FE054A4
:100DE00002600A121D04E9600479018002790002A0
:100DF00093B8C082C08390042FE05402601990041D
:100E000011E0700F900414E07002A3E06009128EEC
:100E10001C50047901800279000293B8900414E018
:100E200024101292A9A2E722C082C083900413E08A
:100E3000C0E090875CE0FCD0E0C39C50051214C475
:100E400080047A007B000293B8C082C0831214CA67
:100E50000293B874F6120356EAFEEBFF8E828F837C
:100E6000A3A3A3A3A3E01206320003488F758EC785
:100E70008E488FD88E900462E0640F60131212FCCB
:100E8000E9700DEEFAEFFB901A5C12928B121E774E
:100E900090048AE08E828F83A3A3A3A3A3A3F074FC
:100EA000148E828F83F0EEFCEFFD7A0D7B0412141A
:100EB000DCA2AFE492E0FAC2AF9004131287CB79C0
:100EC000201212EA029A0F1212F6E96007740D124C
:100ED0008F5D80F0741580C98E828F83A3A3A3A336
:100EE000E060658E828F83A3A3A3A314F0EE240297
:100EF000EF34000A0AFB8A828B83128046FCE9FDEC
:100F00008C828D83E0F508EE2405F8EF128F52E510
:100F10000812ACB5A882A9838A828B8312A6F7E552
:100F20000860258E828F83A3A3A3A3A3E0C3940AA2
:100F30005016EE2405128F56240A8E828F83F08875
:100F4000828983E004028EA5EEFAEFFB1214CA0236
:100F50008EC412A56F22F8EF12A56FE0228E828F49
:100F600083129325121CFE22C082C083900416E0D7
:100F70007002A3E0600B90041612928B121E778011
:100F80000279000293B874F7120356EAFEEBFFEE03
:100F9000240D1288D47401F0EE242F128FF1C0E0DA
:100FA0001288D1D0E0F0EE2430128FF1C0E0EE24B0
:100FB000121288D4D0E012A592C0E0EE2413128859
:100FC000D4D0E0F0EE242B1288D412069DEE242219
:100FD000FCEF3400FDEE242D128FF1F91295E3128F
:100FE0000849E97007EEFAEFFB12123C02974A2417
:100FF0000FF582EF12A8FD22C082C0831212FCE915
:1010000060047920800279010293B8C082C083EA2B
:1010100012A221E0D2E0028D27C082C08312A21A60
:1010200012896670111290A5400C8A828B83A3E00E
:10103000F91212F0806CEA12A209EB128FF4A2E608
:1010400050128A828B83A3E0F9901A5E12928B125F
:101050001E77804E12A21A12896670091290A5504E
:1010600004743080368A828B83A3E0641B7004741E
:101070002280288A828B83A3E0700F12A21A128F1B
:10108000F4245EF582E43422800D12A21A128FF449
:101090002453F582E43422F583E4938A828B83120D
:1010A00090B00293B8EA12A209EB12A8FDA2E322C3
:1010B000F090042CE0F91214D022C082C083900476
:1010C00014E07002A3E06043E9700612917DE480B1
:1010D0001A741B697038900414E0240DFAA3E0120E
:1010E000816CE0640570E412917DE9129186121220
:1010F0002A900414E0240E128E22500312A9AE90FE
:101100000414E4F0A3F079101212EA0293B874E91F
:1011100069704990041412A55DE09004146036E0F3
:10112000240E181818129179A2E2900414E0400FCE
:10113000241108080812917914F0121C5080CC2454
:101140000F08129179C2E7129186901A5A12928B67
:10115000121E77809C12918074E9808F741C6970D4
:10116000869004141296F1901A6412928B121E77D4
:10117000900414E4F0A3F080921292AA2290041436
:10118000E0129292A322F09004141296F52274F4C5
:10119000120356750A00750B00A2AFE492E0FEC27E
:1011A000AF900414E07002A3E06008EEA2E092AFFA
:1011B000029267901A6212928B121E77E94410FA1B
:1011C00090040B801285080A85090BE50824FBF5BD
:1011D00082E50934FFF58312927AE5087002E50989
:1011E00060C912926F5A6A70DC780A12081BAC0848
:1011F000AD091286F9120849900414E508F0A3E538
:1012000009F0128E1C4063900412E014F0EEA2E08C
:1012100092AF900414E0240E1818A3E03400F9E80B
:10122000FEE9FF8E828F83E0FA12929AF91211EE94
:10123000E990040FF0A3E412A236E0A2E750189060
:101240000414E02412129282121B54900414E0241D
:1012500013129282121B489004141292A2A2E1B3BC
:10126000E492E0F9121C38028032900411809BE570
:101270000812A2E9E50912A8FD22E0F508A3E0F5AD
:1012800009221292A9F9228A828B8312929122A3B7
:10129000A3E0F8A3E0F583888222900414129977E2
:1012A000E022E0240F1292A922F812A569E022742C
:1012B000F7120356EAFEEBFF121320EE12A209EF1B
:1012C0001290AA400A128960700590875A80039094
:1012D000875BE0F9EEFCEFFD7A0B7B041214F4E976
:1012E000602FEEFAEFFB901A6012928B121E77EECF
:1012F000240EF582EF12801040081287C0121236B9
:101300008014EEFAEFFB901A5812928B121E77801F
:101310000574F112931902974A8E828F83A3129358
:101320002512122A22F0EEFAEFFB22C082C08312AD
:1013300012360293B874F7120356EAFEEBFF7508F3
:101340000090042FE05402700EEE242FF582EF126D
:10135000801050037508E890042FE05460700DEE83
:10136000242F128FF1A2E150037508E88E828F833B
:10137000A3A3A3A3E0C3947540037508E8EE242D4E
:10138000128FF1701AEE242A128FF170127508F57F
:10139000121320A908EEFAEFFB1212F002974AE5A9
:1013A0000870ED12121880F4C082C083740D8A8216
:1013B0008B83F0121CFE8000D083D082020533C0E4
:1013C00082C083E48A828B83F0A3F0EA242F128008
:1013D0000D4018900412E0C0E090875AE0FCD0E085
:1013E000C39C401879F11212F080CD900411E0C036
:1013F000E090875AE0FCD0E0C39C50E81290B180A6
:10140000E874F4120356E9FFEA2485F582E43422F5
:10141000F583E493244AFE8F0A250AFAE43400FB9C
:101420001214C4EA7001EB600FEF8A828B83A3A3CE
:10143000A3A3F012A6E780047A007B00028032C0EA
:1014400082C083E490042AF090042BF090041E12D2
:1014500094667402900420F090042712946674013C
:10146000900429028D2774EAF0A37412F022C0823E
:10147000C08374F11208DB7402851082851183F039
:101480007401120AACE9F060047AFF7BFF74021267
:101490000AACEAF0A3EB12B190740F80027411123F
:1014A00008490293B8C082C08374FE1208DB740A34
:1014B000851082851183F07401120AAC12B18F7409
:1014C0000280DC74F012035612AF1B120A6D78080A
:1014D000790C12026678081208137A217B040284C0
:1014E000C012142274042274F412035674CE12082B
:1014F000DB900462E0640F6007742E129E39802333
:101500007A187B0412808312020D88088909750AF3
:1015100000750B0078081208137A187B041294E106
:10152000120849743202802F74F7120356EAFEEB58
:10153000FF7A001295FE6007E0640360027AE8EE2D
:101540002417128FF1C3940B4028E0C3941D50223E
:10155000EA7021EE2417128B37EE24221295E9123D
:1015600095FE7026EE241912B3A290047112A6F70C
:10157000802B7AE8EA8E828F83A3F074178E828F95
:1015800083F0EEFA12130202974A90047174FEF08F
:10159000A374FFF0EE24191295F4121CA490042AEF
:1015A000E04401C0E01288D1D0E012960774021224
:1015B000A34A242412A33624221288D412069DEEB4
:1015C0002419FCEF3400FD79831A1A1295E11208F0
:1015D00049E970B3EEFAEFFB12123C80AA7903EEF0
:1015E000FAEFFB121344740222FAEF3400FB795035
:1015F0001213C222FCEF3400FD7A687B0422EE2431
:101600002112A8FA640222F0EE240D12960F22F5A0
:1016100082EF3400F58322C082C08374F71208DBA6
:1016200090042BE070327401F0F9121C02851082D4
:10163000851183AA82AB8312132690047712069D2C
:1016400090042AE04401FB7402120AACAC82AD8320
:101650007A03128062120849740902949F74F71287
:10166000035612982F700474EBA3F090042BE0A2A1
:10167000E25003C2E2F0E0A2E1500512984080057A
:10168000742A12AE9102974A74F712035674FE122E
:1016900008DB12974F12995F85108285118312998A
:1016A00081E0F5087017851082851183AA82AB83CB
:1016B00079531213C2EE2412FAEF12B0F1851082A0
:1016C0008511831296F1A90812126690042BE0A2EC
:1016D000E1500A8E828F83A3E0F912126CE4900429
:1016E0002AF090042BF0740202886B8E828F83A301
:1016F000A31296F522E0FAA3E0FB2274F712035638
:10170000EAFEEBFF74EB8E828F83A3F090042BE054
:10171000A2E1500579EB12126CEEFAEFFB12129C6B
:10172000802874F712035612974FE490042AF09021
:10173000042BF07AFF7BFF8E828F83A3E0F91212D5
:10174000668007EEFAEFFB1213927F010205ADEA05
:10175000FEEBFF7901121C087A187B0412142E7A12
:10176000217B0412142E2274F7120356EAFEEBFFBB
:1017700012129680CE74F7120356EAFEEBFF79013F
:10178000121C088E828F83A3A3A3A3E060047A00B7
:1017900080027AEB1297C05003C2E2F0E0A2E1505F
:1017A000051298408011A2E0500D742A8E828F831A
:1017B000F074EBA312AE95EEFAEFFB12124E808A94
:1017C000EA8E828F83A3F090042BE0A2E22274F7CA
:1017D000120356EAFEEBFF90042BE0D2E1F0790110
:1017E000121C02EE240B1288D412069DEE2402EF86
:1017F0003400FF0E0E7401C0E012132CE9FAD0E0A1
:10180000FBEEFCEFFD12806202886B74F712035648
:1018100012982F700474EBA3F090042BE0A2E25016
:1018200003C2E2F0E0A2E1500312984002974AEAB4
:10183000FEEBFF7901121C088E828F83E064202268
:10184000C2E112984BE0F912126C22F08E828F8363
:10185000A32274F7120356EAFEEBFF7901121C086B
:101860007A187B0412B2EFE060047A0080027AEB0F
:101870001297C05003C2E2F0E0A2E1500312984078
:101880000297B774F7120356EAFEEBFF7901121CB8
:101890000874EB1297C15003C2E2F0E0A2E15003DA
:1018A00012984002974A74F71203561298BC029796
:1018B0004374F71203561298BC02974AEAFEEBFFF4
:1018C0007A187B0412142EEEFAEFFB1212C0227467
:1018D000F712035674EF1208DBEAFEEBFFEE241258
:1018E0001295F4121C92E9605C74098510828511CE
:1018F00083F07401120AAC74EFF012995FF874026D
:10190000120AACE8129981A3A3E0C0E07404120AA1
:10191000ACD0E012A236A3A3A3A3E0640870158E96
:10192000828F83A3A3129970E0C0E07405120AAC01
:10193000D0E080067405120AACE412A59A7406126F
:101940000AAC12994A741102886BAA82AB831213F3
:101950005C851082851183AA82AB83121CFE221241
:10196000A35312B3AC88828983E0FCA3E0F9EC2294
:10197000129977A3A3A32212997B2212B279A3A36F
:1019800022F0A3E912A21612B27522C082C08312FD
:10199000139E0293B8C082C08390044C748BF0A352
:1019A0007421F090044E7469F0A37422F0901A68C8
:1019B0007427F0A37420F0901A6A7489F0A374203D
:1019C000F09004387460F0A37412F090042FE04497
:1019D00001028D2412130E0293B874F6120356906E
:1019E000042DE07002A3E06003129A1490042DE429
:1019F000F0A3F0900431F080031214CA90042CE09C
:101A0000F91214D6EA7001EB70EF80031208497FD7
:101A1000020205AD90042D1296F51214CA2274F735
:101A2000120356E9FA7B0090042CE0F91214FA0232
:101A3000974A74F412035674F11208DB8A828B837E
:101A4000E02427F582E43422F583E493851082852F
:101A50001183F0640B700DE98A828B83A3F012135B
:101A600080029B18E07003029B18640C6003029BC9
:101A7000107403120AAC129E33EA242EF582EB1284
:101A80008FF4C0E07402120AACD0E012A584A3A3C4
:101A9000A3A37808120A6D7405120AAC12A5A18AD4
:101AA000828B83A3A3A3A3A3A3A3128562740912A9
:101AB0000AACECF0A3ED12A26050047C008011EAA5
:101AC0002411F582EB128FF4FC900484E0C39CFC9B
:101AD000740B120AACECF0EA2414F582EB128FF4CA
:101AE000C0E0740C120AACD0E0F0EA2415F582EBE9
:101AF000128FF4C0E0740D120AACD0E0F0EA2416A4
:101B0000F582EB128FF4C0E0740E120AACD0E0F054
:101B10007401120AAC12B18F740F02802FC082C000
:101B200083900431E070047901800279000293B857
:101B3000C082C083900431E06403700479018002A4
:101B400079000293B874F6120356900431129BDCAC
:101B50002466F582E9341AF583129EAAE0C2E7F002
:101B6000C333FCE82CF582E91288D7A3E493FEC3C3
:101B700033FCE433FDEC2466F582ED341AF583E0A2
:101B80007002A3E06005EE900431F08A828B83E05E
:101B9000C333FCE433FDE82CF582E93DF583E4939F
:101BA000F508C4540FC3332446F582E43404F583A6
:101BB0001280467001E9700512136E801C740F5577
:101BC00008C333FCE82CF582E9129BE893C0E0746B
:101BD0000193F583D082121E77029A0FE0C333F887
:101BE000E433F9E822F582EB129612E42274F21241
:101BF000035674FE1208DB890C8A088B09129CA418
:101C0000FA129CC37001EF60238E828F83E50CF083
:101C1000E4A3F0F50A7808120817129CB124020A0E
:101C20000A129CD2120849129C328003129CDC02D8
:101C30008071EEFAEFFB0290B174F012035674FE5D
:101C40001208DB890C8C088D09129CA4F50EEA6041
:101C5000067405250EF50EAA0E129CC37001EF60E6
